:100000000C94A10F0C94D20F0C94D20F0C94D20F1D
:100010000C94D20F0C94D20F0C94D20F0C94D20FDC
:100020000C94D20F0C94D20F0C94D20F0C94D20FCC
:100030000C94D20F0C9417760C94D20F0C94D20F10
:100040000C94D20F0C94D20F0C94D20F0C94D20FAC
:100050000C94D20F0C94D20F0C94D20F0C947C728F
:100060000C94D20F0C945BD50C9431D50C94D20F18
:100070000C94D20F0C94D20F0C94D20F0C94D20F7C
:100080000C94D20F0C94D20F0C94D20F0C94D20F6C
:100090000C9407D50C94DDD40C94D20F0C94A27759
:1000A0000C94D20F0C94D20F0C94D20F0C94D20F4C
:1000B0000C94D20F0C94D20F0C94D20F0C94D20F3C
:1000C0000C94D20F0C94D20F0C94D20F0C94B3D486
:1000D0000C9489D40C94D20F0C945FD40C9435D426
:1000E0000C94D20F084AD73B3BCE016E84BCBFFDB7
:1000F000C12F3D6C74319ABD56833DDA3D00C77FF8
:1001000011BED9E4BB4C3E916BAAAABE0000008090
:100110003F07634236B79BD8A71A39685618AEBA5C
:10012000AB558C1D3CB7CC5763BD6DEDFD753EF6F0
:10013000177231BF000000803F08000000BE92240B
:1001400049123EABAAAA2ABECDCCCC4C3E00000040
:1001500080BEABAAAAAA3E00000000BF000000803B
:100160003F0000000000084178D3BB4387D1133D16
:10017000190E3CC3BD4282AD2B3E68EC8276BED9DF
:100180008FE1A93E4C80EFFFBE01C4FF7F3F00001E
:10019000000000000C94F76F0C9473500C942CAF7B
:1001A0000C94FA540C9464AF0C94AA700C943457C9
:1001B0000C9459700C94825C0C946A700C940F70BF
:1001C0000C94DC6F0C948A540C9450500C94335E55
:1001D0000C9450AF0C94D35B0C943B570C94845408
:1001E0000C94A3610C9446AF0C94A2500C945A70DA
:1001F0000C9422B10C94E56F0C94F8630C94AF59F5
:100200000C947D700C94FC580C94F1710C94475034
:100210000C94CE500C940B700C9438610C9480713B
:100220000C947B510C94C8720C9487540C94FB78FA
:100230000C948D510C94F36F0C9405700C94FD6F1D
:100240000C94EF6F0C94405C0C94F05F0C940C6079
:100250000C946A500C9458700C94CA6F0C9493547C
:100260000C9472510C9496540C943ED70C94655592
:100270000C942A700C946F540C94D5B00C94C55007
:100280000C94D86F0C9443640C9429650C94DC7026
:100290000C94D46F0C943AAF0C9499540C94BC50B9
:1002A0000C9459640C9486640C94B3500C94275CA1
:1002B0000C9418AF0C943E500C945B700C9401702D
:1002C0000C9490540C9429500C946F620C943964E3
:1002D0000C940A700C9459500C94865C0C94C2AE29
:1002E0000C94E96F0C94D75A0C94F1620C94D97069
:1002F0000C948E640C94DC5A0C943E640C94DF6F66
:100300000C94D06F0C94776F0C9484510C94C3AE02
:100310000C94924F0C9409AF0C9469510C948D5429
:100320000C9444D80C94EB550C94B1710C943C5C37
:100330000C945AAF0C94F9624E414E494E495459AF
:10034000494E46CDCCCC3D0AD7233C17B7D13877A0
:10035000CC2B329595E6241FB14F0A0000204100B6
:1003600000C84200401C4620BCBE4CCA1B0E5AAE00
:10037000C59D7400407A10F35A00A0724E1809000F
:1003800010A5D4E80000E87648170000E40B5402FA
:100390000000CA9A3B000000E1F505000080969835
:1003A00000000040420F000000A086010000001085
:1003B0002700000000E803000000006400000000C7
:1003C000000A00000000000100000000002C76D8A8
:1003D00088DC674F0823DFC1DFAE59E1B1B796E58E
:1003E000E3E453C63AE651997696E8E6C28426EBF2
:1003F000898C9B62ED407C6FFCEFBC9C9F40F2BA05
:10040000A56FA5F490055A2AF75C936B6CF9676D9C
:10041000C11BFCE0E40D47FEF520E6B500D0ED90F1
:100420002E0300943577050080841E080000204EBE
:100430000A000000C80C333333330F986E12831157
:1004400041EF8D2114893BE65516CFFEE6DB18D12E
:10045000844B381BF77C1D901DA4BBE42420328400
:10046000725E228100C9F124ECA1E53D27236E6F65
:10047000206D61676E657469632073656E736F725A
:100480002100496E636F7272656374204D4D433570
:100490003838334D413D20004D4D43353838334DCC
:1004A000413D2000482D6669656C643A2028002093
:1004B000202020202020202020202020202020005C
:1004C000202020202020202020202020202020202C
:1004D000002020202020202020202020202020203C
:1004E000200020202020202020202020202020202C
:1004F000202000202020202020202020202020201C
:10050000202000202020202020202020202020200B
:1005100020200044233A43616C6962726174696F00
:100520006E00442A3A53657474696E6773004442DE
:100530003A5265736574204C6F6767657200444377
:100540003A436C656172204C43440043303A416D3C
:100550006D6F6E69610043393A4E697472617465FA
:100560000043383A466F7263652F4D6173730043E1
:10057000373A436F6E6475637469766974790043C2
:10058000363A446973736F6C766564204F3200436A
:10059000312D353A536C6F74312D35204F6E004438
:1005A000443A4D756C746953656E736F7273004491
:1005B000393A43757272656E7400566F6C74616778
:1005C000652B43757272656E740044383A456C65EC
:1005D00063747269630044373A4D6F74696F6E00DB
:1005E00044363A44532054656D700044353A5556AC
:1005F00020496E74656E736974790044343A4F32E1
:1006000020636F6E632E0044333A434F3220636F92
:100610006E632E0044323A504D28313A322E353A2C
:100620003130290044323A504D28313A322E353A91
:100630003130292A0044313A547572626964697410
:10064000790044303A566F6C7461676500393A6FCF
:100650007220334420616363656C2E00393A496E21
:10066000636C2E20616E672E00383A7048207661E8
:100670006C756500373A49522054656D7000373A01
:1006800049522054656D702A00363A4D61676E6597
:10069000746963206669656C6400353A476173204C
:1006A0004C6576656C00343A495220466C616D6544
:1006B00000333A4C6967687420496E742E00323AF0
:1006C000616E642048656967687400323A54656DEC
:1006D0007020507265737375726500313A54656DA0
:1006E000702048756D696469747900303A536F758C
:1006F0006E64204C6576656C00303A536F756E649D
:10070000204C6576656C2A0054696D65206C6170BB
:1007100073653A00576946692049503A00436F6E45
:1007200074726F6C002350726573732044232074BD
:100730006F20656E61626C652000442320746F2019
:10074000656E61626C6500536C6F74230050686F56
:100750006E652053656E736F7200416363656C65EF
:10076000726174696F6E004F7269656E742E2F49E5
:100770006E636C2E00416E672E2056656C6F636948
:10078000747900436F6D702E202620482D666965B0
:100790006C64004750530050726F78696D697479CA
:1007A000004C6967687420496E74656E736974796A
:1007B00000416972205072657373757265005465EB
:1007C0006D7020262048756D6964697479004D6FDD
:1007D00074696F6E00555620496E742E0055562070
:1007E000496E74656E73697479004F3220436F6E81
:1007F0006300434F3220436F6E630053656E736F27
:1008000072206572726F722100234E6F2073656EC5
:10081000736F722100434F3220436F6E63004D654A
:1008200061737572696E6700234E6F2054422073A6
:10083000656E736F723F00234E6F2073656E736F2A
:10084000722100536F756E64204C6576656C004DA7
:100850006561737572696E672E2E00234E6F20736B
:10086000656E736F722100536F756E64204C6576F0
:10087000656C00234E6F2073656E736F7220666F18
:10088000722074656D7020262068756D69646974C6
:100890007921004E6F2053656E736F7221002066C0
:1008A0006F722074656D7020262068756D696469AB
:1008B000747921002353656E736F72204572726FD5
:1008C00072200053656E736F72204572726F7221D1
:1008D000002357726F6E672073656E736F722066A8
:1008E0006F722074656D7020262068756D6964696B
:1008F0007479210057726F6E672053656E736F7243
:10090000210054656D702048756D696469747900C3
:100910004C6967687420496E74656E7369747900F8
:10092000466C616D6520495200482D6669656C64AE
:100930000053656172636820446972656374696F0E
:100940006E00234E6F2070482073656E736F7221A6
:100950000070482076616C75650023496E76616C85
:100960006964206B65792100204D756C746973652D
:100970006E736F7273004D756C746973656E736F0F
:1009800072730044697361626C6500456E61626CEC
:1009900065005265626F6F74696E672E2E2E00239C
:1009A00044413A2D323300237265706C6965733DA2
:1009B0000067657453656C66546573744269742886
:1009C000293A20006973496E7465727275707445B6
:1009D0006E61626C65642831293A2000676574494C
:1009E0006E746572727570744D617070696E67288F
:1009F00031293A2000676574496E746572727570AA
:100A000074536F757263652831293A2000676574E5
:100A1000496E74657272757074536F757263652870
:100A2000293A20006765745261746528293A203399
:100A30002E31343135393F00616363656C2E697343
:100A40004C6F77506F77657228293A200061636395
:100A5000656C2E697341736C65657028293A2000B6
:100A6000616363656C2E6973546170536F75726353
:100A7000654F6E5A28293A2000616363656C2E69C0
:100A800073546170536F757263654F6E5928293ABC
:100A90002000616363656C2E6973546170536F75D8
:100AA0007263654F6E5828293A2000616363656C54
:100AB0002E69734163746976697479536F757263D3
:100AC000654F6E5A28293A2000616363656C2E6970
:100AD000734163746976697479536F757263654F96
:100AE0006E5928293A2000697341637469766974E4
:100AF00079536F757263654F6E5828293A200069E3
:100B000073546170446574656374696F6E4F6E5A97
:100B100028293B2066616C73653F2000697354612E
:100B200070446574656374696F6E4F6E5A28293B13
:100B300020747275653F2000697354617044657458
:100B4000656374696F6E4F6E5928293B2066616C2E
:100B500073653F2000697354617044657465637404
:100B6000696F6E4F6E5928293B20747275653F205E
:100B7000006973546170446574656374696F6E4F86
:100B80006E5828293B2066616C73653F20006973AD
:100B9000546170446574656374696F6E4F6E582854
:100BA000293B20747275653F20006765745375702A
:100BB000707265737342697428293B2066616C7397
:100BC000653F20006765745375707072657373427A
:100BD000697428293B20747275653F200069734150
:100BE00063746976697479416328293A20006973CE
:100BF000496E61637469766974795A456E61626C95
:100C0000656428293A20006973496E6163746976C6
:100C100069747959456E61626C656428293A2000CF
:100C20006973496E616374697669747958456E6158
:100C3000626C656428293A2000697341637469769F
:100C40006974795A456E61626C656428293A20009E
:100C50006973416374697669747959456E61626C30
:100C6000656428293A200069734163746976697460
:100C70007958456E61626C656428293A2000676581
:100C8000744672656546616C6C4475726174696F17
:100C90006E28293A20006765744672656546616C66
:100CA0006C5468726573686F6C6428293A20006719
:100CB000657454696D65496E6163746976697479A8
:100CC00028293A2000676574496E61637469766902
:100CD00074795468726573686F6C642829200067A2
:100CE0006574416374697669747954687265736870
:100CF0006F6C6428292000676574446F75626C65A9
:100D000054617057696E646F772829200067657495
:100D1000446F75626C655461704C6174656E637983
:100D200028293A20006765745461704475726174B3
:100D3000696F6E28293A2000676574417869734F9E
:100D400066667365742826782C2026792C20267AEE
:100D5000293A20006765745461705468726573683D
:100D60006F6C6428293A200058595A2047733A205A
:100D70000058595A20434F554E54533A200073653A
:100D800074206761696E735B5D3A00206661696C0F
:100D9000656400207375636365737366756C002307
:100DA0006761696E735F6F7269675B5D3A00234CC0
:100DB0003347343230304420636F6E6E656374693C
:100DC0006F6E00756E6B6E6F776E00323030302054
:100DD0006470730035303020647073003235302019
:100DE00064707300236779726F207363616C653D73
:100DF00000234E6F204C3347343230304420677923
:100E0000726F2073656E736F722F636865636B20FA
:100E1000776972696E6721004E6F2073656E736F1C
:100E200072210049522054656D706572617475724B
:100E300065004D6561737572696E672E2E004E6F89
:100E40002073656E736F723F0049522054656D7058
:100E500065726174757265004D6561737572696E56
:100E6000672E2E00234E6F2073656E736F7220669F
:100E70006F7220504D21004E6F2073656E736F723C
:100E80002100206E672F4C00504D313A322E353AFA
:100E90003130004D6561737572696E672E2E004E9C
:100EA0006F2053656E736F7221004E6F2044532084
:100EB000546865726D6F6D657465722100445320CE
:100EC000546865726D2E004D6F74696F6E004669CF
:100ED0006E64696E672057694669204950007365E2
:100EE000703D006976616C3D006E697465723D000D
:100EF000230043616C2E204661696C656400436188
:100F00006C2E20446F6E65004E6F206E6565642107
:100F10000043616C6962726174656421004D6167B0
:100F20006E65746F6D657465720043616C696272A1
:100F3000617465202E2E36307300466F7263652013
:100F400053656E736F720043616C696272617465A0
:100F50000062756666657220736F6C6E2E320031AA
:100F60003D4F4B20303D526563616C2E00496E76DB
:100F7000616C6964206B657900313D4F4B20303DD9
:100F8000526563616C2E0062756666657220736FD0
:100F90006C6E2E3100436F6E64756374697669748C
:100FA000790043616C69627261746500496E7661B3
:100FB0006C6964206B657900313D4F4B20303D45B5
:100FC00078697400496E207361742E20736F6C6EA3
:100FD0002E00446973736F6C766564204F32004352
:100FE000616C69627261746500436F6E74726F6CDC
:100FF0002044697361626C656400436F6E74726F44
:101000006C20456E61626C656400496E76616C6946
:1010100064205028506129005365614C6576656CE9
:101020002050285061293A0043616C6962726174F2
:10103000652050004169722054656D70286F432906
:101040003A0043616C2E204D6F74696F6E004453FB
:10105000542054656D702073656E736F7200437514
:101060007272656E742073656E736F72004F3220FA
:1010700073656E736F720055562073656E736F7271
:101080000043616C696272617465004661696C65F8
:10109000640054422063616C2E20646F6E650055BD
:1010A00070706572204C696D69743A3E004C6F77C0
:1010B0006572204C696D69743A3E005475726269BC
:1010C00064697479004661696C65640070482063E6
:1010D000616C2E20646F6E65007048313020507254
:1010E000657373204200704834205072657373201A
:1010F000410043616C696272617465004E45543D04
:10110000426C7565746F6F7468204C45004E455491
:101110003D426C7565746F6F7468004E45543D5761
:101120006946690053657474696E67204661696C2D
:1011300065640053657474696E6720446F6E650062
:101140004368616E6765204E6574776F726B3E0011
:10115000547970653A0042542F57694669204E65AC
:1011600074776F726B004368616E67652053656EBC
:10117000736F723E0043757272656E742053656EB4
:10118000736F72004F7468657200496E642E20346C
:101190002D32306D4100414353373132203C3330E2
:1011A0004100414353373132203C3230410041430A
:1011B00053373132203C3541005368756E74003E20
:1011C0004D617820566F6C743A3E004368616E67DB
:1011D0006520766F6C746167653E00547970652098
:1011E00000566F6C746167652053656E736F720093
:1011F0004368616E67652053656E736F723E00438E
:10120000757272656E742053746174757300496EE3
:10121000636C416E672B416E6756656C004163637A
:10122000656C2B416E6756656C00416E672E2056CB
:10123000656C2E00496E636C2E20416E676C657381
:1012400000416363656C65726174696F6E0041751E
:10125000746F6D61746963004368616E67652074C3
:1012600079706520746F00547970653D004D616739
:101270006E657469632073656E736F720043686195
:101280006E6765207479706520746F0053656E73A6
:101290006F723D4448540054656D702048756D6907
:1012A0006469747900295C67411F856341B81E5DDC
:1012B000413D0A5741A47051410AD74B4152B846AB
:1012C000418FC24141C3F53C41E17A3841F62834AF
:1012D00041F6283041EC512C41E17A2841CDCC2413
:1012E00041AE4721418FC21D415C8F1A41295C17D5
:1012F00041EC511441AE47114166660E4114AE0BEC
:1013000041B81E09415C8F0641000004418FC201B3
:101310004152B8FE40713DFA407B14F64085EBF136
:10132000408FC2ED409A99E9408FC2E540713DE29D
:10133000406666DE4048E1DA40295CD740F628D4B2
:1013400040C3F5D040B81ECD402345432043616CD7
:101350006962726174696F6E20537563636573733C
:1013600066756C002349737375652045433D4520C0
:10137000746F205361766520616E642045786974CE
:10138000002345432043616C2E20537563636573CE
:101390007366756C2C4B3D002345432043616C699B
:1013A00062726174696F6E204661696C65640023C6
:1013B0004661696C65642C54727920416761696E7D
:1013C000006B67006C6200676D00466F72636500BA
:1013D0004D61737300282D313D6E6F6E653B303D5E
:1013E0006F6C6420484D43353838333B313D6E6572
:1013F00077204D4D43353838332900234D61676ED2
:10140000657469632053656E736F723D0028303DCB
:101410006175746F3B313D616363656C3B323D695F
:101420006E636C20616E676C653B20333D616E6757
:101430002076656C290023416363656C6572617475
:10144000696F6E20413D002354696D65206475729B
:101450006174696F6E3D002354696D6520696E7417
:10146000657276616C3D002354656D7020262048BE
:10147000756D69646974792073656E736F723A2053
:101480004448540028303D426C7565746F6F746831
:101490003B313D576946693B323D426C7565746F1F
:1014A0006F7468204C452900234E65743D00235518
:1014B00056207A65726F20766F6C74616765203D87
:1014C000002343616C69627261746564204F32204D
:1014D000636F6E63203D0023566F6C7461676520F7
:1014E00073656E6F723A00556E6B6E6F776E004962
:1014F0006E647573747269616C20342D32306D4185
:1015000000414353373132204D61783D354100234E
:1015100043757272656E742073656E736F723A00F4
:101520002354757262696469747920766F6C746192
:101530006765733A00234C434420616464726573A9
:10154000733D307800235365612D6C6576656C20A2
:1015500050726573737572653D00234F5320766535
:101560007273696F6E3A2000234D6F62696C65205B
:101570004C6F67676572204E616D653A2000534578
:1015800054002D3730002D3530002D333000696E7A
:101590007075742044535463616C69627261746540
:1015A0003A0023444F2043616C6962726174696F31
:1015B0006E204661696C65640023444F2043616C72
:1015C0006962726174696F6E2053756363657373CA
:1015D00066756C0023444F205361747572617469A1
:1015E0006F6E2043616C6962726174696F6E204630
:1015F000696E697368656421002350757420444FD7
:101600002070726F626520696E746F2073617475EB
:10161000726174696F6E206F787967656E2077618B
:101620007465722100235479706520273127206664
:101630006F72204F4B206F722027302720746F204D
:101640006578697400237363616C652066616374F7
:101650006F723D002350757420302E31306B67203F
:1016600077656967687420666F722063616C696270
:101670007261746F6E0043616C696272617465209F
:10168000302E31306B6700313D4F4B20303D457877
:10169000697400234E6F20666F7263652073656EF8
:1016A000736F722048583731312100234858373141
:1016B00031205343414C453D002368783731312078
:1016C0007363616C6520666163746F723D00485896
:1016D000373131205343414C4500235072657373B9
:1016E00020313D4F4B206F7220303D4578697400AA
:1016F000313D4F4B20303D4578697400546172652F
:101700003A4E6F20776569676874002352656D6F84
:10171000766520616C6C2077656967687420746FEA
:10172000207461726520666F72207A65726F002383
:1017300043616C6962726174696F6E20646F6E657B
:1017400000235374617274002343616C6962726197
:1017500074696F6E204D6F6465002343616C69622C
:10176000726174696F6E20636F6D706C657465640F
:101770000023526F7461746520746865206C6F6714
:1017800067657220696E20382D736861706564200A
:101790007061746820322D332074696D6573002385
:1017A00043616C6962726174696E67206D61676E16
:1017B00065746F6D6574657220666F722036307364
:1017C0002E2E2E004D4D43353838334D413D2000EF
:1017D0004D414743414C004D4147545950453D0010
:1017E000235461726520666F7263652073656E7342
:1017F0006F720054464F5243450023536574757011
:1018000020666F7263652073656E736F7200494660
:101810004F524345002343616C69627261746520D5
:10182000666F7263652073656E736F720043464F17
:10183000524345004D41535300464F524345002308
:1018400049737375652045433D5320746F2073744D
:101850006172742045432063616C696272617469CE
:101860006F6E00235075742045432070726F62655F
:101870002D3E3134313375532F636D206F7220311B
:10188000322E38386D532F636D206275666665722F
:1018900020736F6C7574696F6E0020766F6C746165
:1018A00067653D00235475726269646974792055D7
:1018B00070706572204C696D69743A200020766FF3
:1018C0006C746167653D0023547572626964697464
:1018D00079204C6F776572204C696D69743A2000ED
:1018E00023547572626964697479204C6F776572EC
:1018F000204C696D69742056696E663A20004D610E
:10190000782072616E67653D0023566F6C74616765
:10191000652073656E736F723A00342D32306D41FD
:1019200000414353373132204D61783D00414353EC
:10193000373132204D61783D354100234375727255
:10194000656E742073656E736F723A002344532082
:10195000546865726D6F6D657465722063616C6942
:1019600062726174656420666F7220230044535470
:1019700000234E6F206E65656420746F2063616C78
:101980006962726174652063757272656E7420732A
:10199000656E736F722100234143533731322063E8
:1019A000757272656E742073656E736F72206F66E8
:1019B0006673657420563D00235556207A65726F14
:1019C00020766F6C74616765203D0055565A002380
:1019D0004F3220766F6C253D00234F322063616CBF
:1019E0006962726174696F6E3A200023566F6C747D
:1019F0006167652870483D3130293A0023566F6C85
:101A0000746167652870483D34293A0050483400B5
:101A10005554454D503D004448543D004149413DD9
:101A2000004149413D00413D002354696D652064FA
:101A300075726174696F6E3D0054494D45443D00B7
:101A40002354696D6520696E74657276616C3D0022
:101A500054494D45493D00534156453D0047455485
:101A60000053484F57533D004E45543D005769467B
:101A7000692049503A0049504144440041542B00E8
:101A800041542B54595045300041542B5459504522
:101A9000310050494E3D0042543D004C43443D000E
:101AA000436F6E74726F6C2044697361626C65641D
:101AB00000436F6E74726F6C20456E61626C65647A
:101AC000004353004D533D00234D5320456E61624A
:101AD0006C656400234D532044697361626C6564D6
:101AE0000053484F574D5300235265737420706163
:101AF00072616D657465727320746F2064656661D0
:101B0000756C742076616C7565730052455345544D
:101B1000004C6F67676572204E616D653A20004C1E
:101B20004F474745520056455253494F4E00524584
:101B3000424F4F540052534C4F5400534C4F543D5E
:101B400000697465726174696F6E3D0073656E73D0
:101B50006F72233D0043757272656E7420737461F9
:101B60007475733A206379636C653D006E637963C5
:101B70006C653D006E73656E736F72733D006D61D1
:101B8000786E73656E736F72733D00656E61626C23
:101B900065643D00234D756C746973656E736F7277
:101BA00073206D6561737572656D656E7420736504
:101BB0007474696E67733A002353657474696E6751
:101BC00073206F6620616C6C2073656E736F727327
:101BD0003A002353697A65206F6620686561646501
:101BE00072202B20616C6C2073656E736F72733A78
:101BF00020002353697A65206F66206865616465FB
:101C0000723A20004F6666206169722D636F6E64C0
:101C100021004974277320746F6F20636F6F6C21EC
:101C20000054656D702069732066696E65210049F6
:101C300073206169722D636F6E64206F6E3F00497F
:101C400074277320717569746520686F7421004969
:101C5000742773207665727920686F742120004F95
:101C60006666206169722D636F6E64210049742776
:101C70007320746F6F20636F6F6C210054656D70FB
:101C80002069732066696E6521004973206169725D
:101C90002D636F6E64206F6E3F004974277320714F
:101CA0007569746520686F74210049742773207604
:101CB00065727920686F74210054656D70204875D5
:101CC0006D6964697479002320616E6420726561B6
:101CD000647920746F207573652100206D6F6269CF
:101CE0006C65206C6F6767657220737461727465D0
:101CF00064200043616C6962726174696F6E205088
:101D0000726573737572653D00536561206C65760D
:101D1000656C20502863616C63293D002345727215
:101D20006F723A707265737375726520424D5030F0
:101D300038352C20636865636B20776972696E673C
:101D4000210049522054656D702073656E736F7267
:101D500020666F756E6400206D6F62696C65206C23
:101D60006F67676572207374617274696E67202E85
:101D70002E2E2000576946692049503A00235769A2
:101D8000466920495020616464726573733A20008B
:101D90002323205345534C6F67676572202323002C
:101DA0002323202057656C636F6D6520202323005B
:101DB0004C434420616464726573733D3078005312
:101DC000656E736F7220736C6F7420616E64207423
:101DD0007970653A00005EBCE2613FDD83C29C7EA3
:101DE00020A3FD1F41009D23BE46DB65F88C11AF8B
:101DF00032CA57E97400002100240027002A002D70
:101E0000003000330001010000040107010A010055
:101E1000002200250028002B002E00310034000293
:101E2000010000050108010B01000020002300262D
:101E30000029002C002F00320000010000030106E1
:101E40000109010505050507050808080802020241
:101E5000020A0A0808040404040101010101010145
:101E6000010303030303030303040707070C0C0C1C
:101E70000C0C0C0C0C0202020206060606060606F4
:101E8000060B0B0B0B0B0B0B0B0102102020080891
:101E900010204010204080020102010804020101CC
:101EA00002040810204080804020100804020180B5
:101EB000040201804020100804020108040201010C
:101EC0000204081020408001020408102040800015
:101ED000000A0B02090C0D0E0807030401000000A4
:101EE00000000000000000000000000000000000F2
:101EF00000000000000000000000001211100000AF
:101F000000000000000000000000000000000000D1
:101F1000000000000023456E64206F66204D756C44
:101F2000746973656E736F72204379636C65230007
:101F3000496E76616C6964206B657921000044D834
:101F40003ED711241FBECFEFD1E2DEBFCDBF00E0F0
:101F50000CBF1BE0A0E0B2E0E6E8F6ED01E00BBF4D
:101F600002C007900D92A23EB107D9F725E1A2EE7B
:101F7000BBE001C01D92AD38B207E1F71FE0C0EA37
:101F8000DFE000E006C021970109802FFE010E94DA
:101F900051E8CF39D10780E00807A9F70E947FDB1D
:101FA0000C9431EB0C9400000F931F93CF93DF93AD
:101FB000CDB7DEB7A2970FB6F894DEBF0FBECDBF88
:101FC0008E010B5E1F4F682FC8010E94EB751887AA
:101FD0000F831D821E82198289E08A8381E08B83B0
:101FE0008C831C8A1B8ACE0101960E944075CE010B
:101FF00001960E94E37360E0CE0101960E94D474C2
:10200000A2960FB6F894DEBF0FBECDBFDF91CF9181
:102010001F910F9108950F931F9360E08091A60484
:102020000E94837183E090E00197F1F761E0809175
:10203000A6040E94837183E290E00197F1F760E0CB
:102040008091A6040E9483718091A4049091A504BC
:102050009927FC01E757F14E6491FC01ED5BF14ECD
:10206000E491F0E0EE0FFF1FE75DF14E8591949152
:1020700000E717E120E030E0462F0E9485D561158A
:1020800071058105910529F06F5F7F4F8F4F9F4F3D
:102090009F700E942DE320E030E44CE156E40E9462
:1020A000A5E52091340C3091350C4091360C5091BF
:1020B000370C0E948CE320E030E048E453E40E94B7
:1020C000A5E51F910F910895CF92DF92EF92FF92B5
:1020D0000E940B106B017C0120E030E040E050E4F6
:1020E0000E94AEE6181624F40E940B106B017C01CE
:1020F00020E030E040E050E4C701B6010E94AEE6C7
:10210000181624F40E940B106B017C0120E030E0D3
:1021100040E050E4C701B6010E94AEE6181624F470
:102120000E940B106B017C0120E030E040E050E4A5
:10213000C701B6010E94AEE6181624F40E940B10E7
:102140006B017C0120E030E040E050E4C701B601C3
:102150000E94AEE618162CF4C12CD12CE12C80E4A0
:10216000F82EC701B601FF90EF90DF90CF90089551
:10217000CF93DF9320919D042223A9F02091FB04AB
:10218000222389F0EC016FED88E795E10E94D4CD20
:102190008C819D81892B39F0BE0188E795E1DF9123
:1021A000CF910C94F1D3DF91CF91089580919D044C
:1021B000882349F08091FB04882329F060E088E7B8
:1021C00095E10C94FB7808950F931F93CF93DF93C1
:1021D0008C011092390C1092380CC091380CD091AF
:1021E000390CC832D105A4F4809106020E94F57121
:1021F000CC0FDD1FC25AD14F998388838091380C50
:102200009091390C01969093390C8093380CE5CF5E
:102210000E947AB220E030E040EA50E40E948CE371
:1022200020E030E040E85AE30E948CE304301105DE
:1022300099F420E030E040E650E40E948CE39B01FA
:10224000AC0160E070E080E890E40E94C6E4DF91B9
:10225000CF911F910F9108950A30110569F420E084
:1022600030E040E650E40E948CE39B01AC0160E06A
:1022700070E080E291E4E9CF60E070E0CB01E7CF6D
:1022800023E333E948E853E40E94A5E520E030E089
:1022900040E85FE30E94C7E40E94CFE726E636EA03
:1022A00045EA53E40E948CE36093340C7093350C40
:1022B0008093360C9093370C089581E08093FB0453
:1022C00080919D04882341F088E08093831560E02D
:1022D00088E795E10C94C978089580919D04811157
:1022E00010C081E080939D048093FB0480917E1553
:1022F000982F946090937E158C600E943CB20C9451
:102300005D118091FB048823D1F31092831560E066
:1023100088E795E10E94C9781092FB0480917E15B0
:102320008B7F80937E1588600E943CB210929D0442
:1023300008952F923F924F925F926F927F928F9269
:102340009F92AF92BF92CF92DF92EF92FF920F9344
:102350001F93CF93DF936C01C7E6D5E085EB882E02
:1023600084E0982E03E412E1EE24E394F12C22E1C0
:10237000222E312C33E1432E512C40E1642E712C5E
:1023800051E1A52EB12C8091B3049091B4048E1527
:102390009F050CF4C7C021E0C216D10409F0BBC0F0
:1023A000F80182AD93ADF40191838083F4018081C3
:1023B0009181009711F58A819B819093050280930A
:1023C0000402F401819191914F0184309105C1F58E
:1023D0002A813B81309307022093060285319105C3
:1023E00009F478C08631910509F040C02A813B810B
:1023F00030938A04209389044EC08130910539F4CA
:102400008A819B8190939F0480939E04DACF8230CF
:10241000910539F48A819B81909303028093020293
:10242000D0CF039771F68A819B81909301028093AC
:10243000000263E97BE08DE794E10E9457C8C1CFB9
:102440008530910539F42A813B81309388042093AB
:102450008704C4CF8630910529F287309105B9F4FD
:102460002A813B8130938E0420938D04873191051E
:1024700091F42A813B812830310599F57092A704A7
:102480006092A604B092A504A092A40404C08A306D
:10249000910509F0A3CF9C012B5031092A30310559
:1024A00090F42A813B81309301022093000239E1AC
:1024B000389FB001399F700D1124625F7D4F8DE709
:1024C00094E10E94BAC88FEFE81AF80A22960E5FCC
:1024D0001F4F59CF2A813B8130938C0420938B046A
:1024E000DACF2730310549F43092A7042092A604B0
:1024F0005092A5044092A404CECF2630310559F65F
:1025000021E030E03093A7042093A6041092A504A4
:102510001092A404C0CFF40180819181F80193AF9F
:1025200082AF44CFDF91CF911F910F91FF90EF9039
:10253000DF90CF90BF90AF909F908F907F906F90E3
:102540005F904F903F902F9008954F925F926F92BF
:102550007F929F92AF92BF92CF92DF92EF92FF92C3
:102560000F931F93CF93DF93982E8EE0A82EB12C5C
:10257000EE24EA9493E0F92E0FEF13E0D12CC12C56
:10258000D0E0C0E0412C512C3201892D0E94F57120
:10259000C817D90708F44AC0C816D90608F46C0150
:1025A0008017910708F444C08E159F0508F47C013C
:1025B000BC0190E080E00E942BE39B01AC01C301D1
:1025C000B2010E94C7E42B013C0165E070E080E0AD
:1025D00090E00E943D7281E0A81AB108B1F6BE01F8
:1025E0006C0D7D1D6E0D7F1D600F711F90E080E0F2
:1025F0000E942BE39B01AC01C301B2010E94C6E41F
:1026000020E030E040E251E40E94A5E5DF91CF9167
:102610001F910F91FF90EF90DF90CF90BF90AF9000
:102620009F907F906F905F904F900895EC01B8CF8E
:102630008C01BECFCF92DF92EF92FF92CF93C091E9
:102640007212C4304CF4C1300CF04BC0CC2359F1A1
:1026500060E070E0CB013FC0C430D1F70E94A5120A
:1026600020E030E040EA50E40E948CE320E030ECCF
:102670004FE754E40E94A5E520E030E040EA50E452
:102680000E94A5E520E030E040E851E40E948CE3A0
:1026900020E030E040E850E40E94C7E420E030E071
:1026A0004AE754E416C00E94A51220E030E040EA58
:1026B00050E40E948CE320E030EC4FE754E40E94A9
:1026C000A5E52091731230917412409175125091CA
:1026D00076120E94A5E5CF91FF90EF90DF90CF900A
:1026E00008950E94A5122AE137E64CE950E40E94C1
:1026F0008CE32091731230917412409175125091B5
:1027000076120E94C6E46B017C01EC2FEE0FFF0BEA
:10271000E15AFA4F60817181072E000C880B990BEA
:102720000E942DE39B01AC01C701B601D2CF1F93DC
:10273000CF93DF93182FCEE5DEE0812F0E94F57155
:10274000899399936CE370E080E090E00E943D7281
:102750008EE0CE3AD80789F70E947AB220E030E0C6
:1027600040EA50E40E948CE320E030E040E85AE385
:102770000E948CE3DF91CF911F910895CF93DF9357
:10278000FC0124813581232B99F0EC01BC018DEFF4
:102790009EE00E94FFD36EE170E080E090E00E9436
:1027A0003D72BE0184ED90E1DF91CF910C94FFD397
:1027B000DF91CF910895CF93DF93FC012481358180
:1027C000232B69F0EC01BC0184ED90E10E94F1D370
:1027D000BE018DEF9EE0DF91CF910C94F1D3DF919C
:1027E000CF91089580919D048823F9F08091FB0496
:1027F0008823D9F081E00E943CB28BE39FE10197EE
:10280000F1F760E080E00E944DB263E075E088E798
:1028100095E10E9411D461E080E00E944DB263EF27
:1028200074E088E795E10C9411D40895EF92FF923B
:102830000F931F93CF93DF9320919D04222309F4DC
:1028400061C02091FB04222309F45CC08A01EB01E2
:102850007C01209719F1C095D09561E08C2F0E94E2
:102860004DB2B70188E795E10E94F1D362EE74E0C2
:1028700088E795E10E9411D4F701848161E08C0F13
:102880000E944DB2B801110F880B990BDF91CF91C7
:102890001F910F91FF90EF900C943D720E94707207
:1028A000AB01BC018091F20B9091F30BA091F40B62
:1028B000B091F50B8C599F4FAF4FBF4F84179507C1
:1028C000A607B707F8F461E080E00E944DB2B701B7
:1028D00088E795E10E94F1D361ED74E088E795E126
:1028E0000E9411D461E0F70184810E944DB20E94E0
:1028F00070726093F20B7093F30B8093F40B9093D0
:10290000F50BC0CFDF91CF911F910F91FF90EF900A
:102910000895FF920F931F93CF93DF93EC01F62E50
:1029200008811981C8010E944DE4F81621F06F2D2D
:10293000C8010E9455E4CE01DF91CF911F910F9104
:10294000FF900895DC01ED91FC910190F081E02D64
:1029500019948F929F92AF92BF92CF92DF92EF9293
:10296000FF920F931F93CF93DF938C01862F0B3031
:10297000110509F092C090919014992309F0F894F0
:1029800062E10E94D3C3EC0180919014882309F086
:102990007894209701F180E090ECA9E7B4EC809363
:1029A000831490938414A0938514B0938614809319
:1029B000871490938814A0938914B0938A14CE3FFF
:1029C0008FEFD80709F49DC0CF3FDC0709F4EFC1B2
:1029D000CCEFDFEF24C1C0918B14E0908C146E2DEE
:1029E00070E090E080E00E942DE32DEC3CEC4CEC9C
:1029F0005DE30E948CE34B015C016C2F70E090E082
:102A000080E00E942DE39B01AC01C501B4010E944E
:102A1000C7E4609383147093841480938514909317
:102A20008614D0918D14F0908E146D2F6F7770E016
:102A300090E080E00E942DE34B015C016F2D70E07F
:102A400090E080E00E942DE32DEC3CEC4CEC5DE34B
:102A50000E948CE39B01AC01C501B4010E94C7E454
:102A6000D7FD19C0609387147093881480938914DC
:102A700090938A14CE0DCD0FCF0D81E090E0209180
:102A80008F14C21302C090E080E0892B09F487C044
:102A9000CFEFDFEF8CC19058E5CFCFEFDFEF0631FE
:102AA000110509F0BCC090919014992309F0F89495
:102AB00061E00E94D3C3EC0180919014882309F057
:102AC0007894209709F180E090ECA9E7B4EC80932A
:102AD000831490938414A0938514B09386148093E8
:102AE000871490938814A0938914B0938A14CF3FCD
:102AF000DC0709F45CC1209709F451C0229609F063
:102B000067CFCEEFDFEF8BC0C0918C14D0918B14C8
:102B100060918B1470918C1476276727762790E04C
:102B200080E00E942BE32DEC3CEC4CEC5DE30E943A
:102B30008CE3609383147093841480938514909332
:102B40008614E0908E14F0908D146F2D6F77762F91
:102B50006E2D90E080E00E942BE32DEC3CEC4CECE1
:102B60005DE30E948CE3F7FC18C0609387147093B8
:102B700088148093891490938A148C2F8D0F8E0D56
:102B80008F0DC1E0D0E090918F14891302C0D0E086
:102B9000C0E0D195C195D109AACF9058E6CFC09099
:102BA0008314D0908414E0908514F090861420E073
:102BB00030E048EC52E4C701B6010E94AEE6D0E036
:102BC000C0E0181614F4CBEFDFEF20E030E0A901ED
:102BD000C701B6010E9426E387FF02C0CAEFDFEFFC
:102BE000C0908714D0908814E0908914F0908A14D3
:102BF00020E030E048EC52ECC701B6010E9426E329
:102C000087FF02C0C9EFDFEF20E030E040EF52E481
:102C1000C701B6010E94AEE618160CF4C3C00C3012
:102C2000110509F0C4C08CE50E9432B270E060E08A
:102C30008BE294E10E94A2148BE294E10E94C67898
:102C400065E08CE50E943FB610925B0E80935A0EB1
:102C5000C82FD0E0209709F4A8C0C530D1050CF4E6
:102C6000B6C00DE21DE00E942CB6F80180870F5F10
:102C70001F4FC8018D529D408C179D07A4F3C09132
:102C8000350D0091360D602F70E090E080E00E94DD
:102C90002DE32DEC3CEC4CEC5DE30E948CE36B01EE
:102CA0007C016C2F70E090E080E00E942DE39B019E
:102CB000AC01C701B6010E94C7E46B017C01C09260
:102CC0002D0DD0922E0DE0922F0DF092300DD0915F
:102CD000370D1091380D6D2F6F7770E090E080E028
:102CE0000E942DE34B015C01612F70E090E080E0D9
:102CF0000E942DE32DEC3CEC4CEC5DE30E948CE358
:102D00009B01AC01C501B4010E94C7E4D7FD5DC0C1
:102D10006093310D7093320D8093330D9093340D89
:102D2000C00FCD0FC10F8091390DC813B1CE20E077
:102D300030E048EC52E4C701B6010E94AEE6D0E0B4
:102D4000C0E0181614F4CBEFDFEF20E030E040EAEB
:102D500050E4C701B6010E9426E387FF02C0CAEF14
:102D6000DFEFC090310DD090320DE090330DF09038
:102D7000340D20E030E040EF51ECC701B6010E9475
:102D800026E387FF02C0C9EFDFEF20E030E040EF2D
:102D900052E4C701B6010E94AEE6181644F4C8EF2B
:102DA000DFEF05C0C8EFDFEF3ACFCEEFDFEFCE01A8
:102DB000DF91CF911F910F91FF90EF90DF90CF9017
:102DC000BF90AF909F908F9008959058A1CFCDEF76
:102DD000DFEFEDCFCF93DF93EC019A01AB01E889F0
:102DE000F98982E08083211581EE3807410551057C
:102DF00081F160E079E08DE390E00E9495E421505C
:102E00003109410951095695479537952795EC8524
:102E1000FD851082EE85FF852083188EEC89FD8963
:102E200086E08083EA89FB89808180618083EA89EA
:102E3000FB89808188608083EA89FB898081806842
:102E40008083EA89FB8980818F7D8083DF91CF91A8
:102E50000895E889F989108220E1D9CF2F923F9215
:102E60004F925F926F927F928F929F92AF92BF929A
:102E7000CF92DF92EF92FF920F931F93CF93DF9346
:102E8000CDB7DEB766970FB6F894DEBF0FBECDBFE5
:102E90001C0187E390E10E944DB540E855E260E0F7
:102EA00070E087E390E10E94EA1664E670E080E05B
:102EB00090E00E943D728CED95E0A0E0B0E0809340
:102EC0003B1090933C10A0933D10B0933E1064E6ED
:102ED00070E080E090E00E943D728FEF8A8781E091
:102EE0008B8786E88C871D861E861F86188A198A1E
:102EF00089E78A8BC101880F991F9E8B8D8BD12CFE
:102F0000C12CF12CE12C412C512C320187E390E1B2
:102F10000E9409AF08974CF049E050E0BE01665F9F
:102F20007F4F87E390E10E94C3AE65E070E080E0F0
:102F300090E00E943D7210E000E0812C912C540141
:102F400087E390E10E943AAF892B39F4F4E08F16C1
:102F50009104A104B1040CF04EC0023011050CF034
:102F60004AC087E390E10E943AAF892B69F087E37A
:102F700090E10E9418AFE1E0F0E0EC0FFD1FE00FE0
:102F8000F11F80830F5F1F4F65E070E080E090E0ED
:102F90000E943D720230110509F073C099818A8543
:102FA00098136FC09A818C8598136BC0FE0133967D
:102FB000FC8BEB8B87E390E10E943AAF892B39F4CD
:102FC000F4E08F169104A104B1040CF053C0093051
:102FD000110509F05CC08B8190E0982F88272C8127
:102FE000820F911D092E000CAA0BBB0B480E591E17
:102FF0006A1E7B1E43C08FEFC81AD80AE214F3047E
:1030000034F4ED89FE89EC15FD0509F07FCF87E3E7
:1030100090E10E944DB5E114F10409F47101C3017E
:10302000B2010E942DE34B015C01B701FF0C880B3C
:10303000990B0E942DE39B01AC01C501B4010E94D4
:10304000A5E566960FB6F894DEBF0FBECDBFDF9143
:10305000CF911F910F91FF90EF90DF90CF90BF9095
:10306000AF909F908F907F906F905F904F903F9028
:103070002F900895043011050CF0ADCFFFEFEF1A3B
:10308000FF0A8FEF881A980AA80AB80A59CF87E36F
:1030900090E10E9418AFEB89FC898193FC8BEB8B4C
:1030A0000F5F1F4F87CF4F925F926F927F92AF92C9
:1030B000BF92CF92DF92FF920F931F93CF93DF9334
:1030C00000D000D0CDB7DEB75C0187E390E10E946D
:1030D0004DB540E052EC61E070E087E390E10E9482
:1030E000EA168CED95E0A0E0B0E080933B10909361
:1030F0003C10A0933D10B0933E1064E670E080E079
:1031000090E00E943D72D12CC12CF12C65E070E062
:1031100080E090E00E943D7210E000E0412C512CD4
:103120003201F1103AC087E390E10E943AAF892B57
:1031300031F485E1481651046104710474F50330DB
:1031400011055CF587E390E10E943AAF892B69F0A5
:1031500087E390E10E9418AFE1E0F0E0EC0FFD1F83
:10316000E00FF11F80830F5F1F4F65E070E080E08C
:1031700090E00E943D72023011054CF089818B3B3A
:1031800031F4FF24F3948A818A3A09F0F12C8FEF0D
:10319000481A580A680A780AC4CF8FEFC81AD80AA2
:1031A00064E670E080E090E00E943D72AC14BD04E3
:1031B00009F0ACCF8F2D26960FB6F894DEBF0FBE68
:1031C000CDBFDF91CF911F910F91FF90DF90CF90F6
:1031D000BF90AF907F906F905F904F900895CF9386
:1031E000DF93EC01FB01248135810E948ACBCE0163
:1031F000DF91CF910895CF92DF92EF92FF920F93DC
:103200001F93CF93DF93CDB7DEB762970FB6F894D5
:10321000DEBF0FBECDBF2091FE0C222309F4D8C023
:103220002091230D3091240D263531050CF0D0C0AE
:103230004091950450919604493D5F400CF0C8C000
:103240008C012F5F3F4F3093240D2093230D0E945C
:103250007072C090F60CD090F70CE090F80CF090E3
:10326000F90C6C197D098E099F090E942BE320E05F
:1032700030E04AE754E40E94A5E56093FA0C7093AD
:10328000FB0C8093FC0C9093FD0C80919504909125
:1032900096048835924034F488E592E09093960441
:1032A0008093950480919504909196043AEFE32ED3
:1032B0003CE0F32E9C012A5F3C406901C6018E0D63
:1032C0009F1D9A838983F70161917F01CE01019649
:1032D0000E948914FEEFEF16FCE0FF0679F780915B
:1032E0009504909196040496909396048093950487
:1032F000B801CE0101960E9470CBCE0101960E94CA
:1033000042CABC01CE010D960E9470CBCE0101963F
:103310000E94E3CAF80184819581849708F123E231
:1033200030E050E040E0B801CE0101960E948ACB27
:10333000BE016F5F7F4FCE0107960E9470CBCE011A
:1033400007960E9442CABC01CE010D960E9487CA10
:10335000CE0107960E94E3CACE0101960E94E3CAFD
:1033600049895A894115510549F08FEF9CE0009732
:1033700029F0BC01CE010D960E9400B58091950404
:103380009091960423E2C22E2DE0D22E0FEF1CE086
:103390009C012F5F3C407901C701800F911F9A83E8
:1033A0008983F80161918F01CE0101960E948914F1
:1033B000C016D10689F78091950490919604849661
:1033C0009093960480939504CE010D960E94E3CAD3
:1033D00062960FB6F894DEBF0FBECDBFDF91CF91DE
:1033E0001F910F91FF90EF90DF90CF900895AF92D3
:1033F000BF92CF92DF92EF92FF920F931F93CF93E2
:10340000DF93CDB7DEB762970FB6F894DEBF0FBE7D
:10341000CDBF20919D04222309F447C02091FB04D5
:10342000222309F442C07A016B015C010E94707290
:10343000AB01BC018091EE0B9091EF0BA091F00BD2
:10344000B091F10B8C599F4FAF4FBF4F8417950729
:10345000A607B70750F560E08FEFC816D806B1F59C
:1034600080E00E944DB200E0B50188E795E10E943E
:10347000F1D360EC74E088E795E10E9411D4F50186
:10348000848160E0800F0E944DB20E947072609350
:10349000EE0B7093EF0B8093F00B9093F10BB70151
:1034A000FF0C880B990B0E943D7262960FB6F89440
:1034B000DEBF0FBECDBFDF91CF911F910F91FF9067
:1034C000EF90DF90CF90BF90AF90089580E00E9482
:1034D0004DB20E94707228EE33E040E050E00E944E
:1034E00063E4CA01B90120E831E541E050E00E94FF
:1034F00063E4AB01BC01CE0101960E9461C8BE012C
:103500006F5F7F4FCE0107960E9470CB64ED7AE02B
:10351000CE0107960E94DBC9BC01CE010D960E9428
:1035200070CBCE0107960E94E3CACE0101960E949D
:10353000E3CABE01635F7F4F88E795E10E94F1D344
:1035400009891A89C114D10431F00C0D1D1D60E0E8
:10355000802F0E944DB2CE010D960E94E3CA84CF07
:10356000BF92CF92DF92EF92FF920F931F93CF9370
:10357000DF93CDB7DEB762970FB6F894DEBF0FBE0C
:10358000CDBF6C018B017A0180919D04882369F184
:103590008091FB04882349F160E00F3F1007A9F5F3
:1035A00080E00E944DB200E0B60188E795E10E94FC
:1035B000F1D36FEA74E088E795E10E9411D4F60137
:1035C000848160E0800F0E944DB20E94707260930F
:1035D000EE0B7093EF0B8093F00B9093F10BB70110
:1035E000FF0C880B990B0E943D7262960FB6F894FF
:1035F000DEBF0FBECDBFDF91CF911F910F91FF9026
:10360000EF90DF90CF90BF90089580E00E944DB280
:103610000E94707228EE33E040E050E00E9463E4C4
:10362000CA01B90120E831E541E050E00E9463E4BD
:10363000AB01BC01CE0101960E9461C8BE016F5F63
:103640007F4FCE0107960E9470CB64ED7AE0CE01E9
:1036500007960E94DBC9BC01CE010D960E9470CB7B
:10366000CE0107960E94E3CACE0101960E94E3CAEA
:10367000BE01635F7F4F88E795E10E94F1D3B9886F
:1036800060E08B2D0E944DB20115110531F40B2D18
:10369000CE010D960E94E3CA87CF60E0802F0E9482
:1036A0004DB2F6CFCF93DF93EC01483085E0580759
:1036B0006105710509F448C008F099C0493481E0FA
:1036C00058076105710509F4B2C008F040C04434E0
:1036D00081E058076105710509F476C000F54134B1
:1036E00081E058076105710509F456C048F440347B
:1036F00051406105710509F4E4C063E97BE0E3C072
:10370000423481E058076105710509F409C1433469
:1037100051406105710589F76FEE7AE0D4C04634F7
:1037200081E058076105710509F40CC108F49FC0D8
:10373000473481E058076105710509F455C04834E4
:10374000514061057105C9F66CED75E0BCC04230B1
:1037500085E058076105710509F4E2C000F54437BA
:1037600081E058076105710509F4F2C040F4423761
:1037700051406105710509F66BED77E0A4C0411574
:1037800085E058076105710509F49BC0413055403B
:103790006105710509F0B1CF65EF7AE094C045305D
:1037A00085E058076105710509F461C080F4433074
:1037B00085E058076105710509F4AECF44305540E6
:1037C0006105710509F099CF68EE7AE07CC046305A
:1037D00085E058076105710509F4B4C047305540CC
:1037E0006105710509F089CF6AED75E06CC04D3B4C
:1037F00082E458078FEF6807710509F4AFC008F03D
:1038000048C04F3E80E158078FEF6807710561F3AC
:10381000F8F4423385E058076105710509F4ACCF2F
:1038200048F4493055406105710509F066CF6EEDE9
:1038300075E049C0443385E058076105710509F416
:1038400087C04D3F52406F4F710509F495CF55CF5A
:103850004D3D82E258078FEF6807710509F478C083
:1038600048F4473E58416F4F710509F046CF65EE69
:103870007AE029C04F3C80E358078FEF6807710555
:1038800009F4A2CF473C58436F4F710509F45CCF50
:1038900034CF473988E658078FEF6807710509F478
:1038A0007BCF48F54D3A82E558078FEF68077105E1
:1038B00009F451C078F4453B5A446F4F710509F043
:1038C0001CCF65EC77E0CE010E9479CBCE01DF9171
:1038D000CF910895453A8AE558078FEF680771053B
:1038E00009F4A5CF4D3952466F4F710509F005CF48
:1038F0006FEE78E0E8CF473588EA58078FEF680722
:10390000710519F180F445388AE758078FEF680789
:103910007105C1F0473658496F4F710509F0EDCE7A
:1039200062EF7AE0D0CF4F3480EB58078FEF680713
:10393000710509F4F1CE4D33524C6F4F710509F406
:103940001BCFDBCE68ED75E0BECF62E678E0BBCF83
:1039500068E678E0B8CF68E379E0B5CF67EE77E066
:10396000B2CF3F924F925F926F927F928F929F92CF
:10397000AF92BF92CF92DF92EF92FF920F931F937D
:10398000CF93DF93CDB7DEB7EB970FB6F894DEBFDA
:103990000FBECDBF2B013C018AE99FE00E944DB5CF
:1039A00064E670E080E090E00E943D7240E855E2FD
:1039B00060E070E08AE99FE00E94EA1664E670E049
:1039C00080E090E00E943D7263E97EE08AEE93E140
:1039D0000E9462CA6AEE73E1CE0101960E9470CB2A
:1039E00042E350E06FEF7FEFCE0101960E94B01AE4
:1039F000CE0101960E94E3CA68E87EE08AEE93E178
:103A00000E9462CA6AEE73E1CE0101960E9470CBF9
:103A100042E350E06FEF7FEFCE0101960E94161453
:103A2000CE0101960E94E3CA8091440D9091450D0C
:103A30008D7F312CD12CC12CF12CE12C10E000E039
:103A4000019709F47AC09E01205E3F4F39AF28AF3D
:103A5000CE014E969BAF8AAF0E94707264197509B1
:103A600086099709683B7B408105910508F065C090
:103A70008AE99FE00E943AAF892B09F44DC08CED92
:103A800095E0A0E0B0E080939E0F90939F0FA093ED
:103A9000A00FB093A10F0E944FB497FD3DC0823498
:103AA0009105C9F7DE0111964D015D010E944FB4E9
:103AB00097FF39C089818D3479F590E080E0D40199
:103AC0002D914D01820F911DEAADFBADAE17BF07E1
:103AD000B1F78E5B9F4F2E8D30E0322F22274F8D16
:103AE000240F311D82179307B9F40C8110E0102FB9
:103AF00000278D81080F111DEE80F12CFE2CEE2485
:103B00008F81E80EF11CC884D12CDC2CCC24898553
:103B1000C80ED11C3324339462E370E080E090E05F
:103B20000E943D7299CFD5018D935D01E8ADF9AD4D
:103B3000AE17BF0709F0BACFBDCF0E9470726419EB
:103B4000750986099709683B7B408105910510F44A
:103B50003110BBC00E94F2136AEE73E1CE01809671
:103B60000E9470CB42E350E066E070E0CE018096A8
:103B70000E94B01ACE0180960E94E3CA332009F455
:103B8000CCC082E090E09093450D8093440DB60147
:103B9000CE01C2960E948EC8B701CE018C960E94BB
:103BA0008EC8B801CE0180960E948EC8BE01605EAC
:103BB0007F4FCE0186960E9470CB6EE477E0CE01F7
:103BC00086960E94DBC9BE01645D7F4F0E94F1C9E9
:103BD0006EE477E00E94DBC9BE016E5C7F4F0E94FD
:103BE000F1C9BC0180EF93E10E9487CACE0186969D
:103BF0000E94E3CACE0180960E94E3CACE018C9651
:103C00000E94E3CACE01C2960E94E3CA60EF73E14C
:103C1000CE0180960E9470CB4AE050E06FEF7FEFBC
:103C2000CE0180960E941614CE0180960E94E3CAAF
:103C300062E87EE088E795E10E9411D4B601CE01EA
:103C4000C2960E948EC8B701CE018C960E948EC883
:103C5000B801CE0186960E948EC860EE75E0CE0156
:103C600080960E9479CBBE016A5D7F4FCE0180961F
:103C70000E94F1C962E277E00E94DBC9BE01645D87
:103C80007F4F0E94F1C962E277E00E94DBC9BE016A
:103C90006E5C7F4F0E94F1C960EF75E00E94DBC946
:103CA000BC0180EF93E10E9487CACE0180960E94FA
:103CB000E3CACE0186960E94E3CACE018C960E948A
:103CC000E3CACE01C2960E94E3CA62E370E080E0DC
:103CD00090E00E943D728AE99FE00E944DB562E348
:103CE00070E080E090E00E943D72EB960FB6F89491
:103CF000DEBF0FBECDBFDF91CF911F910F91FF901F
:103D0000EF90DF90CF90BF90AF909F908F907F907B
:103D10006F905F904F903F90089567E77EE080EF4F
:103D200093E10E9462CA60EF73E1CE0180960E9427
:103D300070CB4AE050E070E060E0CE0180960E94D7
:103D40001614CE0180960E94E3CA64E67EE080EFFE
:103D500093E10E9462CA8091440D9091450D0297B3
:103D600009F0B3CF1092450D1092440DAECF0F93D2
:103D70001F93CF93DF9300D000D0CDB7DEB7209153
:103D8000D00D2223A9F08C0168E379E0CE010196E1
:103D90000E9479CBB801CE0101960E94F1C9BC0105
:103DA00084ED90E10E94FFD3CE0101960E94E3CA08
:103DB00026960FB6F894DEBF0FBECDBFDF91CF9130
:103DC0001F910F910895CF93DF93CDB7DEB72C9756
:103DD0000FB6F894DEBF0FBECDBF8130910509F05C
:103DE0006EC09093BA128093B9126BE171E1CE016B
:103DF00001960E9467CBCE0101960E94B71ECE01AC
:103E000001960E94E3CA66EF75E0CE0101960E941A
:103E100079CB60E675E1CE0101960E94F1C9BC0143
:103E2000CE0107960E9470CB48EC50E06FEF7FEF19
:103E3000CE0107960E94B01ACE0107960E94E3CAEF
:103E4000CE0101960E94E3CA8DEF9EE00E944DB51F
:103E500040E052EC61E070E08DEF9EE00E94EA16D7
:103E600090E080E00E94D6B465E076E0CE01019655
:103E70000E9479CB6CE675E1CE0101960E94F1C9F2
:103E8000BC01CE0107960E9470CB40ED57E06FEF6A
:103E90007FEFCE0107960E941614CE0107960E946E
:103EA000E3CACE0101960E94E3CA81E02C960FB6C8
:103EB000F894DEBF0FBECDBFDF91CF91089500977C
:103EC000E1F51092BA121092B9126DE071E1CE01D3
:103ED00001960E9467CBCE0101960E94B71ECE01CB
:103EE00001960E94E3CA6CEF75E0CE0101960E9434
:103EF00079CB60E675E1CE0101960E94F1C9BC0163
:103F0000CE0107960E9470CB48EC50E06FEF7FEF38
:103F1000CE0107960E94B01ACE0107960E94E3CA0E
:103F2000CE0101960E94E3CA8DEF9EE00E944DB53E
:103F300040E855E260E070E08FCF82309105A9F44F
:103F40009093BA128093B9126CEF70E1CE01019692
:103F50000E9467CBCE0101960E94B71ECE0101964A
:103F60000E94E3CA60E076E0C0CF80E09FCFBF92BE
:103F7000CF92DF92EF92FF920F931F93CF93DF9335
:103F8000CDB7DEB762970FB6F894DEBF0FBECDBFD8
:103F90008C016B0162E277E0CE010D960E9479CB35
:103FA00060EF7EE0C8010E9467CB76012FEFE21A36
:103FB000F20AB701CE0101960E948EC8BE016F5F62
:103FC0007F4FCE0107960E9470CB6EE477E0CE0162
:103FD00007960E94DBC9BC01C8010E945BCACE01E2
:103FE00007960E94E3CACE0101960E94E3CA8AE0C6
:103FF000B82EBE9CC001BF9C900D1124FC01E6515F
:10400000FD4E7F018081082E000C990B0E94C0EAB2
:10401000892B09F4B2C0B701CE0101960E9479CB79
:10402000BE016F5F7F4FCE0107960E9470CB6FEC91
:104030007AE0CE0107960E94DBC9BC01C8010E944C
:104040005BCACE0107960E94E3CACE0101960E9488
:10405000E3CABC9CC001BD9C900D11249C0126515B
:104060003D4E7901F9016685062E000C770BCE01D5
:1040700001960E948EC8BE016F5F7F4FCE010796EA
:104080000E9470CB64EB7BE0CE0107960E94DBC9F7
:10409000BE01635F7F4F0E94F1C9BC01C8010E944D
:1040A0005BCACE0107960E94E3CACE0101960E9428
:1040B000E3CA69EE7EE0C8010E9404CAF701678581
:1040C000062E000C770BCE0101960E948EC8BE0111
:1040D0006F5F7F4FCE0107960E9470CBBE01635F7A
:1040E0007F4FCE0107960E94F1C9BC01C8010E9412
:1040F0005BCACE0107960E94E3CACE0101960E94D8
:10410000E3CA63EE7EE0C8010E9404CAF701608939
:104110007189CE0101960E948EC8BE016F5F7F4FEC
:10412000CE0107960E9470CBBE01635F7F4FCE0128
:1041300007960E94F1C9BC01C8010E945BCACE016A
:1041400007960E94E3CACE0101960E94E3CA6EED73
:104150007EE0C8010E9404CAF70162897389CE011A
:1041600001960E948EC8BE016F5F7F4FC8010E94FA
:104170005BCACE0101960E94E3CACE010D960E9451
:10418000E3CAC80162960FB6F894DEBF0FBECDBF7A
:10419000DF91CF911F910F91FF90EF90DF90CF9023
:1041A000BF9008954F925F926F927F929F92AF92CD
:1041B000BF92CF92DF92EF92FF920F931F93CF9314
:1041C000DF93CDB7DEB7A9970FB6F894DEBF0FBE69
:1041D000CDBF982E882351F08091D00D882331F0E7
:1041E00063E97BE084ED90E10E94C2CD0E947AC534
:1041F00060E08DE20E94B8C460E18DE20E94B8C424
:1042000068E08DE20E94B8C48091C9129091CA12F0
:1042100097FD63C010E000E01092ED0D1092EE0DDE
:104220001092EF0D1092F00D1092F10D1092F20D10
:104230001092F30D1092F40D1092F50D1092F60DF0
:104240001092F70D1092F80D1092050E1092F90DC4
:104250001092FA0D1092FB0D1092FC0D1092FD0DB4
:104260001092FE0D1092FF0D1092000E1092010E92
:104270001092020E1092030E1092040E1092060E6F
:104280001092070E1092080E1092090E0E947AC525
:1042900089E60E9432B26FE08BE294E10E94AA703C
:1042A0008BE294E10E94C67889E60E9432B241E036
:1042B00050E069E670E08BE294E10E9412790E947E
:1042C0002CB6F82E8BE294E10E94C67883EDF816A6
:1042D000A1F10431110509F054C6992009F4ADC0CB
:1042E0008091330C811153C04090931450909414DA
:1042F0006090951470909614498E5A8E6B8E7C8EB9
:10430000C0909714D0909814E0909914F0909A145B
:10431000CD8EDE8EEF8EF8A280919B1490919C142E
:10432000A0919D14B0919E148EA39FA3A8A7B9A796
:1043300089A39AA3ABA3BCA3ABC06FEA80E20E949F
:1043400063C560E081E20E9463C568E082E20E948A
:1043500063C560E283E20E9463C589E29CE5AFE841
:10436000BDE380930A0E90930B0EA0930C0EB093B6
:104370000D0E60E084E20E9463C50431110509F46A
:10438000ACCF81E08093330C992009F456C064EEE1
:104390007DE0CE0101960E9467CBCE0101960E947E
:1043A000DB13CE0101960E94E3CA89E60E9432B275
:1043B00063E28BE294E10E94AA708BE294E10E9496
:1043C000C67889E60E9432B241E050E069E670E0CA
:1043D0008BE294E10E94127990915A0E80915B0ECB
:1043E0009817F1F30E942CB68C018BE294E10E94A5
:1043F000C678C80124E0959587952A95E1F78370E2
:10440000992764ED7DE08130910559F06BEC7DE0FA
:104410008230910531F06CED7DE0892B11F063EC79
:104420007DE0CE0101960E9467CBCE0101960E94ED
:10443000BE13CE0101960E94E3CA4090931450909F
:1044400094146090951470909614498E5A8E6B8EC9
:104450007C8EC0909714D0909814E0909914F090AE
:104460009A14CD8EDE8EEF8EF8A280919B149091DF
:104470009C14A0919D14B0919E148EA39FA3A8A7F5
:10448000B9A789A39AA3ABA3BCA3992009F44CC0F4
:104490006EEA7DE084ED90E10E9411D48091330CAE
:1044A00063E97DE0811102C06BE87DE084ED90E17D
:1044B0000E9411D484ED90E10E94BECD6FE97DE0B1
:1044C000CE0101960E9467CBCE0101960E94B71ED5
:1044D000CE0101960E94E3CA8E01075E1F4F5E0166
:1044E00095E2A90EB11CD8016D917D918D919D91A0
:1044F0008D0146E050E00E94BDCE62E277E084ED9F
:1045000090E10E941BCF0A151B0569F763E97BE068
:10451000CE0101960E9479CBCE0101960E94B71E72
:10452000CE0101960E94E3CA23E938E144E85FE343
:10453000C301B2010E948CE32B013C014D865E86D3
:104540006F86788A22E430E645E85FE3C701B6016A
:104550000E948CE36B017C01C98ADA8AEB8AFC8AAF
:1045600025E83BEE41E95FE36EA17FA188A599A50F
:104570000E948CE36D8B7E8B8F8B988F409293146F
:10458000509294146092951470929614C09297145D
:10459000D0929814E0929914F0929A1460939B141C
:1045A00070939C1480939D1490939E14992009F409
:1045B000A2C08091D00D882309F49DC06EE77DE0F4
:1045C000CE0101960E9467CBCE0101960E94B71ED4
:1045D000CE0101960E94E3CA8E01035F1F4F6E0158
:1045E000B9E1CB0ED11C7801F801619171918191F3
:1045F00091918F0142E050E00E94BDCE62E277E0EF
:1046000084ED90E10E941BCFC016D10669F763E9E3
:104610007BE0CE0101960E9479CBCE0101960E94EB
:10462000B71ECE0101960E94E3CA4FE954E166E04D
:1046300070E082E30E945EC4A0909F14B090A0142A
:10464000C090A114D090A2140091A3141091A414AE
:1046500061E77DE084ED90E10E9411D44AE050E0F2
:10466000B50184ED90E10E94CECE62E277E084ED68
:1046700090E10E941BCF4AE050E0B60184ED90E14A
:104680000E94CECE62E277E084ED90E10E941BCFE3
:104690004AE050E0B80184ED90E10E94CECE63E99B
:1046A0007BE084ED90E10E94C2CDCE0101960E9494
:1046B000FAC468E67DE084ED90E10E9411D48E0199
:1046C0000F5F1F4FD8016D917D918D919D918D014F
:1046D0004AE050E00E94BDCE62E277E084ED90E1D6
:1046E0000E941BCF0E151F0569F763E97BE084ED7F
:1046F00090E10E94C2CD61E08DE10E94B8C4992092
:10470000B1F08091D00D882391F064E57DE084EDD7
:1047100090E10E9411D4AE014B5D5F4F61E070E00B
:104720008DE10E945EC48DA190E00E9408CF62E0FE
:104730008EE10E94B8C463E08FE10E94B8C464E0D7
:1047400080E20E94B8C4992009F450C08091D00D35
:10475000882309F44BC068E37DE084ED90E10E947A
:1047600011D4AE014B5D5F4F61E070E08EE10E94BD
:104770005EC4CDA0D12CAE014B5D5F4F61E070E017
:104780008FE10E945EC4EDA0F12CAE014B5D5F4F46
:1047900061E070E080E20E945EC40DA110E04AE09A
:1047A00050E0B60184ED90E10E94CECE62E277E067
:1047B00084ED90E10E941BCF4AE050E0B70184ED08
:1047C00090E10E94CECE62E277E084ED90E10E941B
:1047D0001BCF4AE050E0B80184ED90E10E94CECEBC
:1047E00063E97BE084ED90E10E94C2CD65E081E267
:1047F0000E94B8C49920B1F08091D00D882391F027
:1048000065E27DE084ED90E10E9411D4AE014B5D44
:104810005F4F61E070E081E20E945EC48DA190E094
:104820000E9408CF66E082E20E94B8C49920B1F0ED
:104830008091D00D882391F06DE07DE084ED90E1D2
:104840000E9411D4AE014B5D5F4F61E070E082E2E7
:104850000E945EC48DA190E00E9408CF67E083E2D1
:104860000E94B8C49920B1F08091D00D882391F0B6
:1048700067EF7CE084ED90E10E9411D4AE014B5DC6
:104880005F4F61E070E083E20E945EC48DA190E022
:104890000E9408CF68E084E20E94B8C49920B1F079
:1048A0008091D00D882391F06FED7CE084ED90E154
:1048B0000E9411D4AE014B5D5F4F61E070E084E275
:1048C0000E945EC48DA190E00E9408CF69E085E25D
:1048D0000E94B8C49920B1F08091D00D882391F046
:1048E00065EC7CE084ED90E10E9411D4AE014B5D5B
:1048F0005F4F61E070E085E20E945EC48DA190E0B0
:104900000E9408CF6AE086E20E94B8C49920B1F004
:104910008091D00D882391F06FEA7CE084ED90E1E6
:104920000E9411D4AE014B5D5F4F61E070E086E202
:104930000E945EC48DA190E00E9408CF6BE088E2E7
:104940000E94B8C49920B1F08091D00D882391F0D5
:1049500066E97CE084ED90E10E9411D4AE014B5DEC
:104960005F4F61E070E088E20E945EC48DA190E03C
:104970000E9408CF6CE089E20E94B8C4992009F433
:1049800079C08091D00D882309F474C06EE77CE073
:1049900084ED90E10E9411D4AE014B5D5F4F61E068
:1049A00070E089E20E945EC48DA190E00E9408CF71
:1049B00067E67CE084ED90E10E9411D466E070E04F
:1049C00087E20E949DC490E00E9408CF60E57CE0F1
:1049D00084ED90E10E9411D465E070E087E20E94CE
:1049E0009DC490E00E9408CF69E37CE084ED90E1F3
:1049F0000E9411D464E070E087E20E949DC490E0C0
:104A00000E9408CF60E27CE084ED90E10E9411D426
:104A100062E070E087E20E949DC490E00E9408CFAF
:104A200067E07CE084ED90E10E9411D461E070E0E9
:104A300087E20E949DC490E00E9408CF6EEE7BE06A
:104A400084ED90E10E9411D470E060E087E20E9462
:104A50009DC490E00E9408CF6DED7BE084ED90E175
:104A60000E9411D463E070E087E20E949DC490E050
:104A70000E9408CF41E067E070E087E20E94CFC467
:104A800041E063E070E087E20E94CFC441E063E070
:104A900070E08AE20E94CFC4992091F08091D00DFD
:104AA000882371F064EC7BE084ED90E10E9411D4E6
:104AB00063E070E08AE20E949DC490E00E9408CF0B
:104AC00040E063E070E08AE20E94CFC4992091F058
:104AD0008091D00D882371F06AEA7BE084ED90E14B
:104AE0000E9411D463E070E08AE20E949DC490E0CD
:104AF0000E9408CF41E062E070E08AE20E94CFC4E9
:104B0000992091F08091D00D882371F06EE87BE0C0
:104B100084ED90E10E9411D462E070E08AE20E948C
:104B20009DC490E00E9408CF40E062E070E08AE21D
:104B30000E94CFC4992091F08091D00D882371F00C
:104B400061E77BE084ED90E10E9411D462E070E0C7
:104B50008AE20E949DC490E00E9408CF41E061E09B
:104B600070E08AE20E94CFC4992091F08091D00D2C
:104B7000882371F065E57BE084ED90E10E9411D41B
:104B800061E070E08AE20E949DC490E00E9408CF3C
:104B900040E061E070E08AE20E94CFC4992091F089
:104BA0008091D00D882371F068E37BE084ED90E183
:104BB0000E9411D461E070E08AE20E949DC490E0FE
:104BC0000E9408CF41E070E060E08AE20E94CFC41A
:104BD000992091F08091D00D882371F06CE17BE0F9
:104BE00084ED90E10E9411D470E060E08AE20E94BE
:104BF0009DC490E00E9408CF40E070E060E08AE24F
:104C00000E94CFC4992091F08091D00D882371F03B
:104C10006FEF7AE084ED90E10E9411D470E060E0E3
:104C20008AE20E949DC490E00E9408CF41E066E0C5
:104C300070E087E20E94CFC441E065E070E087E267
:104C40000E94CFC441E064E070E087E20E94CFC4DC
:104C500040E062E070E087E20E94CFC440E061E0A3
:104C600070E087E20E94CFC440E070E060E087E23D
:104C70000E94CFC4992009F475C08091D00D88237B
:104C800009F470C067EE7AE084ED90E10E9411D4DF
:104C900066E070E08BE20E949DC490E00E9408CF25
:104CA00069EC7AE084ED90E10E9411D465E070E057
:104CB0008BE20E949DC490E00E9408CF6BEA7AE0EC
:104CC00084ED90E10E9411D464E070E08BE20E94D8
:104CD0009DC490E00E9408CF62E97AE084ED90E103
:104CE0000E9411D462E070E08BE20E949DC490E0CB
:104CF0000E9408CF69E77AE084ED90E10E9411D428
:104D000061E070E08BE20E949DC490E00E9408CFB9
:104D100060E67AE084ED90E10E9411D470E060E0FA
:104D20008BE20E949DC490E00E9408CF6DE47AE07F
:104D300084ED90E10E9411D463E070E08BE20E9468
:104D40009DC490E00E9408CF68E37AE084ED90E192
:104D50000E9411D464E070E08CE20E949DC490E057
:104D60000E9408CF40E064E070E08CE20E94CFC473
:104D7000AE014B5D5F4F61E070E08CE20E945EC46B
:104D80006DA1607F66608CE20E94B8C4992009F42E
:104D900064C08091D00D882309F45FC064E27AE09A
:104DA00084ED90E10E9411D4AE014B5D5F4F61E054
:104DB00070E08CE20E945EC46DA16F706650770B4C
:104DC000072E000C880B990B0E942DE39B01AC0170
:104DD00060E070E080E090E40E9479E720E030E05D
:104DE00048EC50E40E948CE30E94BFCE6DE07AE074
:104DF00084ED90E10E9411D4AE014B5D5F4F61E004
:104E000070E080E30E945EC44DA150E070E060E07D
:104E10002AE084ED90E10E9472CD84ED90E10E9441
:104E2000BECD65EF79E084ED90E10E9411D461E0A0
:104E300070E080E30E949DC490E00E9408CF6CED7A
:104E400079E084ED90E10E9411D461E070E08FE29E
:104E50000E949DC490E00E9408CF41E061E070E0B4
:104E60008FE20E94CFC4992091F08091D00D8823C9
:104E700071F064EC79E084ED90E10E9411D461E07E
:104E800070E08EE20E949DC490E00E9408CF41E055
:104E900061E070E08EE20E94CFC440E067E070E025
:104EA00081E30E94CFC4992009F455C08091D00DB0
:104EB000882309F450C061EB79E084ED90E10E9411
:104EC00011D467E070E081E30E949DC490E00E94ED
:104ED00008CF6AE076E084ED90E10E941BCFAE013E
:104EE0004B5D5F4F61E070E080E00E945EC48DA189
:104EF0000E94077763E97BE084ED90E10E94C2CDD8
:104F00000DE110E069E679E084ED90E10E941BCFAD
:104F100040E150E0B80184ED90E10E94CECE6EE019
:104F200076E084ED90E10E941BCFAE014B5D5F4FB8
:104F300061E070E0802F0E945EC48DA10E9407771F
:104F400063E97BE084ED90E10E94C2CD0F5F1F4FCB
:104F50000A331105B9F6A9960FB6F894DEBF0FBE55
:104F6000CDBFDF91CF911F910F91FF90EF90DF9018
:104F7000CF90BF90AF909F907F906F905F904F9039
:104F80000895992091F08091D00D882371F061EF00
:104F90007DE0CE0101960E9467CBCE0101960E9472
:104FA000BE13CE0101960E94E3CA64E670E080E081
:104FB00090E00E943D720F5F1F4F2EC94F925F928B
:104FC0006F927F928F929F92AF92BF92CF92DF9219
:104FD000EF92FF921F93CF93DF93CDB7DEB72C975D
:104FE0000FB6F894DEBF0FBECDBF182F8091EC0C2A
:104FF0008111D2C080E492E090930902809308026C
:105000000E94C67280932E1581E492E00E94C672BF
:1050100080932F1582E492E00E94C672809330152F
:1050200083E492E00E94C6728093311580E492E09E
:105030000E94C6728F3FE1F0E0900802F0900902F2
:1050400032E3A32E35E1B32E6501C7018E5295419F
:105050004C0126E3C21625E1D20609F441C0C40181
:105060008C0D9D1D0E94C672F60181936F01F1CFD8
:1050700081E492E00E94C6728F3FF1F682E492E0F2
:105080000E94C6728F3FC1F683E492E00E94C6720E
:105090008F3F91F680E090E0A0E8BFE380932E156B
:1050A00090932F15A0933015B09331152EE2C22E98
:1050B00025E1D22EF12CE12C809108029091090279
:1050C000E4E0EE16F10409F4B7CFF60161916F0147
:1050D0008E0D9F1D0E9455E4FFEFEF1AFF0AECCFE3
:1050E000C70104960E94C6728F3F99F5C7010596C5
:1050F0000E94C6728F3F69F5C70106960E94C6726C
:105100008F3F39F5C70107960E94C6728F3F09F598
:1051100080E090E0A0E8BFE38093321590933315D0
:10512000A0933415B0933515F12CE12CF501619164
:105130005F01809108029091090204968E0D9F1DD7
:105140000E9455E4FFEFEF1AFF0A24E0E216F10493
:1051500069F780912E1590912F15A0913015B0917F
:10516000311580932A1590932B15A0932C15B0938D
:105170002D150E9470726093E80C7093E90C809377
:10518000EA0C9093EB0C81E08093EC0C68EE73E0FA
:1051900080E090E00E943D728091E00C81110DC092
:1051A0000E9470726093DC0C7093DD0C8093DE0CB7
:1051B0009093DF0C81E08093E00C0E947072C090AD
:1051C000DC0CD090DD0CE090DE0CF090DF0C6C1964
:1051D0007D098E099F09693E73408105910508F498
:1051E0004BC10E9470726093DC0C7093DD0C809355
:1051F000DE0C9093DF0C8BE30E94F571BC01990FDC
:10520000880B990B0E942DE320E030E040E85AE340
:105210000E948CE320E030E44CE955E40E948CE3EA
:105220006B017C01C092D80CD092D90CE092DA0CC0
:10523000F092DB0C87E390E00E94D40F4B015C01FD
:1052400080920A0290920B02A0920C02B0920D0280
:1052500020E030E04AE754E4C701B6010E948CE345
:1052600020E030E04DE454E40E94A5E520E030E089
:1052700048E453E40E94A5E56B017C01C0923E1511
:10528000D0923F15E0924015F092411520912A15D9
:1052900030912B1540912C1550912D150E948CE3C7
:1052A0002B013C0120E030E040E250E40E94AEE6F9
:1052B00018160CF02AC18091321590913315A091E7
:1052C0003415B091351580932A1590932B15A09322
:1052D0002C15B0932D1520912A1530912B15409146
:1052E0002C1550912D15C701B6010E948CE36B015E
:1052F0007C0120E030E048EC51E4C501B4010E949B
:10530000C6E420E53DE847E95CE30E948CE320E049
:1053100030E040E85FE30E94C7E49B01AC01C701B5
:10532000B6010E94A5E5AB01BC0140932615509340
:105330002715609328157093291522E0CE01079652
:105340000E94EBCA61E176E0CE0101960E9479CB22
:10535000BE01695F7F4FCE0101960E94F1C965E1F0
:1053600076E00E94DBC9BC018AEE93E10E9487CA05
:10537000CE0101960E94E3CACE0107960E94E3CABD
:1053800040910A0250910B0260910C0270910D0243
:1053900021E0CE0107960E94EBCA60E976E0CE01DB
:1053A00001960E9479CBBE01695F7F4FCE010196C5
:1053B0000E94F1C9BC0186EF93E10E9487CACE0129
:1053C00001960E94E3CACE0107960E94E3CA6AEEE4
:1053D00073E1CE0101960E9470CB62E277E0CE01CC
:1053E00001960E94DBC966EF73E10E94F1C96BE18F
:1053F00076E00E94DBC9BC0180EF93E10E9487CA7E
:10540000CE0101960E94E3CA66EF73E1CE010196D8
:105410000E9470CB4AE050E06FEF7FEFCE01019623
:105420000E94B01ACE0101960E94E3CA65E070E0C6
:1054300080E090E00E943D726FEE78E0CE01019630
:105440000E9479CBCE0101960E94B810CE01019640
:105450000E94E3CA6AEE73E1CE0101960E9470CB0E
:105460004AE050E06FEF7FEFCE0101960E941614E4
:10547000CE0101960E94E3CA0E947072C090E80CAF
:10548000D090E90CE090EA0CF090EB0C6C197D09DF
:105490008E099F096235734081059105E0F00E94F5
:1054A00070726093E80C7093E90C8093EA0C90930F
:1054B000EB0C87E390E00E94D40F60930A02709394
:1054C0000B0280930C0290930D026EE170E080E07D
:1054D00090E00E943D7211112BC010E0812F2C969C
:1054E0000FB6F894DEBF0FBECDBFDF91CF911F91F5
:1054F000FF90EF90DF90CF90BF90AF909F908F90F4
:105500007F906F905F904F90089520E030E040E0F2
:1055100050E4C301B2010E9426E387FFDCCE8091F4
:105520002E1590912F15A0913015B0913115CBCE3D
:1055300080900A0290900B02A0900C02B0900D0295
:105540004090D80C5090D90C6090DA0C7090DB0C25
:105550004092361550923715609238157092391571
:1055600080923A1590923B15A0923C15B0923D1551
:10557000123059F0133009F431C1113009F0ADCFB8
:105580001093D70C1092D60CA9CF8091D70C8823FA
:1055900009F4A3CFC0903E15D0903F15E090401580
:1055A000F090411526E636E646E65FE3C701B60110
:1055B0000E94AEE618160CF0B3C023E333E343EFCA
:1055C0005FE3C701B6010E9426E387FFA9C020E080
:1055D00030E048EC51E4C501B4010E94C6E420E586
:1055E0003DE847E95CE30E948CE320E030E040E8DE
:1055F0005FE30E94C7E42FE23DED44EB5FE30E94CE
:105600008CE36093D20C7093D30C8093D40C909362
:10561000D50C20E038E240E258E46091D20C709161
:10562000D30C8091D40C9091D50C0E948CE320E097
:1056300030E04AE754E40E94A5E5A30192010E94EC
:10564000A5E54B015C0120E030E040E05FE30E9413
:10565000AEE618160CF0B0C020E030E040EC5FE39E
:10566000C501B4010E9426E387FFA6C080922A15D7
:1056700090922B15A0922C15B0922D1526E636E6A9
:1056800046E65FE3C701B6010E94AEE618160CF0CD
:1056900075C023E333E343EF5FE3C701B6010E9424
:1056A00026E387FF6BC080922E1590922F15A09253
:1056B0003015B092311581E08093D60C61E873E12A
:1056C000CE0101960E9467CBCE0101960E94DB13AA
:1056D000CE0101960E94E3CA40912A1550912B15E4
:1056E00060912C1570912D1523E0CE0101960E943A
:1056F000EBCACE0101960E94BE13CE0101960E9414
:10570000E3CA64E673E1CE0101960E9467CBCE0145
:1057100001960E94BE13CE0101960E94E3CADECE1E
:1057200020E030E040E151E4C701B6010E94AEE65E
:1057300018160CF06ECF26E636E646E851E4C701AF
:10574000B6010E9426E387FF64CF20E030E048ECFA
:1057500051E4C501B4010E94C6E420E53DE847E9F3
:105760005CE30E948CE320E030E040E85FE30E94CD
:10577000C7E42BE734E14EE451E441CF20E030E0D0
:1057800040E151E4C701B6010E94AEE618160CF0E4
:1057900092CF26E636E646E851E4C701B6010E94FC
:1057A00026E387FF88CF8092321590923315A0921E
:1057B0003415B09235157FCF1092D60C6FEA73E195
:1057C000CE0101960E9467CBCE0101960E94BE13C6
:1057D000CE0101960E94E3CA15E180CE8091D70CDC
:1057E000882309F47ACE84ED90E10E94BECD8091A9
:1057F000D60C882309F47DC0C0903E15D0903F158B
:10580000E0904015F090411526E636E646E65FE367
:10581000C701B6010E94AEE61816ECF523E333E3A8
:1058200043EF5FE3C701B6010E9426E387FF33C061
:105830009EE2C92E95E1D92EF12CE12CF601619161
:105840006F0180910802909109028E0D9F1D0E94A8
:1058500055E4FFEFEF1AFF0A24E0E216F10471F7B6
:105860001092D60C1092D70C1A3008F444C068E994
:1058700073E11E3109F032CECE0101960E9467CB52
:10588000CE0101960E94BE13CE0101960E94E3CA8A
:105890001092F50C23CE20E030E040E151E4C70146
:1058A000B6010E94AEE61816DCF626E636E646E8B5
:1058B00051E4C701B6010E9426E387FFD1CF82E3FE
:1058C000C82E85E1D82EF12CE12CF60161916F01F3
:1058D000809108029091090204968E0D9F1D0E94EE
:1058E00055E4FFEFEF1AFF0A24E0E216F10469F72E
:1058F000B7CF1EE1B5CF133009F0F0CD69E473E105
:10590000BBCFCF92DF92EF92FF920F931F93CF9373
:10591000DF93CDB7DEB72C970FB6F894DEBF0FBE7E
:10592000CDBFD82E0DB71EB78091C60C811105C012
:105930000E94707281E08093C60C8091BE0C811130
:1059400005C00E94707281E08093BE0C8091B60CFD
:10595000811105C00E94707281E08093B60C60E0F6
:105960008D2D0E94B57164E670E080E090E00E94A9
:105970003D721092B50C1092B40CE090B40CF09003
:10598000B50C8EE1E816F104D4F48D2D0E94F5716A
:10599000F701EE0FFF1FE858F34F918380836EE10C
:1059A00070E080E090E00E943D728091B40C909194
:1059B000B50C01969093B50C8093B40CDECF87E3C1
:1059C00090E00E94D40F60937F04709380048093D2
:1059D000810490938204E8E7FCE02AE33CE0D901EB
:1059E0009CE0E43BF90729F0819191918D939D937F
:1059F000F7CF8EE190E09093770C8093760C4DB7C3
:105A00005EB7EDB7FEB7FC970FB6F894FEBF0FBEBA
:105A1000EDBFADB7BEB711967D0180E0F901619190
:105A200071919F01F701619371937F018F5F8E31B7
:105A3000A9F78DE190E0FD0130E020E0281739075B
:105A40007CF4608171812F5F3F4FE280F380E61626
:105A5000F70624F4F182E082738362833296EECFFC
:105A6000019749F75E966D917C915F975C968D9159
:105A70009C91680F791F77FF02C06F5F7F4F75950C
:105A800067950FB6F8945EBF0FBE4DBF072E000C92
:105A9000880B990B0E942DE320E030E44CE955E49B
:105AA0000E948CE320E030EC4FE754E40E94A5E52F
:105AB0006B017C01C092F00CD092F10CE092F20CE0
:105AC000F092F30C20E030E040E05FE36091250DC0
:105AD0007091260D8091270D9091280D0E94C7E4AA
:105AE0000E9451E6FB01EE0FFF1FEE0FFF1FEB556B
:105AF000FD4E2591359145915491C701B6010E9403
:105B00008CE32091290D30912A0D40912B0D50915D
:105B10002C0D0E94A5E5AB01BC014093CE0C509327
:105B2000CF0C6093D00C7093D10C22E0CE0107967D
:105B30000E94EBCA6BE276E0CE0101960E9479CB1F
:105B4000BE01695F7F4FCE0101960E94F1C96FE2ED
:105B500076E00E94DBC9BC018AEE93E10E9487CA0D
:105B6000CE0101960E94E3CACE0107960E94E3CAC5
:105B700040917F045091800460918104709182046F
:105B800021E0CE0107960E94EBCA60E976E0CE01E3
:105B900001960E9479CBBE01695F7F4FCE010196CD
:105BA0000E94F1C9BC0186EF93E10E9487CACE0131
:105BB00001960E94E3CACE0107960E94E3CA6AEEEC
:105BC00073E1CE0101960E9470CB66EF73E1CE01C6
:105BD00001960E94F1C965E376E00E94DBC9BC0131
:105BE00080EF93E10E9487CACE0101960E94E3CA2A
:105BF00066EF73E1CE0101960E9470CB4AE050E05F
:105C000070E060E0CE0101960E94B01ACE010196CC
:105C10000E94E3CA65E070E080E090E00E943D727F
:105C20006FEE78E0CE0101960E9479CBCE0101960D
:105C30000E94B810CE0101960E94E3CA6AEE73E199
:105C4000CE0101960E9470CB4AE050E06FEF7FEFEB
:105C5000CE0101960E941614CE0101960E94E3CA5D
:105C60000FB6F8941EBF0FBE0DBF2C960FB6F8945A
:105C7000DEBF0FBECDBFDF91CF911F910F91FF907F
:105C8000EF90DF90CF9008952F923F924F925F92C6
:105C90006F927F928F929F92AF92BF92CF92DF923C
:105CA000EF92FF920F931F93CF93DF93CDB7DEB7A1
:105CB00068970FB6F894DEBF0FBECDBF2B013C0135
:105CC0000E9470726D877E878F87988B8AE99FE02C
:105CD0000E944DB562E370E080E090E00E943D726A
:105CE00061E08091A6040E94B57160E08091A404F7
:105CF0000E94B57164E670E080E090E00E943D7221
:105D00006091A0047091A1048091A2049091A304D9
:105D10000E9440110E9464107B018C010E94187245
:105D20004B015C0160E570E080E090E00E943D7214
:105D300065E476E080EF93E10E9457C820E030E010
:105D40004AE754E4C301B2010E948CE36D8B7E8B61
:105D50008F8B988F412C512C320160E070E0CB0189
:105D60000E942DE32D893E894F89588D0E9426E39C
:105D700087FF87C10E9470722D853E854F855889A7
:105D8000621B730B840B950B0E942BE320E030E029
:105D90004AE754E40E94A5E5AB01BC0123E0CE0133
:105DA00001960E94EBCABE016F5F7F4F8AEE93E1BE
:105DB0000E949ECACE0101960E94E3CA0E9464100E
:105DC000D62EC72E382E292E0E941872698B7A8BF8
:105DD0008B8B9C8BDC01CB0188199909AA09BB0923
:105DE0004C015D0191ED891697E09906A104B1047B
:105DF000BCF020E030E0A9016D2D7C2D832D922D8B
:105E00000E94AEE6181684F426EA3BE944EC5BE314
:105E10006D2D7C2D832D922D0E9426E387FF10C0CF
:105E2000812C912C54012EC026EA3BE944EC5BEB1B
:105E30006D2D7C2D832D922D0E94AEE6181684F3D5
:105E4000C501B40128EE33E040E050E00E9463E475
:105E5000CA01B9010E942DE34B015C019701A80121
:105E60006D2D7C2D832D922D0E94C6E420E030E024
:105E70004AE754E40E948CE3A50194010E94A5E541
:105E80004B015C016AEE73E1CE0101960E9470CB7A
:105E900063E477E0CE0101960E94DBC9BC018AEE83
:105EA00093E10E9487CACE0101960E94E3CA23E0D3
:105EB0004D2D5C2D632D722DCE0101960E94EBCAF3
:105EC000BE016F5F7F4FCE0107960E9470CB63E6E5
:105ED00076E0CE0107960E94DBC9BC0184EE93E117
:105EE0000E9487CACE0107960E94E3CACE0101969E
:105EF0000E94E3CA22E0B501A401CE0107960E94E8
:105F0000EBCA67EA77E0CE0101960E9479CB6AEE90
:105F100073E1CE0101960E94F1C966E676E00E9427
:105F2000DBC964EE73E10E94F1C966E178E00E948A
:105F3000DBC9BE01695F7F4F0E94F1C96AE676E066
:105F40000E94DBC9BC0180EF93E10E945BCACE01D5
:105F500001960E94E3CACE0107960E94E3CA20E0A0
:105F600030E0A901C501B4010E94AEE687FD06C07C
:105F700062E277E084EE93E10E9451CA22E0B5012B
:105F8000A401CE0101960E94EBCABE016F5F7F4F54
:105F9000CE0107960E9470CB6AE676E0CE010796A6
:105FA0000E94DBC9BC0184EE93E10E945BCACE0172
:105FB00007960E94E3CACE0101960E94E3CA60EFF1
:105FC00073E1CE0101960E9470CBCE0101960E9432
:105FD000BE13CE0101960E94E3CAC301B20125E0BF
:105FE00030E040E050E00E9463E4672B682B692BAF
:105FF00021F567EC7EE0CE0101960E9467CB45E07B
:1060000050E070E060E0CE0101960E94B01ACE012F
:1060100001960E94E3CA64EE73E1CE0101960E94EC
:1060200070CB45E050E06FEF7FEFCE0101960E940C
:106030001614CE0101960E94E3CA63E97BE080EF6B
:1060400093E10E9457C862E370E080E090E00E9414
:106050003D720E9470722D853E854F855889621B66
:10606000730B840B950B3FEF431A530A630A730AB1
:1060700089889A88AB88BC88ED2CFC2C032D122DC6
:106080006FCE60E08091A6040E94B57168960FB64D
:10609000F894DEBF0FBECDBFDF91CF911F910F915E
:1060A000FF90EF90DF90CF90BF90AF909F908F9038
:1060B0007F906F905F904F903F902F9008958F92B8
:1060C0009F92AF92BF92CF92DF92EF92FF920F9387
:1060D0001F93CF93DF93CDB7DEB7EA970FB6F8944F
:1060E000DEBF0FBECDBFF82E63E97BE0CE01C596C3
:1060F0000E9479CB8E010B5E1F4F6F2DC8010E944D
:10610000EB7518870F831D821E82198289E08A83AE
:1061100081E08B838C831C8A1B8ACE0101960E94AE
:106120004075CE0101960E94E373CE0101960E9454
:1061300036C60E8110E00330110509F488C16DEBFD
:106140007EE0CE01C5960E9462CA63E97BE080EFE3
:1061500093E10E9457C8BE016B5C7F4FCE018396CE
:106160000E9470CB4AE050E070E060E0CE01839680
:106170000E94B01ACE0183960E94E3CA61E080E0DB
:106180000E944DB260E976E0CE01C5960E9457C8E4
:1061900086E4C82E8DE0D82EF12CE12CE016F10615
:1061A0000CF0F0C06E2DCE0101960E94D474F60161
:1061B00021913191419151916F010E94C7E44B01AE
:1061C0005C01FFEFEF1AFF0A20E030E04CEF52ECE9
:1061D0000E9426E387FF33C0B701CE0189960E9453
:1061E0008EC864E67AE0CE0183960E9479CBBE0128
:1061F000675D7F4FCE0183960E94F1C96EE676E01F
:106200000E94DBC9BC0180EF93E10E945BCACE0112
:1062100083960E94E3CACE0189960E94E3CA0130A8
:10622000110509F055C081E0E816F10409F0B6CF78
:1062300060EF73E1CE01C5960E9487CAAFCF22E01E
:10624000B501A401CE018F960E94EBCAB701CE0121
:1062500089960E948EC864E67AE0CE0183960E94F9
:1062600079CBBE01675D7F4FCE0183960E94F1C955
:106270006EEE75E00E94DBC9BE01615D7F4F0E943A
:10628000F1C9BC0184EE93E10E9487CACE018396D6
:106290000E94E3CACE0189960E94E3CACE018F967E
:1062A0000E94E3CA64EE73E1CE0183960E9470CB34
:1062B00062E277E0CE0183960E94DBC9BC0180EFE9
:1062C00093E10E945BCACE0183960E94E3CAA7CFE6
:1062D0000230110511F522E0B501A401CE0183962B
:1062E0000E94EBCABE016D5D7F4FCE0189960E9470
:1062F00070CB62E277E0CE0189960E94DBC9BC01D7
:10630000CE01C5960E945BCACE0189960E94E3CA5F
:10631000CE0183960E94E3CA41CF0330110509F4F0
:106320003DCF64EE73E1CE0183960E9470CB44E1D1
:1063300050E06FEF7FEFCE0183960E941614CE01DE
:1063400083960E94E3CA6FEE78E0CE0183960E94A6
:1063500079CBCE0183960E94B810CE0183960E941D
:10636000E3CA80919D04882309F418CF8091FB042F
:10637000882309F413CF60ED77E080E090E00E947D
:106380003D720CCFCE01C5960E94DFC880EF93E12D
:106390000E94DFC80115110579F56AEA7EE080EFF9
:1063A00093E10E9462CA6FE97EE0CE0183960E946B
:1063B00067CB4AE050E06FEF7FEFCE0183960E94FB
:1063C0001614CE0183960E94E3CACE01C5960E94A0
:1063D000E3CAEA960FB6F894DEBF0FBECDBFDF91D9
:1063E000CF911F910F91FF90EF90DF90CF90BF90D2
:1063F000AF909F908F900895043011050CF5BE0169
:106400006B5C7F4FCE0183960E9470CB4AE050E0D8
:106410006FEF7FEFCE0183960E941614CE01839614
:106420000E94E3CA6FEE78E0CE0183960E9479CB9A
:10643000CE0183960E94B810CE0183960E94E3CAD3
:106440006AE776E080EF93E10E9451CABECF6DE823
:1064500076E0CE01C5960E9457C8BE016B5C7F4FA7
:10646000CE0183960E9470CB4AE050E070E060E07D
:10647000CE0183960E94B01ACE0183960E94E3CA91
:1064800063E97BE080EF93E10E9457C860EF73E11E
:10649000CE01C5960E9487CA10E000E0602FCE01B1
:1064A00001960E94D4746B017C0122E0BC01A6011C
:1064B000CE0183960115110509F077C00E94EBCA41
:1064C000BE016D5D7F4F88E795E10E94F1D3CE015B
:1064D00083960E94E3CA22E0B701A601CE0183960B
:1064E0000E94EBCABE016D5D7F4FCE0189960E946E
:1064F00070CB62E277E0CE0189960E94DBC9BC01D5
:1065000080EF93E10E945BCACE0189960E94E3CAA4
:10651000CE0183960E94E3CA0F5F1F4F033011051F
:1065200009F0BCCFCE01C5960E94DFC8BE016B5CEE
:106530007F4FCE0183960E9470CB4AE050E06FEF10
:106540007FEFCE0183960E941614CE0183960E949F
:10655000E3CA6FEE78E0CE0183960E9479CBCE013C
:1065600083960E94B810CE0183960E94E3CA80EF02
:1065700093E10E94DFC863E976E0CE0183960E9432
:1065800079CB60EF73E1CE0183960E94F1C96AE78F
:1065900076E00E94DBC9BC0180EF93E10E9487CACC
:1065A000CE0183960E94E3CA10CF0E94EBCABE01BF
:1065B0006D5D7F4FCE0189960E9470CB62E277E0DD
:1065C000CE0189960E94DBC9BC01CE01C5960E940E
:1065D0005BCACE0189960E94E3CA79CFAF92BF927F
:1065E000CF92DF92EF92FF920F931F93CF93DF939F
:1065F000CDB7DEB72C970FB6F894DEBF0FBECDBF78
:106600008091CF0D811102C00E94F2138091A904E4
:106610009091AA04029751F08091440D9091450DFC
:10662000009709F4BAC1039709F4B7C162E37EE0A9
:106630008AEE93E10E9462CA6AEE73E1CE0101968E
:106640000E9470CB44E150E070E060E0CE01019622
:106650000E94B01ACE0101960E94E3CA63E27EE076
:106660008AEE93E10E9462CA6AEE73E1CE0101965E
:106670000E9470CB44E150E06FEF7FEFCE010196B6
:106680000E941614CE0101960E94E3CA87E00E9480
:1066900091C58C0186E00E9491C5BC0190E080E02C
:1066A0000E942BE32AE037ED43EA5CE30E948CE38F
:1066B00023E333E948E853E40E94C6E46B017C011C
:1066C00084E0A82EB12C20E030E048EC52E4C70171
:1066D000B6010E94AEE618160CF05FC081E0A81A61
:1066E000B108E9F064E670E080E090E00E943D725D
:1066F00086E00E9491C5BC0190E080E00E942BE3FF
:106700002AE037ED43EA5CE30E948CE323E333E9BC
:1067100048E853E40E94C6E46B017C01D4CF68E1F1
:106720007EE08AEE93E10E9462CA6AEE73E1CE01D6
:1067300001960E9470CB4AE050E070E060E0CE012C
:1067400001960E94B01ACE0101960E94E3CA6DE93B
:1067500076E0CE0101960E9479CB6AEE73E1CE011C
:1067600001960E94F1C9BC0180EF93E10E9487CAA3
:10677000CE0101960E94E3CA8091440D9091450D8F
:10678000049721F41092450D1092440D81E090E0A1
:106790009093AA048093A904DFC0B80190E080E040
:1067A0000E942BE32AE037ED43EA5CE30E948CE38E
:1067B00023E333E948E853E40E94C6E4AB01BC019B
:1067C00021E0CE0101960E94EBCA6FEA76E0CE018D
:1067D00007960E9479CBBE016F5F7F4FCE0107966F
:1067E0000E94F1C9BC0180EF93E10E9487CACE01EB
:1067F00007960E94E3CACE0101960E94E3CA83E095
:1068000090E09093450D8093440D60EF73E1CE01CD
:1068100001960E9470CB42E350E06FEF7FEFCE0114
:1068200001960E941614CE0101960E94E3CA6FEEF3
:1068300078E0CE0101960E9479CBCE0101960E94AC
:10684000B810CE0101960E94E3CA68EB76E080EFB3
:1068500093E10E9451CA21E0B701A601CE01019641
:106860000E94EBCA60E976E0CE0107960E9479CBE0
:10687000BE016F5F7F4FCE0107960E94F1C9BC0138
:1068800086EF93E10E9487CACE0107960E94E3CA71
:10689000CE0101960E94E3CA62E277E0CE01019642
:1068A0000E9479CB66EF73E1CE0101960E94F1C997
:1068B000BC018AEE93E10E9487CACE0101960E9434
:1068C000E3CA6AEE73E1CE0101960E9470CB4AE002
:1068D00050E070E060E0CE0101960E94F719CE0111
:1068E00001960E94E3CA6FEE78E0CE0101960E9405
:1068F00079CBCE0101960E94B810CE0101960E947C
:10690000E3CA68EB76E086EF93E10E9451CA66EF36
:1069100073E1CE0101960E9470CB62E277E0CE0176
:1069200001960E94DBC960EF73E10E94F1C9BC01CE
:1069300080EF93E10E9487CACE0101960E94E3CACC
:106940008091440D9091450D039731F484E090E0DF
:106950009093450D8093440D64E670E080E090E0F4
:106960000E943D728091CF0D882331F060E273E088
:1069700080E090E00E943D722C960FB6F894DEBF46
:106980000FBECDBFDF91CF911F910F91FF90EF9080
:10699000DF90CF90BF90AF9008958AE99FE00E946A
:1069A0004DB564E670E080E090E00E943D7268E5DD
:1069B0007EE08AEE93E10E9462CA6AEE73E1CE0144
:1069C00001960E9470CB44E150E070E060E0CE019F
:1069D00001960E94B01ACE0101960E94E3CA69E4B2
:1069E0007EE08AEE93E10E9462CA6AEE73E1CE0114
:1069F00001960E9470CB44E150E06FEF7FEFCE0133
:106A000001960E941614CE0101960E94E3CA8CE4FE
:106A10000E946BB56B017C0104E010E0A7019601B8
:106A2000C701B6010E9413E8882309F449C0015048
:106A3000110961F068EC70E080E090E00E943D7226
:106A40008CE40E946BB56B017C01E8CF6EE37EE0C5
:106A50008AEE93E10E9462CA6AEE73E1CE0101966A
:106A60000E9470CB4AE050E070E060E0CE010196F9
:106A70000E94B01ACE0101960E94E3CA6DE976E049
:106A8000CE0101960E9479CB6AEE73E1CE010196A8
:106A90000E94F1C9BC0180EF93E10E9487CACE0138
:106AA00001960E94E3CA8091440D9091450D039791
:106AB00021F41092450D1092440D82E090E068CED2
:106AC00021E0B701A601CE0107960E94EBCA6FEA4A
:106AD00076E0CE0101960E9479CBBE01695F7F4FBF
:106AE000CE0101960E94F1C9BC0180EF93E10E94A2
:106AF00087CACE0101960E94E3CACE0107960E9482
:106B0000E3CA83E090E09093450D8093440D60EFDD
:106B100073E1CE0101960E9470CB42E350E06FEF2B
:106B20007FEFCE0101960E941614CE0101960E94BD
:106B3000E3CA6FEE78E0CE0101960E9479CBCE01D8
:106B400001960E94B810CE0101960E94E3CA68EB3C
:106B500076E080EF93E10E9451CA86E60E946BB511
:106B60006B017C0104E010E0A7019601C701B601AA
:106B70000E9413E8882381F00150110909F484C0B0
:106B800068EC70E080E090E00E943D7286E60E9432
:106B90006BB56B017C01E8CF21E0B701A601CE0106
:106BA00007960E94EBCA60E976E0CE0101960E944A
:106BB00079CBBE01695F7F4FCE0101960E94F1C97A
:106BC000BC0186EF93E10E9487CACE0101960E9424
:106BD000E3CACE0107960E94E3CA62E277E0CE01E3
:106BE00001960E9479CB66EF73E1CE0101960E9477
:106BF000F1C9BC018AEE93E10E9487CACE010196D9
:106C00000E94E3CA6AEE73E1CE0101960E9470CB46
:106C10004AE050E06FEF7FEFCE0101960E94F71936
:106C2000CE0101960E94E3CA6FEE78E0CE01019694
:106C30000E9479CBCE0101960E94B810CE01019638
:106C40000E94E3CA68EB76E086EF93E10E9451CAA6
:106C500066EF73E1CE0101960E9470CB62E277E0AD
:106C6000CE0101960E94DBC960EF73E10E94F1C979
:106C7000BC0180EF93E10E9487CACE0101960E9479
:106C8000E3CA83E090E064CE63E97BE086EF93E1C2
:106C90000E9457C8DDCF4F925F926F927F928F9282
:106CA0009F92AF92BF92CF92DF92EF92FF92CF93DB
:106CB000DF93CDB7DEB72C970FB6F894DEBF0FBECB
:106CC000CDBF0E94F2130E9476B72B013C010E94B7
:106CD0003DB94B015C016091EB047091EC04809133
:106CE000ED049091EE040E942DE36B017C010E9463
:106CF00076B70E942DE3A70196010E94A5E521E049
:106D00003EED42E45EE30E9479E79B01AC0160E066
:106D100070E080E89FE30E94C6E420E03AE24DE2A2
:106D200057E40E948CE36B017C01C301B2010E9415
:106D30002DE320E030E048EC52E40E94A5E5AB01F1
:106D4000BC0122E0CE0101960E94EBCABE016F5F3A
:106D50007F4F84EE93E10E949ECACE0101960E946D
:106D6000E3CA63EC79E084EE93E10E9451CA64EED9
:106D700073E18AEE93E10E9487CA6FEB79E0CE015E
:106D800001960E9479CB64EE73E1CE0101960E94D8
:106D9000F1C9BC0184EE93E10E9487CACE0101963D
:106DA0000E94E3CA60E976E080EF93E10E9457C851
:106DB00021E0B501A401CE0101960E94EBCABE01FB
:106DC0006F5F7F4F80EF93E10E945BCACE01019617
:106DD0000E94E3CA6BEB76E080EF93E10E9451CA18
:106DE00021E0B701A601CE0101960E94EBCABE01C7
:106DF0006F5F7F4FCE0107960E9470CB6FE278E005
:106E0000CE0107960E94DBC9BC0180EF93E10E948E
:106E10005BCACE0107960E94E3CACE0101960E948A
:106E2000E3CA64EE73E1CE0101960E9470CB62E288
:106E300077E0CE0101960E94DBC960EF73E10E940A
:106E4000F1C9BC0180EF93E10E9487CACE0101968F
:106E50000E94E3CA21E0B501A401CE0101960E947F
:106E6000EBCABE016F5F7F4F86EF93E10E949ECA1F
:106E7000CE0101960E94E3CA66EF73E1CE0101964E
:106E80000E9470CB4AE050E070E060E0CE010196D5
:106E90000E94B01ACE0101960E94E3CA65E070E03C
:106EA00080E090E00E943D726FEE78E0CE010196A6
:106EB0000E9479CBCE0101960E94B810CE010196B6
:106EC0000E94E3CA6AEE73E1CE0101960E9470CB84
:106ED0004AE050E06FEF7FEFCE0101960E9416145A
:106EE000CE0101960E94E3CA20E0B701A601CE01BF
:106EF00001960E94EBCABE016F5F7F4FCE010796DD
:106F00000E9470CB6FE278E0CE0107960E94DBC949
:106F1000BC0186EF93E10E9487CACE0107960E94CA
:106F2000E3CACE0101960E94E3CA66EF73E1CE0187
:106F300001960E9470CB4AE050E064EF7FEFCE01F3
:106F400001960E941614CE0101960E94E3CA65E0E4
:106F500070E080E090E00E943D728091CF0D882328
:106F600031F068E572E080E090E00E943D722C967E
:106F70000FB6F894DEBF0FBECDBFDF91CF91FF906B
:106F8000EF90DF90CF90BF90AF909F908F907F90C9
:106F90006F905F904F9008958F929F92AF92BF92A3
:106FA000CF92DF92EF92FF920F931F93CF93DF93D5
:106FB000CDB7DEB7E6970FB6F894DEBF0FBECDBFF4
:106FC0009E012F5F3F4F79018E010B5D1F4F813076
:106FD000910509F0B0C061EC76E0C9010E9479CB5F
:106FE00064EC76E0CE0107960E9479CB67EC76E000
:106FF000CE010D960E9479CB67E972E1C8010E942B
:1070000067CB44E650E06FEF7FEFC8010E94B01AF3
:10701000C8010E94E3CA6CE872E18EE094E10E942C
:1070200062CA6091F0047091F104CE018B960E94C7
:107030008EC86EE074E1C8010E9470CBBE01655D30
:107040007F4FC8010E94F1C9BC01CE01C1960E94C8
:1070500070CB40ED57E06FEF7FEFCE01C1960E94FD
:107060001614CE01C1960E94E3CAC8010E94E3CA69
:10707000CE018B960E94E3CA6DE772E1C8010E94BF
:1070800067CB44E650E06FEF7FEFC8010E94B01A73
:10709000C8010E94E3CA6AEC76E0C8010E9479CB7D
:1070A00023E030E0A801B701CE018B960E94A3CC6B
:1070B000BE01655D7F4F8EE094E10E949ECACE01C5
:1070C0008B960E94E3CAC8010E94E3CA8091121401
:1070D00090911314892B09F444C470E060E08EE0B1
:1070E00094E10E94AFC9082E000C990BC0970A9733
:1070F00008F037C48EE094E10E94D4C84B016EECD6
:1071000076E0C8010E9479CB86E0889DB001899D18
:10711000700D11246E0D7F1DC8010E94F1C9BC01C4
:107120008EE094E10E9487CAC8010E94E3CA0E94CF
:10713000BC99D82E77C28630910509F0B4C063EDB2
:1071400076E0C9010E9479CB68ED76E0CE01079622
:107150000E9479CB60EE76E0CE010D960E9479CB4D
:107160006DE672E1C8010E9467CB44E650E06FEF24
:107170007FEFC8010E94B01AC8010E94E3CA67E607
:1071800072E18EE094E10E9462CA8091D9129091DE
:10719000DA12019626E0289F6001299FD00C112465
:1071A000CE0CDF1C6EE074E1C8010E9470CBB6010A
:1071B000C8010E94F1C9BC01CE018B960E9470CB20
:1071C00040ED57E06FEF7FEFCE018B960E941614D3
:1071D000CE018B960E94E3CAC8010E94E3CA68E50B
:1071E00072E1C8010E9467CB44E650E06FEF7FEF89
:1071F000C8010E94B01AC8010E94E3CA63E97BE09B
:10720000C8010E9479CB23E030E0A801B701CE018C
:107210008B960E94A3CCBE01655D7F4F8EE094E10A
:107220000E949ECACE018B960E94E3CAC8010E94AA
:10723000E3CA8091121490911314892B09F491C31D
:1072400070E060E08EE094E10E94AFC9082E000C6F
:10725000990BC0970A9708F084C38EE094E10E94CE
:10726000D4C8AB01BC014150510961097109CE017B
:107270008B960E9461C86CEE76E0C8010E9479CBC3
:10728000BE01655D7F4FC8010E94F1C9BC018EE05F
:1072900094E10E9487CAC8010E94E3CACE018B967E
:1072A0000E94E3CA44CF8930910509F0E0C069012A
:1072B00063E97BE0C6010E9479CB36E0C30ED11CA6
:1072C000C016D106A9F76EE472E1C7010E9462CA36
:1072D00061E472E1CE0107960E9462CA64E372E142
:1072E000CE010D960E9462CA6AE272E1CE01439617
:1072F0000E9462CA6DE172E1CE0149960E9462CAA3
:107300006EE072E1CE014F960E9462CA6FEF71E1AA
:10731000C8010E9467CB44E650E06FEF7FEFC801E1
:107320000E94B01AC8010E94E3CA63E97BE08EE0C4
:1073300094E10E9457C88091C9129091CA1226E028
:10734000289FB001299F700D11246E0D7F1DC8016B
:107350000E9470CB40ED57E06FEF7FEFC8010E94B5
:107360001614C8010E94E3CA60EF71E1C8010E94CF
:1073700067CB44E650E06FEF7FEFC8010E94B01A80
:10738000C8010E94E3CA6EE074E1C8010E9470CB9C
:1073900026E030E0A801B701CE018B960E94A3CC75
:1073A000BE01655D7F4F8EE094E10E949ECACE01D2
:1073B0008B960E94E3CAC8010E94E3CA809112140E
:1073C00090911314892B09F450C070E060E08EE0B6
:1073D00094E10E94AFC9082E000C990BC0970A9740
:1073E00008F043C065EF76E0C8010E9479CB6EE0FB
:1073F00074E1C8010E94F1C9BC018EE094E10E94D1
:1074000087CAC8010E94E3CA0E94BC99D82E0650C0
:107410001109C8010E94E3CAE016F106C1F763E34F
:1074200071E1D11002C064E271E1C7010E9467CB33
:1074300048EC50E06FEF7FEFC7010E941614C701C0
:107440000E94E3CAE6960FB6F894DEBF0FBECDBF2A
:10745000DF91CF911F910F91FF90EF90DF90CF9030
:10746000BF90AF909F908F900895D12CD0CF8A3F3E
:107470002FEF920709F0F7C06AEF76E0C7010E948C
:1074800079CB64E077E0CE0107960E9479CB6CE07F
:1074900077E0CE010D960E9479CB64E177E0CE01D2
:1074A00043960E9479CB61EE71E1C8010E9467CBDF
:1074B00044E650E06FEF7FEFC8010E94B01AC801A8
:1074C0000E94E3CA6BED71E18EE094E10E9462CA12
:1074D00080916F12670136E08302C00CD11C112429
:1074E0006EE074E1C8010E9470CBB601C8010E9431
:1074F000F1C9BC01CE018B960E9470CB40ED57E0E4
:107500006FEF7FEFCE018B960E941614CE018B9603
:107510000E94E3CAC8010E94E3CA6BEC71E1C80192
:107520000E9467CB44E650E06FEF7FEFC8010E94F6
:10753000B01AC8010E94E3CA6EE074E1C8010E945B
:1075400070CB24E030E0A801B701CE018B960E94F9
:10755000A3CCBE01655D7F4F8EE094E10E949ECA80
:10756000CE018B960E94E3CAC8010E94E3CA8091B3
:10757000121490911314892B09F473C070E060E029
:107580008EE094E10E94AFC9082E000C990BC097C1
:107590000A9708F066C08EE094E10E94D4C8623079
:1075A0007105810591050CF449C06FEB71E1C801CB
:1075B0000E9467CB44E650E06FEF7FEFC8010E9466
:1075C0001614C8010E94E3CA44EF51E063E070E082
:1075D000CE018B960E94D0CB6AE177E0C8010E9471
:1075E00079CB6EE074E1C8010E94F1C961E277E0F5
:1075F0000E94DBC9BE01655D7F4F0E94F1C9BC01DD
:107600008EE094E10E9487CAC8010E94E3CACE01BD
:107610008B960E94E3CA0E94BC99D82ECE01439655
:107620000E94E3CACE010D960E94E3CACE010796DE
:107630000E94E3CAC7010E94E3CAF1CE6AE177E083
:10764000C8010E9479CB6EE074E1C8010E94F1C9C3
:10765000BC018EE094E10E9487CAC8010E94E3CA7F
:10766000DACFD12CDBCF0F9609F0E8C0670163E9D0
:107670007BE0C6010E9479CB36E0C30ED11CC01658
:10768000D106A9F769EB71E1C7010E9462CA809136
:10769000721281112FC02091731230917412409197
:1076A00075125091761260E070E080EA90E40E94DA
:1076B000A5E5AB01BC0122E0CE018B960E94EBCA8E
:1076C00064E277E0C8010E9479CBBE01655D7F4F1F
:1076D000C8010E94F1C96BED77E00E94DBC9BC01D3
:1076E000C7010E945BCAC8010E94E3CACE018B9603
:1076F0000E94E3CA6EEA71E1CE0107960E9462CA57
:1077000062EA71E1CE010D960E9462CA66E971E1FA
:10771000CE0143960E9462CA6AE871E1CE014996A1
:107720000E9462CA64E871E1CE014F960E9462CA6B
:1077300065E771E1C8010E9467CB44E650E06FEF56
:107740007FEFC8010E94B01AC8010E94E3CA63E932
:107750007BE08EE094E10E9457C880917212B701DD
:1077600096E08902600D711D1124C8010E9470CB42
:1077700040ED57E06FEF7FEFC8010E941614C8017B
:107780000E94E3CA66E671E1C8010E9467CB44E645
:1077900050E06FEF7FEFC8010E94B01AC8010E944D
:1077A000E3CA6EE074E1C8010E9470CB26E030E0CD
:1077B000A801B701CE018B960E94A3CCBE01655DE6
:1077C0007F4F8EE094E10E949ECACE018B960E946C
:1077D000E3CAC8010E94E3CA809112149091131465
:1077E000892B51F170E060E08EE094E10E94AFC916
:1077F000082E000C990BC0970A97F0F467E277E027
:10780000C8010E9479CB6EE074E1C8010E94F1C901
:10781000BC018EE094E10E9487CAC8010E94E3CABD
:107820000E94BC99D82E06501109C8010E94E3CAD3
:10783000E016F106C1F7F3CDD12CF5CF6EE277E07B
:10784000C7010E9479CB61E377E0CE0107960E94E1
:1078500079CB66E377E0CE010D960E9479CB66E5A1
:1078600071E1C8010E9467CB44E650E06FEF7FEF03
:10787000C8010E94B01AC8010E94E3CA60E571E124
:107880008EE094E10E9462CA8091B9129091BA127E
:1078900026E0289F6001299FD00C1124CE0CDF1C0C
:1078A0006EE074E1C8010E9470CBB601C8010E946D
:1078B000F1C9BC01CE018B960E9470CB40ED57E020
:1078C0006FEF7FEFCE018B960E941614CE018B9640
:1078D0000E94E3CAC8010E94E3CA60E471E1C801E2
:1078E0000E9467CB44E650E06FEF7FEFC8010E9433
:1078F000B01AC8010E94E3CA6EE074E1C8010E9498
:1079000070CB23E030E0A801B701CE018B960E9436
:10791000A3CCBE01655D7F4F8EE094E10E949ECABC
:10792000CE018B960E94E3CAC8010E94E3CA8091EF
:10793000121490911314892BA1F070E060E08EE096
:1079400094E10E94AFC9082E000C990BC0970A97CA
:1079500040F48EE094E10E94D4C8CB010E94E31E63
:10796000E8CBD12C5FCE3F924F925F926F927F9285
:107970008F929F92AF92BF92CF92DF92EF92FF923F
:107980000F931F93CF93DF93CDB7DEB7C057D109C5
:107990000FB6F894DEBF0FBECDBF23966CAF7DAFA0
:1079A0008EAF9FAF23972F962CAF3DAF4EAF5FAFFB
:1079B0002F9763E97BE0CE01C1960E9479CB63E902
:1079C0007BE0CE01C7960E9479CB2396CCACDDAC90
:1079D000EEACFFAC239728EEC21623E0D206E104FA
:1079E000F10464F030E9C32EDD24D394E12CF12CB2
:1079F0002396CCAEDDAEEEAEFFAE23972F96CCAC89
:107A0000DDACEEACFFAC2F9720E1C21627E2D20628
:107A1000E104F10464F020E1C22E27E2D22EE12C31
:107A2000F12C2F96CCAEDDAEEEAEFFAE2F9780914F
:107A3000CF0D882351F0C12CD12C7601C3942F9601
:107A4000CCAEDDAEEEAEFFAE2F970E947072A79661
:107A50006CAF7DAF8EAF9FAFA7970E9470726B9691
:107A60006CAF7DAF8EAF9FAF6B97A7966CAD7DADC2
:107A70008EAD9FADA79728EE33E040E050E00E9426
:107A800063E4E1962CAF3DAF4EAF5FAFE197312C91
:107A900027961CAE1DAE1EAE1FAE27978E01075E49
:107AA0001F4F9E01235F3F4F3EAF2DAF2396CCACBF
:107AB000DDACEEACFFAC2397F094E094D094C0948E
:107AC000C11CD11CE11CF11C6796CCAEDDAEEEAE44
:107AD000FFAE67976B966CAD7DAD8EAD9FAD6B972E
:107AE000A796CCACDDACEEACFFACA7976C197D09CA
:107AF0008E099F092F96CCACDDACEEACFFAC2F9776
:107B00006C157D058E059F050CF0EBC70E942DE3DB
:107B100020E030E04AE754E40E94A5E5AB01BC0157
:107B200023E0C8010E94EBCAB8018AEE93E10E94EB
:107B30009ECAC8010E94E3CAA70196012A303105F6
:107B4000410551058CF4E1964CAD5DAD6EAD7FAD58
:107B5000E197C8010E9461C8B8018AEE93E10E94D2
:107B60009ECAC8010E94E3CA8091CF0D67EA77E000
:107B7000882309F4EFC28AEE93E10E9457C88091EE
:107B80006E0D90916F0D039709F453C0CE010196CD
:107B90000E94FAC463E97BE080EF93E10E9457C83A
:107BA000AE014F5F5F4F5A01C12CD12C7601D50138
:107BB0004D905D906D907D905D01A3019201C30198
:107BC000B2010E948CE39B01AC01C701B6010E9487
:107BD000C7E46B017C0123E0B301A201C8010E944C
:107BE000EBCAB801CE014F960E9470CB62E277E0FB
:107BF000CE014F960E94DBC9BC0180EF93E10E9449
:107C00005BCACE014F960E94E3CAC8010E94E3CA34
:107C1000EDADFEADAE16BF0651F6C701B6010E942E
:107C2000CFE763966CAF7DAF8EAF9FAF6397332482
:107C300033948091330C882309F410C280916E0D27
:107C400090916F0D0397039708F008C289E60E9490
:107C500032B268EA70E08BE294E10E94A2148BE2F7
:107C600094E10E94C67846E050E069E670E08BE25D
:107C700094E10E94127980915A0E90915B0E891BBB
:107C8000990B86309105ECF30E942CB6B82E0E9419
:107C90002CB6A82E0E942CB6D82E0E942CB6C82E28
:107CA0000E942CB6F82E0E942CB6E82EA996AFAEF4
:107CB000A997A8961FAEA897A9966EAD7FADA99774
:107CC0006B29072E000C880B990B0E942DE32B01CA
:107CD0003C014092D50D5092D60D6092D70D709216
:107CE000D80DAB96CFAEAB97AA961FAEAA97AB9620
:107CF0006EAD7FADAB976D29072E000C880B990BED
:107D00000E942DE34B015C018092D90D9092DA0D17
:107D1000A092DB0DB092DC0DAD96EFAEAD97AC96B8
:107D20001FAEAC97AD966EAD7FADAD976F29072EA8
:107D3000000C880B990B0E942DE32B966CAF7DAF46
:107D40008EAF9FAF2B976093DD0D7093DE0D809308
:107D5000DF0D9093E00D8091050EC0900A0ED0903B
:107D60000B0EE0900C0EF0900D0E882309F407C264
:107D70002091ED0D3091EE0D4091EF0D5091F00DF1
:107D8000C301B2010E94C6E4A70196010E948CE3E0
:107D90006093E10D7093E20D8093E30D9093E40DF9
:107DA0002091F10D3091F20D4091F30D5091F40DB1
:107DB000C501B4010E94C6E4A70196010E948CE3AC
:107DC0006093E50D7093E60D8093E70D9093E80DB9
:107DD0002091F50D3091F60D4091F70D5091F80D71
:107DE0002B966CAD7DAD8EAD9FAD2B970E94C6E4FA
:107DF000A70196010E948CE36093E90D7093EA0D50
:107E00008093EB0D9093EC0D20E030E0A9016091A0
:107E1000060E7091070E8091080E9091090E0E9437
:107E2000AEE618160CF081C0C090E10DD090E20DC6
:107E3000E090E30DF090E40D20E030E0A901C701EF
:107E4000B6010E94AEE6181624F0F7FAF094F7F89F
:107E5000F094A70196016091F90D7091FA0D80914F
:107E6000FB0D9091FC0D0E94AEE6181644F41092A2
:107E7000E10D1092E20D1092E30D1092E40DC0900E
:107E8000E50DD090E60DE090E70DF090E80D20E0D4
:107E900030E0A901C701B6010E94AEE6181624F031
:107EA000F7FAF094F7F8F094A70196016091FD0DB0
:107EB0007091FE0D8091FF0D9091000E0E94AEE634
:107EC000181644F41092E50D1092E60D1092E70D8D
:107ED0001092E80DC090E90DD090EA0DE090EB0D06
:107EE000F090EC0D20E030E0A901C701B6010E943E
:107EF000AEE6181624F0F7FAF094F7F8F094A7011C
:107F000096016091010E7091020E8091030E909186
:107F1000040E0E94AEE6181644F41092E90D109279
:107F2000EA0D1092EB0D1092EC0D4091E50D509181
:107F3000E60D6091E70D7091E80D8091E90D90914B
:107F4000EA0DA091EB0DB091EC0DC090E10DD09039
:107F5000E20DE090E30DF090E40DCD86DE86EF8635
:107F6000F88A498B5A8B6B8B7C8B8D8B9E8BAF8B5E
:107F7000B88F63E97BE0CE01C1960E9457C85E01CD
:107F8000FDE0AF0EB11CC12CD12C7601D5014D9076
:107F90005D906D907D905D01A3019201C301B201DE
:107FA0000E948CE39B01AC01C701B6010E94C7E4AB
:107FB0006B017C0121E0B301A201C8010E94EBCA60
:107FC000B801CE014F960E9470CB62E277E0CE01FD
:107FD0004F960E94DBC9BC01CE01C1960E945BCACC
:107FE000CE014F960E94E3CAC8010E94E3CAA016C0
:107FF000B10661F6C701B6010E94CFE72B966CAFC0
:108000007DAF8EAF9FAF2B9721E0AB01BC01CE01BE
:108010004F960E94EBCA62E37BE0C8010E9479CBD5
:108020006AEE73E1C8010E94F1C96AE377E00E9439
:10803000DBC9BE01615E7F4F0E94F1C96EE377E04C
:108040000E94DBC9BC01CE01C1960E945BCAC80177
:108050000E94E3CACE014F960E94E3CA2396CCAC9D
:10806000DDACEEACFFAC23972DE2C21621E0D206C8
:10807000E104F10434F00E94F21360E080E00E9419
:108080004DB280916E0D90916F0D039709F461C20E
:1080900023E063964CAD5DAD6EAD7FAD6397CE01D1
:1080A0004F960E94EBCA62E37BE0C8010E9479CB45
:1080B0006AEE73E1C8010E94F1C965E477E00E94AD
:1080C000DBC9BE01615E7F4F0E94F1C969E477E0C0
:1080D0000E94DBC9BC0180EF93E10E945BCAC8012A
:1080E0000E94E3CACE014F960E94E3CA2AE939E909
:1080F00049E55FE363966CAD7DAD8EAD9FAD639753
:108100000E94AEE618160CF05FC023E333E343E9A8
:108110005FE363966CAD7DAD8EAD9FAD63970E94BE
:1081200026E3880F880B382280916E0D90916F0D99
:10813000181619060CF04AC08230910509F449C09E
:10814000853091050CF045C08330910509F0B9C325
:10815000312CFFC1C8010E9479CB6AEE73E1C801DE
:108160000E94F1C964ED7AE00E94DBC9BC018AEE8D
:1081700093E10E9487CAC8010E94E3CA00CDA3010F
:108180009201C701B6010E948CE36093E10D7093E8
:10819000E20D8093E30D9093E40DA5019401C701D6
:1081A000B6010E948CE36093E50D7093E60D809319
:1081B000E70D9093E80D2B962CAD3DAD4EAD5FAD28
:1081C0002B97C701B60116CE312CAECF332009F460
:1081D0007BC389849A84AB84BC8449805A806B8039
:1081E0007C80CD80DE80EF80F88420E030E0A90143
:1081F000C501B4010E9426E3882309F44FC3A301FB
:108200009201C301B2010E948CE36F966CAF7DAF07
:108210008EAF9FAF6F97A7019601C701B6010E946D
:108220008CE39B01AC016F966CAD7DAD8EAD9FADC7
:108230006F970E94C7E40E94CFE7A50194010E94B6
:1082400046E520EE3EE245E652E40E948CE36F965E
:108250006CAF7DAF8EAF9FAF6F9720E030E0A9018C
:10826000C701B6010E9426E3882309F41CC3A301B9
:108270009201C301B2010E948CE3A3966CAF7DAF63
:108280008EAF9FAFA397A5019401C501B4010E94D1
:108290008CE39B01AC01A3966CAD7DAD8EAD9FAD23
:1082A000A3970E94C7E40E94CFE7A70196010E940E
:1082B00046E520EE3EE245E652E40E948CE3A396BA
:1082C0006CAF7DAF8EAF9FAFA39720E030E0A901E8
:1082D000C301B2010E9426E3882309F4E9C2A50183
:1082E0009401C501B4010E948CE34B015C01A7011C
:1082F0009601C701B6010E948CE39B01AC01C50148
:10830000B4010E94C7E40E94CFE7A30192010E943A
:1083100046E56B017C016AEE73E1C8010E9470CBF7
:108320006BED72E1C8010E94F1C9BC0180EF93E1DD
:108330000E9487CAC8010E94E3CA60EF73E1C801C6
:108340000E9470CBC8010E94DB13C8010E94E3CADF
:1083500021E06F964CAD5DAD6EAD7FAD6F97CE01F8
:108360008B960E94EBCA21E0A3964CAD5DAD6EAD3D
:108370007FADA397CE0185960E94EBCA20EE3EE228
:1083800045E652E4C701B6010E948CE3AB01BC0193
:1083900021E0C8010E94EBCAB801CE014F960E94AD
:1083A00070CB62E277E0CE014F960E94DBC9BE013E
:1083B0006B5D7F4F0E94F1C962E277E00E94DBC9EA
:1083C000BE01655D7F4F0E94F1C9BC0180EF93E162
:1083D0000E9487CACE014F960E94E3CAC8010E943C
:1083E000E3CACE0185960E94E3CACE018B960E9415
:1083F000E3CA6CE477E0C8010E9479CB60EF73E1D7
:10840000C8010E94F1C9BC0184EE93E10E9487CAB1
:10841000C8010E94E3CA64EE73E1C8010E9470CBF8
:10842000C8010E94FB18C8010E94E3CA60EF73E113
:1084300084EE93E10E9487CA60EF73E1C8010E9455
:1084400070CBC8010E94BE13C8010E94E3CA2396E4
:10845000CCACDDACEEACFFAC23972DE2C21621E034
:10846000D206E104F1048CF427966CAD7DAD8EAD9F
:108470009FAD279725E030E040E050E00E9463E4A4
:10848000672B682B692B09F042C06AEE73E1C801C3
:108490000E9470CB60E577E0C8010E94DBC9BC0197
:1084A000CE01C7960E9487CAC8010E94E3CABE01D6
:1084B000695C7F4FC8010E9470CB45E050E06FEFD0
:1084C0007FEFC8010E94B01AC8010E94E3CA63E9A5
:1084D0007BE0C8010E9479CBC8010E94B810C80196
:1084E0000E94E3CA60EF73E1C8010E9470CB45E0CF
:1084F00050E070E060E0C8010E941614C8010E94BC
:10850000E3CA63E97BE080EF93E10E9457C86FAD57
:1085100021967FAD219722968FAD229723969FAD0E
:1085200023972396CCACDDACEEACFFAC2397F7FEE3
:108530000CC064966FAD649765967FAD659766963F
:108540008FAD669767969FAD67970E943D72332403
:1085500033948091330C882309F40DC180916E0D02
:1085600090916F0D0397039708F005C16DE677E0D2
:10857000C8010E9479CBBE016F5C7F4FC8010E9489
:10858000F1C9BC01CE01C1960E9487CAC8010E94F0
:10859000E3CABE016F5C7F4FC8010E9470CBC80167
:1085A0000E94BE13C8010E94E3CABE016F5C7F4FE8
:1085B000C8010E9470CBC8010E94FB18C8010E942C
:1085C000E3CA21E02B964CAD5DAD6EAD7FAD2B9730
:1085D000CE014F960E94EBCA6BE377E0C8010E9480
:1085E00079CBBE01615E7F4FC8010E94F1C96EE385
:1085F00077E00E94DBC9BC01CE01C1960E9487CA08
:10860000C8010E94E3CACE014F960E94E3CABE0190
:108610006F5C7F4FC8010E9470CBC8010E94FB189D
:10862000C8010E94E3CA6AEE73E1C8010E9470CBE0
:10863000BE016F5C7F4FC8010E94F1C9BC01CE0131
:10864000C1960E9487CAC8010E94E3CA6AEE73E11C
:10865000C8010E9470CB6FE777E0C8010E94DBC9B8
:10866000BC01CE01C7960E9487CAC8010E94E3CA16
:108670004D895E896F89788D20E0CE018B960E94AE
:10868000EBCA49895A896B897C8920E0CE0185969D
:108690000E94EBCA4D855E856F85788920E0C80110
:1086A0000E94EBCAB801CE014F960E9470CB62E2E5
:1086B00077E0CE014F960E94DBC9BE016B5D7F4F14
:1086C0000E94F1C962E277E00E94DBC9BE01655DEC
:1086D0007F4F0E94F1C9BC0184EE93E10E9487CADA
:1086E000CE014F960E94E3CAC8010E94E3CACE01A0
:1086F00085960E94E3CACE018B960E94E3CA239618
:10870000CCACDDACEEACFFAC23972DE2C21621E081
:10871000D206E104F10484F427966CAD7DAD8EADF4
:108720009FAD279725E030E040E050E00E9463E4F1
:10873000672B682B692BF9F464EE73E1C8010E9482
:1087400070CB45E050E070E060E0C8010E94161474
:10875000C8010E94E3CABE01695C7F4FC8010E9444
:1087600070CB45E050E06FEF7FEFC8010E94B01A78
:10877000C8010E94E3CA8091CF0DBE01695C7F4FA2
:10878000882309F4A3C1C8010E9470CB4AE050E0DD
:1087900067E070E0C8010E94F719C8010E94E3CAAF
:1087A000332009F180916E0D90916F0D0297D9F4ED
:1087B000BE01695C7F4FC8010E9470CB45E050E06C
:1087C0006FEF7FEFC8010E94B01AC8010E94E3CA90
:1087D00063E97BE0C8010E9479CBC8010E94B81010
:1087E000C8010E94E3CA80916E0D90916F0D0297AF
:1087F000F9F0BE01695C7F4FC8010E9470CB45E073
:1088000050E06FEF7FEFC8010E94B01AC8010E94CC
:10881000E3CA64EE73E1C8010E9470CB4AE050E005
:108820006FEF7FEFC8010E941614C8010E94E3CACF
:108830000E9470726B017C016B962CAD3DAD4EAD0C
:108840005FAD6B97C21AD30AE40AF50A2796CCAE3D
:10885000DDAEEEAEFFAE279723968CAD9DADAEADEF
:10886000BFAD2397C816D906EA06FB0644F4BC013F
:10887000CD016C197D098E099F090E943D720E94ED
:1088800070726B966CAF7DAF8EAF9FAF6B9763E9E5
:108890007BE080EF93E10E9457C81CC96BED7FE03D
:1088A00089EC9FE3CECC6BED7FE089EC9FE301CDBB
:1088B0008BEDC82E8FE0D82E89ECE82E8FE3F82EB2
:1088C0002ACD059709F444CC67E577E0C8010E94FA
:1088D00079CB60EF73E1C8010E94F1C9BC0180EF60
:1088E00093E10E9487CAC8010E94E3CA60EF73E166
:1088F000C8010E9470CBC8010E94BE13C8010E942B
:10890000E3CA60EF73E1C8010E9470CBC8010E9406
:10891000FB18C8010E94E3CA23E063964CAD5DAD2D
:108920006EAD7FAD6397CE014F960E94EBCA66E4B1
:1089300077E0C8010E9479CBBE01615E7F4FC8011C
:108940000E94F1C969E477E00E94DBC9BC0180EFB5
:1089500093E10E9487CAC8010E94E3CACE014F96E4
:108960000E94E3CA60EF73E1C8010E9470CBC801A6
:108970000E94FB18C8010E94E3CA6AEE73E1C801B5
:108980000E9470CB60EF73E1C8010E94F1C9BC0185
:1089900080EF93E10E9487CAC8010E94E3CA6AEE91
:1089A00073E1C8010E9470CB64E677E0C8010E94C1
:1089B000DBC9BC01CE01C7960E9487CAC8010E94CC
:1089C000E3CA49855A856B857C8522E0CE018B966A
:1089D0000E94EBCA4D815E816F81788522E0CE01D5
:1089E00085960E94EBCA49815A816B817C8122E085
:1089F000C8010E94EBCAB801CE014F960E9470CB0D
:108A000062E277E0CE014F960E94DBC9BE016B5D4A
:108A10007F4F0E94F1C962E277E00E94DBC9BE018C
:108A2000655D7F4F0E94F1C9BC0184EE93E10E9415
:108A300087CACE014F960E94E3CAC8010E94E3CACA
:108A4000CE0185960E94E3CACE018B960E94E3CAAE
:108A50002396CCACDDACEEACFFAC23972DE2C21676
:108A600021E0D206E104F1048CF427966CAD7DADD3
:108A70008EAD9FAD279725E030E040E050E00E94AA
:108A800063E4672B682B692B09F062CBBE01695C3C
:108A90007F4FC8010E9470CB45E050E06FEF7FEF41
:108AA000C8010E94B01AC8010E94E3CA64EE73E1D3
:108AB000C8010E9470CB45E050E070E060E0C80162
:108AC0000E941614C8010E94E3CA42CBC8010E944A
:108AD00070CB4AE050E06FEF7FEFC8010E94B01A00
:108AE0005CCECE01C7960E94E3CACE01C1960E9419
:108AF000E3CAC059DF4F0FB6F894DEBF0FBECDBF3B
:108B0000DF91CF911F910F91FF90EF90DF90CF9069
:108B1000BF90AF909F908F907F906F905F904F909D
:108B20003F9008954F925F926F927F928F929F92A3
:108B3000AF92BF92CF92DF92EF92FF920F931F936B
:108B4000CF93DF93CDB7DEB7A8970FB6F894DEBF0B
:108B50000FBECDBF2091D9123091DA122F3F3F4F77
:108B600009F434C58C0163E97BE0CE0149960E948B
:108B700079CB63E97BE0CE014F960E9479CB80915F
:108B8000D9129091DA128130910509F036C5109210
:108B900039141092381480E30E9432B268E070E019
:108BA00080917A1490917B140E94A21469E070E085
:108BB00080917A1490917B140E94A21461E070E07D
:108BC00080917A1490917B140E94A21480917A145F
:108BD00090917B140E94C6788091381480FD39C032
:108BE00080E30E9432B267E070E080917A14909145
:108BF0007B140E94A21480917A1490917B140E949D
:108C0000C67841E050E060E370E080917A14909182
:108C10007B140E94127980917A1490917B14DC016C
:108C2000ED91FC910084F185E02D19951816190637
:108C300094F780917A1490917B14DC01ED91FC9172
:108C40000284F385E02D199590933914809338149C
:108C5000BDCF80E30E9432B270E060E080917A1470
:108C600090917B140E94A21480917A1490917B14AD
:108C70000E94C67846E050E060E370E080917A148C
:108C800090917B140E94127980917A1490917B14B8
:108C9000DC01ED91FC910084F185E02D199506979A
:108CA0009CF380917A1490917B14DC01ED91FC91FE
:108CB0000284F385E02D19959093531480935214F8
:108CC00080917A1490917B14DC01ED91FC910284E7
:108CD000F385E02D19959093551480935414809149
:108CE0007A1490917B14DC01ED91FC910284F38560
:108CF000E02D1995909357148093561480917A140F
:108D000090917B14DC01ED91FC910284F385E02DC0
:108D10001995909359148093581480917A149091D6
:108D20007B14DC01ED91FC910284F385E02D199513
:108D300090935B1480935A1480917A1490917B14D1
:108D4000DC01ED91FC910284F385E02D199590935F
:108D50005D1480935C1480917A1490917B140E942E
:108D6000C67820E0309154146091521470915314DD
:108D700090E080E0620F731F811D911D60936E145F
:108D800070936F14809370149093711420E030915D
:108D90005814C0905614D0905714F12CE12CC20EE8
:108DA000D31EE11CF11CC0927214D0927314E09295
:108DB0007414F092751420E030915C1440905A14B1
:108DC00050905B14712C612C420E531E611C711C5F
:108DD00040927614509277146092781470927914BD
:108DE00080903E1490903F14A0904014B090411495
:108DF000681979098A099B090E942DE39B01AC013E
:108E00000E94C7E46DA37EA38FA398A760913A1434
:108E100070913B1480913C1490913D14681979092C
:108E20008A099B090E942DE39B01AC016DA17EA1E3
:108E30008FA198A50E94A5E520E030E040E85FE31F
:108E40000E94C6E460935E1470935F148093601474
:108E5000909361148090461490904714A090481409
:108E6000B0904914C701B601681979098A099B09AC
:108E70000E942DE39B01AC010E94C7E46B017C01C1
:108E80006091421470914314809144149091451460
:108E9000681979098A099B090E942DE39B01AC019D
:108EA000C701B6010E94A5E520E030E040E85FE39D
:108EB0000E94C6E4609362147093631480936414F8
:108EC00090936514C0904E14D0904F14E0905014BD
:108ED000F0905114C301B2016C197D098E099F09EC
:108EE0000E942DE39B01AC010E94C7E44B015C0191
:108EF00060914A1470914B1480914C1490914D14D0
:108F00006C197D098E099F090E942DE39B01AC011C
:108F1000C501B4010E94A5E520E030E040E85FE330
:108F20000E94C6E46093661470936714809368147B
:108F30009093691465E070E080E090E00E943D72DB
:108F400080905E1490905F14A0906014B0906114B3
:108F5000C0906214D0906314E0906414F090651493
:108F60008091661490916714A0916814B09169146F
:108F70008DA39EA3AFA3B8A722E0AC01BD01CE0193
:108F800043960E94EBCA22E0B701A601CE010D96DE
:108F90000E94EBCA22E0B501A401CE0101960E9415
:108FA000EBCABE016F5F7F4FCE0107960E9470CB68
:108FB00062E277E0CE0107960E94DBC9BE01635FE3
:108FC0007F4F0E94F1C962E277E00E94DBC9BE01D7
:108FD0006D5E7F4F0E94F1C962E277E00E94DBC9BB
:108FE000BC0180EF93E10E9487CACE0107960E94E0
:108FF000E3CACE0101960E94E3CACE010D960E94FB
:10900000E3CACE0143960E94E3CA60EF73E1CE014A
:1090100001960E9470CBCE0101960E94BE13CE0134
:1090200001960E94E3CAA7019601C501B4019058B8
:109030000E9446E52BED3FE049EC5FE30E94C7E468
:109040002091E7043091E8044091E9045091EA044A
:109050000E94C7E42B013C0120E030E0A9010E94FE
:1090600026E387FD5EC34092EA0B5092EB0B6092C1
:10907000EC0B7092ED0B4090EA0B5090EB0B609074
:10908000EC0B7090ED0B2BED3FE049EC50E4C3018D
:10909000B2010E94AEE6181684F42BED3FE049ECD5
:1090A00050E4C301B2010E94C6E46093EA0B7093DE
:1090B000EB0B8093EC0B9093ED0B20E030E044E35E
:1090C00053E46091EA0B7091EB0B8091EC0B909163
:1090D000ED0B0E948CE32BED3FE049E450E40E944D
:1090E000A5E56093E60B7093E70B8093E80B9093F4
:1090F000E90B0E9451E6CE0107960E948EC867E8F0
:1091000077E0CE0101960E9479CBBE01695F7F4F67
:10911000CE0101960E94F1C961E977E00E94DBC9A6
:10912000BC0186EF93E10E9487CACE0101960E949E
:10913000E3CACE0107960E94E3CA4090E60B509026
:10914000E70B6090E80B7090E90B20E030E044EB17
:1091500052E4C301B2010E9426E318160CF4F2C2D5
:1091600020E030E040E05FE3C301B2010E94C7E4C9
:109170000E9451E6CE0107960E948EC868E977E00A
:10918000CE0101960E9479CBBE01695F7F4FCE016F
:1091900001960E94F1C9BC01CE0149960E9487CA7E
:1091A000CE0101960E94E3CACE0107960E94E3CA4F
:1091B00069EF78E0CE014F960E9457C8BE01675E06
:1091C0007F4FCE0101960E9470CB4AE050E070E0E4
:1091D00060E0CE0101960E94B01ACE0101960E9475
:1091E000E3CA0E947072AB01BC018091EE0B9091BA
:1091F000EF0BA091F00BB091F10B8C599F4FAF4F3B
:10920000BF4F84179507A607B70708F020C363E987
:109210007BE0CE0101960E9479CBCE0101960E949F
:10922000B810CE0101960E94E3CABE01615E7F4F75
:1092300088E795E10E94F1D362E277E0CE010196E2
:109240000E9479CBBE01615E7F4FCE0101960E94E4
:10925000F1C9BC01CE0149960E945BCACE010196BC
:109260000E94E3CA0E9470724090FA0B5090FB0B70
:109270006090FC0B7090FD0B6419750986099709C5
:109280000E942BE320E030E04AE754E40E94A5E589
:10929000AB01BC0123E0CE0107960E94EBCA67EA4E
:1092A00077E0CE0101960E9479CBBE01695F7F4FC6
:1092B000CE0101960E94F1C964ED7AE00E94DBC9FB
:1092C000BC0184EE93E10E9487CACE0101960E9400
:1092D000E3CACE0107960E94E3CA64EE73E1CE01B1
:1092E00001960E9470CB66EF73E1CE0101960E9459
:1092F000F1C9BE01675E7F4F0E94F1C9BC01CE017A
:1093000049960E9487CACE0101960E94E3CA64EA88
:1093100074E080EF93E10E9462CA21E0B501A401EC
:10932000CE0101960E94EBCABE016F5F7F4F80EFB6
:1093300093E10E945BCACE0101960E94E3CA21E03C
:109340004DA15EA16FA178A5CE010D960E94EBCA3A
:1093500021E0B701A601CE0107960E94EBCA62E2A6
:1093600077E0CE0101960E9479CBBE01695F7F4F05
:10937000CE0101960E94F1C962E277E00E94DBC94A
:10938000BE01635F7F4F0E94F1C96EE977E00E94E2
:10939000DBC9BC0180EF93E10E945BCACE0101965C
:1093A0000E94E3CACE0107960E94E3CACE010D9641
:1093B0000E94E3CAA5019401C501B4010E948CE397
:1093C0004B015C01A7019601C701B6010E948CE325
:1093D0009B01AC01C501B4010E94C7E46B017C0193
:1093E0002DA13EA14FA158A5CA01B9010E948CE34D
:1093F0009B01AC01C701B6010E94C7E40E94CFE700
:109400006093E20B7093E30B8093E40B9093E50B76
:1094100062EA77E080EF93E10E9451CA4091E20B4B
:109420005091E30B6091E40B7091E50B21E0CE01CC
:1094300001960E94EBCABE016F5F7F4FCE01079677
:109440000E9470CB64EC7BE0CE0107960E94DBC9E2
:10945000BC0186EF93E10E9487CACE0107960E9465
:10946000E3CACE0101960E94E3CA66EF73E180EF82
:1094700093E10E945BCAC090E20BD090E30BE090B6
:10948000E40BF090E50B20E030E04AE754E4C7013C
:10949000B6010E94AEE687FD29C020E030E04AE731
:1094A00054E4C701B6010E94A5E5AB01BC0123E06D
:1094B000CE0101960E94EBCABE016F5F7F4FCE01C5
:1094C00007960E9470CB65EC7BE0CE0107960E9468
:1094D000DBC9BC0186EF93E10E9487CACE010796E3
:1094E0000E94E3CACE0101960E94E3CA20E030E662
:1094F0004AE656E46091E20B7091E30B8091E40B35
:109500009091E50B0E9426E3BE01675E7F4F87FFC7
:10951000BDC1CE0101960E9470CB66EA77E0CE0114
:1095200001960E94DBC960EF73E10E94F1C9BC01A2
:1095300080EF93E10E9487CACE0101960E94E3CAA0
:1095400003301105A1F460EF73E1CE0101960E9492
:1095500070CBCE0101960E94BE13CE0101960E94EF
:10956000E3CA63E97BE080EF93E10E9457C869EAB0
:1095700077E0CE0101960E9479CB66EF73E1CE01D0
:1095800001960E94F1C9BC01CE0107960E9470CBE2
:109590004AE050E06FEF7FEFCE0107960E9416146D
:1095A000CE0107960E94E3CACE0101960E94E3CA4B
:1095B0006AE070E080E090E00E943D72CE014F963C
:1095C0000E94E3CACE0149960E94E3CAA8960FB64C
:1095D000F894DEBF0FBECDBFDF91CF911F910F91E9
:1095E000FF90EF90DF90CF90BF90AF909F908F90C3
:1095F0007F906F905F904F900895892B09F013CD65
:109600000E941B7940900D0550900E0560900F054B
:10961000709010056091360E7091370E072E000C79
:10962000880B990B0E942DE3A30192010E948CE309
:109630002091090530910A0540910B0550910C05C8
:109640000E948CE32091220E3091230E4091240E33
:109650005091250E0E94C7E44B015C0180922E0EB2
:1096600090922F0EA092300EB092310E6091340E77
:109670007091350E072E000C880B990B0E942DE37C
:10968000A30192010E948CE320910505309106050B
:1096900040910705509108050E948CE320911E0E11
:1096A00030911F0E4091200E5091210E0E94C7E470
:1096B0006B017C01C0922A0ED0922B0EE0922C0EF0
:1096C000F0922D0E6091320E7091330E072E000C29
:1096D000880B990B0E942DE3A30192010E948CE359
:1096E0002091010530910205409103055091040538
:1096F0000E948CE320911A0E30911B0E40911C0E9B
:1097000050911D0E0E94C7E46DA37EA38FA398A75E
:109710006093260E7093270E8093280E9093290E47
:1097200082CC2BED3FE049EC50E4C301B2010E9432
:10973000C7E46093EA0B7093EB0B8093EC0B909370
:10974000ED0B99CC20E030E044E353E4C301B201D7
:109750000E9426E31816CCF0A301920160E070E8A5
:1097600084E393E40E94C6E46093E60B7093E70BF6
:109770008093E80B9093E90B0E9451E6CE01079687
:109780000E948EC86BE977E0FBCC20E030E047E830
:1097900053E4C301B2010E9426E31816CCF120E085
:1097A00030E044E353E4C301B2010E94C6E420E088
:1097B00030E040E05FE30E94C7E46093E60B709303
:1097C000E70B8093E80B9093E90B0E9451E6CE01E2
:1097D00007960E948EC86BE977E0CE0101960E9441
:1097E00079CBBE01695F7F4FCE0101960E94F1C91E
:1097F000BC01CE0149960E9487CACE0101960E9403
:10980000E3CACE0107960E94E3CA68EF77E0D2CCA4
:10981000A301920160E070E084EB93E40E94C6E44F
:1098200020E030E040E05FE30E94C7E46093E60B95
:109830007093E70B8093E80B9093E90B0E9451E63D
:10984000CE0107960E948EC868E977E0C6CF0E94D5
:1098500070720E942BE32B013C016091EE0B709122
:10986000EF0B8091F00B9091F10B0E942DE320E023
:1098700030E048EC51E40E94C7E49B01AC01C30115
:10988000B2010E9426E387FDC2CCD6CC80EF93E1E3
:109890000E9487CA8DCEDF92EF92FF920F931F93A3
:1098A000CF93DF93CDB7DEB72C970FB6F894DEBF1A
:1098B0000FBECDBF8C011092EE0C63E97BE0CE01B0
:1098C00007960E9479CBF12CE12CDD24D3948DEF07
:1098D0009EE00E943AAF1816190694F48091EE0C9F
:1098E00081110EC08DEF9EE00E9418AF8A30D1F535
:1098F0008B859C85892B09F443C0D092EE0C40C027
:1099000062E370E080E090E00E943D72EF2851F049
:109910008DEF9EE00E9422B164E670E080E090E06E
:109920000E943D728091EE0C811131C08B859C8527
:10993000892B69F563E97BE0C8010E9479CBCE01F0
:1099400007960E94E3CAC8012C960FB6F894DEBFB2
:109950000FBECDBFDF91CF911F910F91FF90EF9080
:10996000DF9008958D3021F29091EE0C9111C0CFCF
:10997000682FCE0107960E942ECA8FEFE81AF80AC8
:109980006FE070E080E090E00E943D72A0CF809197
:10999000D00D882379F0BE01695F7F4FCE0101961B
:1099A0000E9470CBCE0101960E94BE13CE0101969B
:1099B0000E94E3CABE01695F7F4FC8010E945ECB6F
:1099C000BECF8F929F92AF92BF92CF92DF92EF92D3
:1099D000FF920F931F93CF93DF93CDB7DEB76897B6
:1099E0000FB6F894DEBF0FBECDBF6C018091B912E7
:1099F0009091BA120197C9F063E97BE0C6010E9419
:109A000079CBC60168960FB6F894DEBF0FBECDBF06
:109A1000DF91CF911F910F91FF90EF90DF90CF904A
:109A2000BF90AF909F908F90089562EB77E0CE014A
:109A30000D960E9479CBBE01635F7F4F8DEF9EE054
:109A40000E94F1D36CE271E080E090E00E943D72F0
:109A5000CE0143960E944B4C64E670E080E090E0BB
:109A60000E943D7210E000E085E0A82EB12C9AE043
:109A7000892E912C6DEB77E0CE0101960E9479CB77
:109A8000BE016F5F7F4FCE0143960E9494C97C0157
:109A9000CE0101960E94E3CAA7014F5F5F4FBE014E
:109AA0006D5E7F4FCE0101960E94EF18BE016F5F81
:109AB0007F4FCE010D960E949ECACE0101960E9454
:109AC000E3CA89899A89892B09F170E060E0CE01A7
:109AD0000D960E94AFC9082E000C990BC0970A97EB
:109AE000A8F46FEB77E0CE0101960E9479CBBE011E
:109AF0006F5F7F4FCE010D960E94C0C9E82ECE0148
:109B000001960E94E3CAFF24F394E110F12C6EEC5D
:109B10007EE0CE0101960E9467CB44E150E06FEFFA
:109B20007FEFCE0101960E94F719CE0101960E94A7
:109B3000E3CA0F5F1F4F62E370E080E090E00E9495
:109B40003D72C801B5010E943DE80197D1F461E082
:109B500070E0CE0101960E94A7878D819E81892B9E
:109B600009F46AC0BE016F5F7F4F8EE094E10E94EE
:109B700087CA0E94D0A7FF24F394CE0101960E94C9
:109B8000E3CACE0101960E944B4CBE016F5F7F4F2E
:109B9000CE0143960E949ECACE0101960E94E3CA5E
:109BA00062E370E080E090E00E943D7204361105AF
:109BB00019F0FF2009F45ECF8091D00D8823F1F0D9
:109BC00068E379E0CE0101960E9479CBBE01635F24
:109BD0007F4FCE0101960E94F1C9BC01CE010796CC
:109BE0000E9470CBCE0107960E94BE13CE0107964D
:109BF0000E94E3CACE0101960E94E3CA89899A892C
:109C0000892B61F070E060E0CE010D960E94AFC933
:109C1000082E000C990BC0970A9738F167EC77E093
:109C2000C6010E9479CBCE0143960E94E3CACE01C1
:109C30000D960E94E3CAE5CE043111050CF49DCFC8
:109C4000C801B4010E943DE8892B09F096CFBE01FE
:109C5000635F7F4F8DEF9EE00E94F1D368EC70E070
:109C600080E090E00E943D7288CF6FEB77E0CE01FC
:109C700001960E9479CBBE016F5F7F4FCE010D969A
:109C80000E94C0C9182FCE0101960E94E3CA11118B
:109C9000C5CFBE01635F7F4FC6010E945ECBC3CFBD
:109CA0003F924F925F926F927F928F929F92AF926C
:109CB000BF92CF92DF92EF92FF920F931F93CF93B9
:109CC000DF93CDB7DEB7E4970FB6F894DEBF0FBED3
:109CD000CDBF8091EF0C8823D1F01092EF0CE49669
:109CE0000FB6F894DEBF0FBECDBFDF91CF911F91AD
:109CF0000F91FF90EF90DF90CF90BF90AF909F902B
:109D00008F907F906F905F904F903F90089581E08B
:109D10008093EF0C63E97BE0CE0185960E9479CBBE
:109D200063E97BE0CE018B960E9479CB10E000E0E6
:109D300082E0382E98EEC92E93E0D92EE12CF12C3A
:109D4000F8013197E231F105C0F48827E555F14B70
:109D50008F4F0C9451E8924F29503E50475050502D
:109D600059506A507350A250B350BC50C550CE5099
:109D7000695172517B5184518D5163E97BE0CE0171
:109D800085960E9457C88091B9129091BA12892B7A
:109D900031F46CEF75E0CE0185960E9457C8809132
:109DA000B9129091BA12019731F466EF75E0CE01C5
:109DB00085960E9457C88091B9129091BA12029765
:109DC00031F460E076E0CE0185960E9457C889A5FF
:109DD0009AA5892B31F060E675E1CE0185960E9447
:109DE0005BCA65E076E0CE0101960E9479CB6CE615
:109DF00075E1CE0101960E94F1C9BC01CE018B969E
:109E00000E9487CACE0101960E94E3CA8091B912CE
:109E10009091BA12019709F046C0BE016B5D7F4F69
:109E2000CE0101960E9470CB48EC50E06FEF7FEFBF
:109E3000CE0101960E94B01ACE0101960E94E3CA9B
:109E4000BE01655D7F4FCE0101960E9470CB40ED53
:109E500057E06FEF7FEFCE0101960E941614CE01FE
:109E600001960E94E3CACE0101960E94E14C8D81C9
:109E70009E810097A1F0E981FA812081222379F067
:109E8000079768F064E177E0CE0185960E9462CA88
:109E9000BE016F5F7F4FCE018B960E9487CACE01B5
:109EA00001960E94E3CABE016B5D7F4FCE01019611
:109EB0000E9470CB48EC50E06FEF7FEFCE0101962F
:109EC0000E94F719CE0101960E94E3CABE01655DAA
:109ED0007F4FCE0101960E9470CB48EC50E06FEFAF
:109EE0007FEFCE0101960E941614CE0101960E94CA
:109EF000E3CA0E9492B9982EB12CA12C911016C2DF
:109F00008FEFA81AB80A95E6A916B10409F411C290
:109F10000E9492B9982E64E170E080E090E00E9487
:109F20003D72ECCF68E077E0CE0185960E9462CA70
:109F30000E9470724B015C010E947072A701960131
:109F40000E9495E4CA01B90120E831E541E050E002
:109F50000E9495E420E13EE040E050E00E9463E48E
:109F600029AB3AAB4BAB5CAB2CE330E040E050E0CC
:109F70000E9463E429013A01AB01BC01CE010196C4
:109F80000E9461C8B301A201CE0107960E9461C878
:109F900049A95AA96BA97CA9CE010D960E9461C856
:109FA000C501B40120E03CE546E255E00E9495E49D
:109FB000BA01A901CE0149960E9461C8BE01675E3F
:109FC0007F4FCE0143960E9470CB63ED77E0CE01C8
:109FD00043960E94DBC9BE01635F7F4F0E94F1C9B7
:109FE00066ED77E00E94DBC9BE01695F7F4F0E948A
:109FF000F1C963E676E00E94DBC9BE016F5F7F4F67
:10A000000E94F1C963E477E00E94DBC9BC01CE0184
:10A010004F960E9470CBCE0143960E94E3CACE01B8
:10A0200049960E94E3CACE010D960E94E3CACE0172
:10A0300007960E94E3CACE0101960E94E3CABE01C0
:10A04000615E7F4FCE018B960E949ECACE014F96D5
:10A0500028CF8091440D9091450D69EF76E00197EE
:10A0600011F06BEE76E0CE0185960E9462CA6BED30
:10A0700076E0CE018B960E9462CA15CF6BEC76E03B
:10A08000CE0185960E9462CA6EEB76E0F2CF61EB5C
:10A0900076E0CE0185960E9462CA66EA76E0E9CF54
:10A0A0006AE976E0CE0185960E9462CA69E876E0A8
:10A0B000E0CF8091440D9091450D6EE776E00397D7
:10A0C00011F064E776E0CE0185960E9462CA69E6E7
:10A0D00076E0CFCF6CE576E0CE0185960E9462CA2D
:10A0E0006DE476E0C6CF62E476E0CE0185960E940C
:10A0F00062CA6091701270917112CE0107960E942F
:10A100008EC865E277E0CE0101960E9479CBBE0150
:10A11000695F7F4FCE0101960E94F1C962E077E04E
:10A120000E94DBC9BC01CE0185960E945BCACE01AC
:10A1300001960E94E3CACE0107960E94E3CA65E336
:10A1400076E097CF8091440D9091450D64E276E0E2
:10A15000029711F064E176E0CE0185960E9462CA12
:10A1600067E076E086CF6BEF75E0CE0185960E94C2
:10A1700062CA6BEE75E07DCF60EE75E0CE0185962C
:10A180000E9462CA66ED75E074CF6AEC75E0CE019C
:10A1900085960E9462CA6AEB75E06BCFB09072122E
:10A1A0006FEA75E0CE0185960E9462CA83E08B1546
:10A1B00024F192E0B9160CF073C0BB2031F181E0BC
:10A1C000B81609F464C060917212062E000C770B69
:10A1D000CE0107960E948EC866EA7AE0CE0101960B
:10A1E0000E9479CBBE01695F7F4FCE0101960E942C
:10A1F000F1C9BC0180EF93E13FC094E0B912E3CF15
:10A200006DED77E080EF93E146C0809073129090FF
:10A210007412A0907512B090761220E030E048E4FD
:10A2200052E4C501B4010E9426E387FF02C0332433
:10A230003394A501940160E070E080EA90E40E940C
:10A24000A5E5AB01BC01232DCE0107960E94EBCA08
:10A2500067EA77E0CE0101960E9479CBBE01695F83
:10A260007F4FCE0101960E94F1C962EE77E00E9415
:10A27000DBC9BC01CE0185960E945BCACE01019666
:10A280000E94E3CACE0107960E94E3CA06C069EDA8
:10A2900077E0CE0185960E9451CA6FE975E0E9CE5C
:10A2A0008B2D9AE08902B0011124CE0107960E94FD
:10A2B0008EC865E277E0CE0101960E9479CBBE019F
:10A2C000695F7F4FCE0101960E94F1C96BED77E087
:10A2D000CECF6FE875E0CE0185960E9462CA6FE727
:10A2E00075E0C7CE6FE675E0CE0185960E9462CA22
:10A2F00061E675E0BECE66E575E0CE0185960E940A
:10A3000062CA6BE475E0B5CE6EE375E0CE0185966A
:10A310000E9462CA6EE275E0ACCE62E275E0CE01E8
:10A3200085960E9462CA63E175E0A3CE1092EF0C9D
:10A3300021C061E070E0CE0101960E94A787BE01B6
:10A340006F5F7F4F8EE094E10E949ECACE0101961E
:10A350000E94E3CA8091121490911314892B51F436
:10A360008091EF0C882331F00F5F1F4F03311105EF
:10A3700009F0E6CCCE018B960E94E3CACE01859609
:10A380000E94E3CAACCC2F923F924F925F926F92A1
:10A390007F928F929F92AF92BF92CF92DF92EF9275
:10A3A000FF920F931F93CF93DF93CDB7DEB76697DE
:10A3B0000FB6F894DEBF0FBECDBF8C01E090420D0A
:10A3C000F090430D8091D00D882349F067EA79E041
:10A3D00084ED90E10E9411D4C8010E9408CFC80109
:10A3E0000596059710F40C9448658091420D909164
:10A3F000430D80179107E1F00E94F2130E945D1156
:10A400000C3E2FEF120724F01093430D0093420DE2
:10A41000B801CE0101960E948EC8BE016F5F7F4FCA
:10A420008CEF93E10E949ECACE0101960E94E3CA7E
:10A4300063E97BE080EF93E10E9457C862E277E036
:10A44000CE0101960E9479CB4AE050E06FEF7FEF9A
:10A45000CE0101960E94F719CE0101960E94E3CA2F
:10A46000033EFFEF1F0714F00C9454650E3C3FEFC2
:10A47000130749F0023E4FEF140729F078010A3B19
:10A480005FEF150751F541E050E068E074E1CE015F
:10A4900001960E94EF18BE016F5F7F4F84EE93E13B
:10A4A0000E949ECACE0101960E94E3CA84EE93E107
:10A4B0000E94D4C87801E61AF70A8091E8139091B7
:10A4C000E913892B39F0E091E413F091E5138081D1
:10A4D000811103C08AE0E81AF108C70188960A973B
:10A4E00008F0B5C062EE7FEF6E197F09CE010196CC
:10A4F0000E948EC868E678E0CE0107960E9479CB6C
:10A50000BE016F5F7F4FCE0107960E94F1C9BC016B
:10A5100088E094E10E9487CACE0107960E94E3CAB0
:10A52000CE0101960E94E3CA65EE77E0CE01019666
:10A530000E9479CB68E074E1CE0101960E94F1C9D6
:10A54000BC018AEE93E10E9487CACE0101960E9467
:10A55000E3CA6AEE73E1CE0101960E9470CBCE0190
:10A5600001960E94BE13CE0101960E94E3CA69EED5
:10A5700077E0CE0107960E9479CB68E074E1CE01C6
:10A5800007960E94F1C9BC01CE0101960E9470CBD2
:10A5900048EC50E06FEF7FEFCE0101960E94B01AB9
:10A5A000CE0101960E94E3CACE0107960E94E3CA3B
:10A5B00041E050E068E074E1CE0101960E94EF189E
:10A5C000BE016F5F7F4F84EE93E10E949ECACE0171
:10A5D00001960E94E3CA84EE93E10E94D4C8DC0194
:10A5E000CB010197A109B1096DE477E089309105AC
:10A5F000A105B10508F075C1FC018827ED5FFC4A93
:10A600008F4F0C9451E86F54845487548A548D545E
:10A6100090549354965499540E946D1166960FB6B7
:10A62000F894DEBF0FBECDBFDF91CF911F910F9188
:10A63000FF90EF90DF90CF90BF90AF909F908F9062
:10A640007F906F905F904F903F902F900895C7013B
:10A65000CC960A9708F0CBC06EEC7FEF6E197F099D
:10A66000CE0101960E948EC86FEE78E0CE0107966B
:10A670000E9479CBBE016F5F7F4FCE0107960E948B
:10A68000F1C9BC0188E094E10E9487CACE01079617
:10A690000E94E3CACE0101960E94E3CA41E050E065
:10A6A00068E074E1CE0101960E94EF18BE016F5F71
:10A6B0007F4F84EE93E10E949ECACE0101960E94D4
:10A6C000E3CA84EE93E10E94D4C8B62EC62ED72EDC
:10A6D000B6E0CB16D10409F488C10CF02DC1F1E02D
:10A6E000CF16D1040CF4B7C067E477E080EF93E1B4
:10A6F0000E9462CAF601E956FB4F80818A3008F059
:10A7000024C1B601CE0101960E948EC86DE57AE0A3
:10A71000CE0107960E9479CBBE016F5F7F4FCE01BD
:10A7200007960E94F1C9BC0186EF93E10E9487CA97
:10A73000CE0107960E94E3CACE0101960E94E3CAA9
:10A740006AE377E0CE0101960E9467CB4AE050E0D1
:10A750006FEF7FEFCE0101960E94B01ACE010196F5
:10A760000E94E3CA65E070E080E090E00E943D72E4
:10A7700066EF73E1CE0101960E9470CB4AE050E093
:10A780006FEF7FEFCE0101960E941614CE01019665
:10A790000E94E3CA65E277E080EF93E10E9462CA1B
:10A7A00066EF73E180EF93E10E945BCA6DE177E0B1
:10A7B000CE0101960E9467CB4AE050E06FEF7FEF39
:10A7C000CE0101960E94B01ACE0101960E94E3CA02
:10A7D00065E070E080E090E00E943D7260EF73E120
:10A7E000CE0101960E9470CB4AE050E086C0C701BE
:10A7F000805B9F4F0A9718F56AEB7FEF6E197F0910
:10A80000CE0101960E948EC86BED77E0CE010796CF
:10A810000E9479CBBE016F5F7F4FCE0107960E94E9
:10A82000F1C9BC0188E094E10E9487CACE01079675
:10A830000E94E3CACE0101960E94E3CA0CC09EECBE
:10A84000E9169FEFF90609F429CFA2EEEA16AFEF59
:10A85000FA0609F469CEF092430DE092420D809120
:10A86000F4139091F513009799F14197A8F40230F1
:10A87000110594F060EF73E1CE0101960E9470CB58
:10A880004AE050E06FEF7FEFCE0101960E94161470
:10A89000CE0101960E94E3CA60EF73E1CE010196FA
:10A8A0000E9470CBCE0101960E94BE13CE0101968C
:10A8B0000E94E3CA60EF73E1CE0101960E9470CB63
:10A8C000CE0101960E94FB18CE0101960E94E3CAB8
:10A8D00064E670E080E090E00E943D729FCE6EEBF7
:10A8E00077E08AEE93E10E9462CA6AEE73E1CE01DC
:10A8F00001960E9470CB4CED55E06FEF7FEFCE01DB
:10A9000001960E94161496CF61EB77E0EACF61EAD8
:10A9100077E0E7CF67E977E0E4CF63E977E0E1CF7D
:10A9200063E877E0DECF65E777E0DBCF67E677E0E7
:10A93000D8CF6AE577E0D5CF27E0C216D10409F079
:10A940008ACF80E00E94DE2786CF36E3B30E8A30BE
:10A9500031F58BE0808361E08B2D0E948371B6011D
:10A96000CE0107960E948EC8BE01695F7F4FCE015F
:10A9700001960E9470CB6FEE77E0CE0101960E94A7
:10A98000DBC9BC0180EF93E10E945BCACE01019656
:10A990000E94E3CACE0107960E94E3CA07CF8AE06D
:10A9A0008083B601CE0107960E948EC8BE01695F02
:10A9B0007F4FCE0101960E9470CB65EF77E0CE010C
:10A9C00001960E94DBC9BC0180EF93E10E945BCA43
:10A9D000CE0101960E94E3CACE0107960E94E3CA07
:10A9E00060E08B2D0E948371E1CE88E390E00E94AD
:10A9F000812C31CF0E94F21389E390E00E941A1358
:10AA000020E030E04AE754E40E948CE3AB01BC0153
:10AA100021E0CE0101960E94EBCA6AEF77E0CE01F9
:10AA200007960E9479CBBE016F5F7F4FCE010796DC
:10AA30000E94F1C96DEF77E00E94DBC9BC0180EF95
:10AA400093E10E9487CACE0107960E94E3CACE0115
:10AA500001960E94E3CA61E078E08AEE93E10E94E9
:10AA600057C86AEE73E1CE0101960E9470CB4AE0AE
:10AA700050E068E070E0CE0101960E94B01ACE016D
:10AA800001960E94E3CA60EF73E1CE0101960E9435
:10AA900070CB4AE050E06FEF7FEFCE0101960E944D
:10AAA0001614CE0101960E94E3CA6AEE73E180EFAC
:10AAB00093E10E945BCA8091CF0D882309F4CFCE29
:10AAC00064E670E080E090E02BC4C0900402D09077
:10AAD00005020E94F21389E390E00E941A1320E01D
:10AAE00030E04AE754E40E948CE30E9451E6CE0134
:10AAF00001960E948EC86AEF77E0CE0107960E9409
:10AB000079CBBE016F5F7F4FCE0107960E94F1C9DE
:10AB10006DEF77E00E94DBC9BC0180EF93E10E94FA
:10AB200087CACE0107960E94E3CACE0101960E9411
:10AB3000E3CA8091F4139091F51323E0F22E099764
:10AB400010F092E0F92E80916F1240E050E0BA01CF
:10AB50008330DCF4C6010E94A5124B015C016091B8
:10AB6000701270917112072E000C880B990B0E94C5
:10AB70002DE3A50194010E948CE320E030EC4FE727
:10AB800054E40E94A5E5AB01BC012F2DCE01019636
:10AB90000E94EBCA62E378E0CE0107960E9479CB6F
:10ABA000BE016F5F7F4FCE0107960E94F1C969E039
:10ABB00078E00E94DBC9BC0180EF93E10E945BCA90
:10ABC000CE0107960E94E3CACE0101960E94E3CA15
:10ABD0006CE078E042CF8091CF0D882309F439C131
:10ABE0008AE99FE00E944DB562E370E080E090E06A
:10ABF0000E943D7261E08091A6040E94B57160E000
:10AC00008091A4040E94B57164E670E080E090E059
:10AC10000E943D726091A0047091A1048091A204F1
:10AC20009091A3040E9440110E946410AB01BC01EA
:10AC300023E0CE0107960E94EBCABE01695F7F4FF9
:10AC4000CE0101960E9470CB6FE278E0CE010196B2
:10AC50000E94DBC9BC018AEE93E10E9487CACE0143
:10AC600001960E94E3CACE0107960E94E3CA67E6F6
:10AC700076E0CE0101960E9479CB6AEE73E1CE01B7
:10AC800001960E94F1C9BC0180EF93E10E9487CA3E
:10AC9000CE0101960E94E3CA0E9464106B017C0100
:10ACA0000E9418724B015C018BE19EE40197F1F761
:10ACB0000E9464102B013C010E9418729B01AC01A0
:10ACC000281939094A095B0949015A0131ED8316EE
:10ACD00037E09306A104B104CCF0A7019601C301AB
:10ACE000B2010E94C6E46B017C0120E030E0A901C2
:10ACF0000E94AEE6181674F426EA3BE944EC5BE3E6
:10AD0000C701B6010E9426E387FF0EC040E050E075
:10AD1000BA0126C026EA3BE944EC5BEBC701B60169
:10AD20000E94AEE6181694F3C501B40128EE33E094
:10AD300040E050E00E9463E4CA01B9010E942DE3A3
:10AD40004B015C0120E030E04AE754E4C701B60162
:10AD50000E948CE3A50194010E94A5E5AB01BC0112
:10AD600022E0CE0107960E94EBCABE01695F7F4FC9
:10AD7000CE0101960E9470CB6AE676E0CE01019684
:10AD80000E94DBC9BC0184EE93E10E9487CACE0118
:10AD900001960E94E3CACE0107960E94E3CA65E1CC
:10ADA00078E0CE0101960E9479CB64EE73E1CE018A
:10ADB00001960E94F1C9BC0180EF93E10E945BCA39
:10ADC000CE0101960E94E3CA62E277E0CE010196CD
:10ADD0000E9479CB64EE73E1CE0101960E94F1C925
:10ADE000BC018AEE93E10E945BCACE0101960E94EB
:10ADF000E3CA6EEC77E0CE0101960E9467CB4AE091
:10AE000050E070E060E0CE0101960E94B01ACE01E1
:10AE100001960E94E3CA6AEE73E1CE0101960E9498
:10AE200070CB45E050E06FEF7FEFCE0101960E94BE
:10AE30001614CE0101960E94E3CA69E178E080EF22
:10AE400093E10E9451CA60E08091A6040E94B5710E
:10AE500006CD60918F04709190048091910490913F
:10AE600092040E94442EFBCC8091890490918A0424
:10AE70000E945F30F4CC40918B044E8B60E0842FB5
:10AE80000E94B5718091CF0D811191C18091E51221
:10AE900081118DC18FE0C82ED12CE12CF12C6DEDEC
:10AEA00077E080EF93E10E9462CA60EF73E1CE0128
:10AEB00001960E9470CB4AE050E06FEF7FEFCE0129
:10AEC00001960E94B01ACE0101960E94E3CA312C6D
:10AED000212C198A1D8A1D861E861F86188AA2E3C8
:10AEE0006A2E712C812C912C54018E890E94F5714F
:10AEF000092E000CAA0BBB0B880E991EAA1EBB1EA6
:10AF000065E070E080E090E00E943D7251E0651ADB
:10AF1000710859F74090F2045090F3046090F404E3
:10AF20007090F504C501B4010E942DE320E030E0EB
:10AF300040EA50E40E948CE320E030E040E85AE32D
:10AF40000E948CE320E030E048E452E40E94A5E552
:10AF5000A30192010E94C6E420E030E040E751E402
:10AF60000E948CE34B015C01A30192016AE979E93B
:10AF700089E390E40E94C6E49B01AC01C501B401E1
:10AF80000E94A5E520E030E0A9010E94C7E420E08E
:10AF900030E040E251E40E948CE34B015C01232D40
:10AFA000322D49895D890E94AEE6181624F4382CAA
:10AFB000292CA98ABD8A20E030E0A901B401C5018D
:10AFC0000E9426E387FF04C0812C912CA12CB12C78
:10AFD00022E0A401B501CE0107960E94EBCABE0192
:10AFE000695F7F4FCE0101960E9470CB6CE278E0E2
:10AFF000CE0101960E94DBC9BC018AEE93E10E945A
:10B0000087CACE0101960E94E3CACE0107960E942C
:10B01000E3CA6AEE73E1CE0101960E9470CB4AE06A
:10B0200050E070E060E0CE0101960E941614CE015F
:10B0300001960E94E3CA0E947072AB01BC0180912C
:10B04000F20B9091F30BA091F40BB091F50B8C598E
:10B050009F4FAF4FBF4F84179507A607B70708F05C
:10B06000ACC00E94D6106CE370E080E090E00E94DB
:10B070003D728D859E85AF85B8890196A11DB11D54
:10B080008D879E87AF87B88BC816D906EA06FB0660
:10B090000CF025CF64E670E080E090E00E943D7205
:10B0A0000E94F21364E670E080E090E00E943D723E
:10B0B00065ED77E08AEE93E10E9462CA6AEE73E181
:10B0C000CE0101960E9470CB44E150E070E060E058
:10B0D000CE0101960E94B01ACE0101960E94E3CAE9
:10B0E00022E0432D522D69897D89CE0107960E9469
:10B0F000EBCABE01695F7F4FCE0101960E9470CB03
:10B100006CE278E0CE0101960E94DBC9BC018AEEB8
:10B1100093E10E9487CACE0101960E94E3CACE0144
:10B1200007960E94E3CA6AEE73E1CE0101960E947F
:10B1300070CB42E350E06FEF7FEFCE0101960E94AB
:10B140001614CE0101960E94E3CA64E170E080E02B
:10B1500090E00E943D720E94D6106EE170E080E0A7
:10B1600090E00E943D726EE170E080E090E00E940D
:10B170003D7261E378E0CE0101960E9479CB6AEEE0
:10B1800073E1CE0101960E94F1C965E378E00E9467
:10B19000DBC960EF73E10E94F1C9BC0180EF93E16C
:10B1A0000E9487CACE0101960E94E3CA58CBB3E041
:10B1B000CB2ED12CE12CF12C72CE0E9470720E9409
:10B1C0002BE34B015C016091F20B7091F30B8091CA
:10B1D000F40B9091F50B0E942DE320E030E048EC59
:10B1E00051E40E94C7E49B01AC01C501B4010E9477
:10B1F00026E387FD36CF37CF80918D0490918E0462
:10B2000099270E94A5122DE038E643E55BE30E94F2
:10B210008CE36B017C012091290530912A05409136
:10B220002B0550912C050E9426E318160CF47BC0C8
:10B23000609111057091120580911305909114058C
:10B2400020E030E048EC52E40E948CE320E030E063
:10B2500048EA51E40E948CE32091F6043091F7040F
:10B260004091F8045091F9040E94A5E56B017C011E
:10B270006AEE77E08AEE93E10E9462CA6AEE73E1B9
:10B28000CE0101960E9470CB42E350E070E060E096
:10B29000CE0101960E94B01ACE0101960E94E3CA27
:10B2A00022E0B701A601CE0101960E94EBCA6FE32E
:10B2B00078E0CE0107960E9479CBBE016F5F7F4F89
:10B2C000CE0107960E94F1C969E378E00E94DBC9CC
:10B2D000BC0180EF93E10E9487CACE0107960E94CD
:10B2E000E3CACE0101960E94E3CA60EF73E1CE018A
:10B2F00001960E9470CB42E350E06FEF7FEFCE01EA
:10B3000001960E941614CE0101960E94E3CA809114
:10B31000CF0D882309F4A3CA60E273E080E090E0D7
:10B320000E943D729CCA20913D0530913E0540919E
:10B330003F0550914005C701B6010E94AEE687FF68
:10B3400005C0C701B6010E94A4B37ACF609125055C
:10B3500070912605809127059091280571CF0E9454
:10B36000F2136EE178E080EF93E10E9462CA60EF31
:10B3700073E1CE0101960E9470CB4AE050E070E08C
:10B3800060E0CE0101960E94B01ACE0101960E94A3
:10B39000E3CA65E178E08AEE93E10E9462CA6AEE50
:10B3A00073E1CE0101960E9470CB44E150E06FEF53
:10B3B0007FEFCE0101960E941614CE0101960E94E5
:10B3C000E3CA8091F60B9091F70B8230910509F05A
:10B3D00041C00E942AC7811104C01092F70B10923D
:10B3E000F60B8091F60B9091F70B029709F448C089
:10B3F00069E078E080EF93E10E9462CA60EF73E158
:10B40000CE0101960E9470CB4AE050E070E060E00F
:10B41000CE0101960E94B01ACE0101960E94E3CAA5
:10B4200060EF73E1CE0101960E9470CB62E277E09B
:10B43000CE0101960E94DBC96AEE73E10E94F1C958
:10B44000BC0180EF93E10E9487CACE0101960E9461
:10B45000E3CA5DCF892B61F60E942AC7882339F0A1
:10B4600082E090E09093F70B8093F60BBACF0E94A6
:10B470002AC78111F5CF0E942AC78111F1CFB1CF20
:10B480008AE090E00E942E176B017C0120E030E002
:10B49000A9010E9426E3181634F08AE090E00E9489
:10B4A0002E176B017C01FBE0AF2EB12C20E030E0C9
:10B4B00042ED53E4C701B6010E9426E318168CF052
:10B4C00091E0A91AB10869F068EC70E080E090E0C2
:10B4D0000E943D7283E090E00E942E176B017C0178
:10B4E000E5CF20E030E0A901C701B6010E9426E3C4
:10B4F00018166CF16BEF77E080EF93E10E9462CA5F
:10B5000060EF73E1CE0101960E9470CB42E350E000
:10B510006FEF7FEFCE0101960E941614CE010196C7
:10B520000E94E3CA62EF77E08AEE93E10E9462CA6A
:10B530006AEE73E1CE0101960E9470CB42E350E0C7
:10B5400070E060E0CE0101960E94B01ADCCE20E0EF
:10B5500030E048EC52E4C701B6010E9426E321E046
:10B5600087FF20E0B701A601CE0101960E94EBCA39
:10B570006EE378E0CE0107960E9479CBBE016F5F43
:10B580007F4FCE0107960E94F1C963E478E00E94E4
:10B59000DBC9BC0180EF93E10E9487CACE01079608
:10B5A0000E94E3CACE0101960E94E3CAA9CF0E947D
:10B5B00070720E94B11C53C9E0908704F090880417
:10B5C00067E478E08AEE93E10E9457C80E94F21384
:10B5D0006AEE73E1CE0101960E9470CB4AE050E022
:10B5E0006FEF7FEFCE0101960E94B01ACE01019657
:10B5F0000E94E3CAC7010E949713698B7A8B8B8BD9
:10B600009C8B8090D7049090D804A090D904B090DF
:10B61000DA04A50194016091D3047091D40480915F
:10B62000D5049091D6040E94C6E42B013C0120E091
:10B6300030E0A9010E9426E3882309F48AC0C09063
:10B64000DF04D090E004E090E104F090E20420E018
:10B6500030E0A901C701B6010E9426E318160CF0DC
:10B6600078C02091DB043091DC044091DD045091DE
:10B67000DE042D873E874F87588BC701B6010E9495
:10B6800026E3882309F465C0A70196016D857E85B0
:10B690008F8598890E94A5E50E94FDE66D877E87CB
:10B6A0008F87988BA501940169897A898B899C89F8
:10B6B0000E94C6E4A30192010E94A5E52D853E8566
:10B6C0004F8558890E948CE30E941FE69B01AC01C4
:10B6D000C701B6010E948CE36B017C016AEE73E145
:10B6E000CE0101960E9470CB4AE050E070E060E02D
:10B6F000CE0101960E94B01ACE0101960E94E3CAC3
:10B7000020E030E64AEE56E4C701B6010E94AEE6FC
:10B7100018161CF568E278E080EF93E10E9462CA97
:10B7200060EF73E1CE0101960E9470CB4AE050E0D9
:10B730006FEF7FEFCE0101960E941614CE010196A5
:10B740000E94E3CA64E670E080E090E00E943D72EF
:10B75000DECDC12CD12C7601C1CF21E0B701A601ED
:10B76000CE0107960E94EBCA61E578E0CE01019612
:10B770000E9479CBBE01695F7F4FCE0101960E9486
:10B78000F1C965E578E00E94DBC9BC0180EF93E177
:10B790000E9487CACE0101960E94E3CACE01079695
:10B7A0000E94E3CABDCFE0900402F09005020E941F
:10B7B000F21365E070E080E090E00E943D728091BD
:10B7C0006F1240E050E0BA018330DCF4C7010E9400
:10B7D000A5126B017C016091701270917112072E9D
:10B7E000000C880B990B0E942DE3A70196010E9483
:10B7F0008CE320E030EC4FE754E40E94A5E5AB0178
:10B80000BC0123E0CE0101960E94EBCA62E378E01E
:10B81000CE0107960E9479CBBE016F5F7F4FCE01AC
:10B8200007960E94F1C969E078E00E94DBC9BC017B
:10B8300080EF93E10E9487CACE0107960E94E3CA77
:10B84000CE0101960E94E3CA69E578E006C98091BD
:10B85000120C91E089278093120C8091CF0D8823E0
:10B8600031F060EF73E18DEF9EE00E94FFD368EC52
:10B8700070E080E090E054CD1092CF0D0C942F54E6
:10B8800081E08093CF0D8093F3128091EA12882398
:10B8900049F161E678E08CEF93E10E9457C886EEAB
:10B8A0009FEF9093430D8093420D2091ED123091C4
:10B8B000EE128091EF129091F0128217930724F00C
:10B8C0001092F0121092EF121092E1121092E21206
:10B8D0001092E3121092E4126CE271E080E090E0CA
:10B8E0000E943D726CEF73E182E094E10E9487CA8E
:10B8F0008091420D9091430D9093C60D8093C50D9C
:10B900000C942F540E94504E0C942F5487E390E1D6
:10B910000E944DB540E052EC61E070E087E390E1B9
:10B920000E94EA168CED95E0A0E0B0E080933B1019
:10B9300090933C10A0933D10B0933E1064E670E0ED
:10B9400080E090E00E943D728091F60B9091F70BA1
:10B95000019709F0D3C083E090E00E945318811151
:10B960000BC01092F70B1092F60B8091F60B909192
:10B97000F70B019709F0DBC06FE478E080EF93E10B
:10B980000E9462CA60EF73E1CE0101960E9470CB03
:10B99000CE0101960E94B71ECE0101960E94E3CA15
:10B9A00062E370E080E090E00E943D7260EF73E13E
:10B9B000CE0101960E9470CB42E350E06FEF7FEF23
:10B9C000CE0101960E94B01ACE0101960E94E3CAF0
:10B9D00063E478E08AEE93E10E9462CA6AEE73E162
:10B9E000CE0101960E9470CB44E150E06FEF7FEFF3
:10B9F000CE0101960E941614CE0101960E94E3CA60
:10BA00008BEB8F838AEA888781E089876801180138
:10BA1000412C512C3201C6016AE070E00E943DE8E1
:10BA2000892B49F443E050E0BE01695F7F4F87E313
:10BA300090E10E94C3AE65E070E080E090E00E947B
:10BA40003D725FEFC51AD50A7801812C912C540103
:10BA500087E390E10E943AAF892B39F484E088169D
:10BA60009104A104B1040CF081C096E0E916F10440
:10BA70000CF07CC087E390E10E943AAF892B71F013
:10BA800087E390E10E9418AFE1E0F0E0EC0FFD1FCA
:10BA9000EE0DFF1D8083AFEFEA1AFA0A65E070E051
:10BAA00080E090E00E943D72B6E0EB16F10401F5F3
:10BAB00099818F8198131CC09A818885981318C02A
:10BAC0009B818985981314C08D8190E0B0E0A0E03F
:10BAD000BA2FA92F982F88272C81820F911DA11D85
:10BAE000B11D480E591E6A1E7B1EEFEF2E1A3E0A2C
:10BAF000FFEF8F1A9F0AAF0ABF0AAACF81E090E03A
:10BB00000E945318882339F081E090E09093F70B5E
:10BB10008093F60B2ACF83E090E00E9453188111A6
:10BB2000F3CF83E090E00E9453188111EDCF67E6D8
:10BB300078E08AEE93E10E9462CA6AEE73E1CE0178
:10BB400001960E9470CB44E150E06FEF7FEFCE0191
:10BB500001960E941614CE0101960E94E3CA6BE57D
:10BB600078E080EF93E10E9462CA4AC034E0231675
:10BB7000310434F440E9C41641E0D40609F04BCF57
:10BB8000C301B2010E942DE320E030E040E251E425
:10BB90000E94A5E520E030E040E85EE30E948CE3EF
:10BBA0006B017C0120E030E040EA51E40E94AEE607
:10BBB00018160CF055C021E0B701A601CE01019680
:10BBC0000E94EBCA64E678E0CE0107960E9479CB2A
:10BBD000BE016F5F7F4FCE0107960E94F1C967E6F5
:10BBE00078E00E94DBC9BC0180EF93E10E9487CA24
:10BBF000CE0107960E94E3CACE0101960E94E3CAD5
:10BC000060EF73E1CE0101960E9470CB4AE050E0F4
:10BC100070E060E0CE0101960E94B01ACE0101965C
:10BC20000E94E3CA60EF73E1CE0101960E9470CBDF
:10BC300062E277E0CE0101960E94DBC96AEE73E111
:10BC40000E94F1C9BC0180EF93E10E9487CACE0136
:10BC500001960E94E3CA87E390E10E944DB557CB5D
:10BC600067E378E07ECF62E079E0CE0101960E9442
:10BC700067CB4AE050E06FEF7FEFCE0101960E9464
:10BC80001614CE0101960E94E3CA60919E04709141
:10BC90009F048091F0049091F1040E94A91474E132
:10BCA000872E912CA12CB12CD12CC12C4FEFC41A72
:10BCB000D40AC501B4010E943D7260919E04709146
:10BCC0009F048091F0049091F1040E94A9147C01DA
:10BCD00053E0C516D10434F02EE1C216D10444F469
:10BCE000EF2851F034E1830E911CA11CB11CDECF72
:10BCF000E114F10409F00CC18091F0049091F10479
:10BD00008B30910509F0DFC08091871490918814E1
:10BD1000A0918914B0918A1480933E0D90933F0DA9
:10BD2000A093400DB093410D8091831490918414A1
:10BD3000A0918514B091861480933A0D90933B0D99
:10BD4000A0933C0DB0933D0D40913E0D50913F0DA1
:10BD50006091400D7091410D21E0CE0101960E944D
:10BD6000EBCA60E976E0CE0107960E9479CBBE016E
:10BD70006F5F7F4FCE0107960E94F1C9BC0180EF33
:10BD800093E10E9487CACE0107960E94E3CACE01C2
:10BD900001960E94E3CA40913A0D50913B0D60918B
:10BDA0003C0D70913D0D21E0CE0101960E94EBCA41
:10BDB0006AE678E0CE0107960E9479CBBE016F5FFC
:10BDC0007F4FCE0107960E94F1C9BC0180EF93E13D
:10BDD0000E945BCACE0107960E94E3CACE0101967B
:10BDE0000E94E3CA6CE378E080EF93E10E9451CABD
:10BDF00063E97BE0CE0101960E9479CB44E150E0FB
:10BE000070E060E0CE0101960E94B01ACE0101966A
:10BE10000E94E3CAC0903E0DD0903F0DE090400DCF
:10BE2000F090410D20E030E0A901C701B6010E9469
:10BE3000AEE620E030E040E05FE387FD64C0C7018C
:10BE4000B6010E94C7E40E9451E6AB01BC01CE01DD
:10BE500001960E9461C8BE016F5F7F4F8AEE93E139
:10BE60000E949ECACE0101960E94E3CA60E087E06C
:10BE70000E944DB26AEE73E188E795E10E94F1D32A
:10BE80006FED88E795E10E94D4CD60E778E088E720
:10BE900095E10E941BCF60913A0D70913B0D80910E
:10BEA0003C0D90913D0D0E9451E64AE050E088E73C
:10BEB00095E10E94CECE6CE378E088E795E10E94A0
:10BEC0001BCF0C9460558631910509F41DCF0C975A
:10BED00009F03ACF8091310D9091320DA091330D40
:10BEE000B091340D80933E0D90933F0DA093400D83
:10BEF000B093410D80912D0D90912E0DA0912F0D9D
:10BF0000B091300D19CFC701B6010E94C6E49BCF96
:10BF10008FEFE816F806D4F064EF78E0CE010196D2
:10BF20000E9467CB4AE050E070E060E0CE010196ED
:10BF30000E94B01ACE0101960E94E3CA61ED78E03A
:10BF400080EF93E10E9462CA0C942F549EEFE91691
:10BF50009FEFF90681F163EC78E0CE0101960E9433
:10BF600067CB4AE050E070E060E0CE0101960E94AD
:10BF7000B01ACE0101960E94E3CA64EB78E080EF2C
:10BF800093E10E9462CAB701CE0101960E948EC859
:10BF9000BE016F5F7F4F80EF93E10E945BCACE01CD
:10BFA00001960E94E3CA6EE978E080EF93E10E9477
:10BFB00004CA0C942F5463E978E0CE0101960E94E4
:10BFC00067CB4AE050E070E060E0CE0101960E944D
:10BFD000B01ACE0101960E94E3CA63E778E0B0CFC1
:10BFE0008091A804882311F40C942F5463E97BE01A
:10BFF000CE0101960E9479CB4AE050E061E070E00A
:10C00000CE0101960E94B01ACE0101960E94E3CAA9
:10C010000E944B360C942F548091CF0D811109C092
:10C020008091E5126EE1462E512C612C712C8823F3
:10C0300029F053E0452E512C612C712C60E179E000
:10C0400080EF93E10E9462CA60EF73E1CE01019636
:10C050000E9470CB4AE050E06FEF7FEFCE01019677
:10C060000E941614CE0101960E94E3CA812C912CE5
:10C0700054011D861E861F86188A83E20E9432B2F2
:10C0800067E070E08BE294E10E94A2148BE294E1FD
:10C090000E94C67866E970E080E090E00E943D7200
:10C0A00083E20E9432B260E270E08BE294E10E948F
:10C0B000A2148BE294E10E94C67866E970E080E009
:10C0C00090E00E943D7242E050E063E270E08BE25B
:10C0D00094E10E941279C12CD12C760180915A0EE4
:10C0E00090915B0E891B990B181619065CF40E943F
:10C0F0002CB6FE2CED2CDC2CCC24C80ED11CE11C63
:10C10000F11CECCFC701B6010E942DE32AE939E901
:10C1100049E95FE30E94A5E50E9451E6AB01BC013D
:10C1200084169506A606B70614F44A015C01CE01F2
:10C1300007960E9461C8BE01695F7F4FCE010196DC
:10C140000E9470CB63E778E0CE0101960E94DBC9C4
:10C15000BC018AEE93E10E9487CACE0101960E943B
:10C16000E3CACE0107960E94E3CA6AEE73E1CE01EC
:10C1700001960E9470CB4EE150E070E060E0CE018D
:10C1800001960E94F719CE0101960E94E3CA2D85FF
:10C190003E854F8558892F5F3F4F4F4F5F4F2D870B
:10C1A0003E874F87588B42165306640675060CF07F
:10C1B00064CFB501A401CE0107960E9461C8BE01FB
:10C1C000695F7F4FCE0101960E9470CB63E778E0F4
:10C1D000CE0101960E94DBC9BC018AEE93E10E9468
:10C1E00087CACE0101960E94E3CACE0107960E943B
:10C1F000E3CA6AEE73E1CE0101960E9470CB4AE079
:10C2000050E070E060E0CE0101960E94B01ACE01CD
:10C2100001960E94E3CAB501A401CE0101960E94D5
:10C2200061C862EB78E0CE0107960E9479CBBE012F
:10C230006F5F7F4FCE0107960E94F1C967E778E0F4
:10C240000E94DBC960EF73E10E94F1C9BC0180EF7D
:10C2500093E10E9487CACE0107960E94E3CACE01ED
:10C2600001960E94E3CA62E370E080E090E058C863
:10C27000E0900202F090030281E08093FA0464E609
:10C2800070E080E090E00E943D720E94F213C701CE
:10C290000E94A5120E9451E620E034E0A901461B4D
:10C2A000570BBA01CE0101960E948EC86CE778E068
:10C2B000CE0107960E9479CBBE016F5F7F4FCE0102
:10C2C00007960E94F1C9BC0180EF93E10E9487CAE2
:10C2D000CE0107960E94E3CACE0101960E94E3CAEE
:10C2E00060E087E00E944DB260E279E0CE01019605
:10C2F0000E9467CB42E350E068E070E0CE01019617
:10C300000E94B01ACE0101960E94E3CA60EF73E169
:10C31000CE0101960E9470CB42E350E06FEF7FEFB9
:10C32000CE0101960E941614CE0101960E94E3CA26
:10C3300063E878E0CE0101960E9479CB60EF73E16B
:10C34000CE0101967BC880910002909101020E946B
:10C35000A5120E9451E67093F90B6093F80B62E30B
:10C3600070E080E090E00E943D726091F80B709167
:10C37000F90BCE0101960E948EC8BE016F5F7F4F00
:10C3800080EF93E10E949ECACE0101960E94E3CA0B
:10C390008091811490918214892B09F45EC06DE71D
:10C3A00074E1CE0107960E9470CBBE01695F7F4F9A
:10C3B000CE0101960E9470CB44E150E070E060E055
:10C3C000CE0101960E94B01ACE0101960E94E3CAE6
:10C3D0006DE878E0CE0101960E9479CB60EF73E1C1
:10C3E000CE0101960E94F1C9BC018AEE93E10E9440
:10C3F00087CACE0101960E94E3CA6AEE73E1CE01BC
:10C4000001960E9470CB44E150E06FEF7FEFCE01C8
:10C4100001960E941614CE0101960E94E3CABE0145
:10C42000695F7F4FCE0101960E9470CB62E277E098
:10C43000CE0101960E94DBC96AEE73E10E94F1C948
:10C44000BC0180EF93E10E9487CACE0101960E9451
:10C45000E3CACE0107960C94855968E978E08AEE24
:10C4600093E10E9457C86AEE73E1CE0101960E94E3
:10C4700070CB44E150E070E060E0CE0101960E9494
:10C48000B01ACE0101960E94E3CA6CE778E0CE01B3
:10C4900001960E9479CB60EF73E1CE0101960E9474
:10C4A000F1C9BC018AEE93E10E9487CACE010196D0
:10C4B0000E94E3CA6AEE73E1CE0101960E9470CB3E
:10C4C00044E150E06FEF7FEFCE0101960E94161419
:10C4D000CE0101960E94E3CA6DE878E02BCF8091EF
:10C4E000A804882311F40C942F548091CF0D81114E
:10C4F00004C08091E512882331F082E090E00E9430
:10C5000092450C942F54C0908F04D0909004E090EA
:10C510009104F090920420E030E040E450E4C70140
:10C52000B6010E94AEE618160CF054C020E030E0D0
:10C530004AEF54E4C701B6010E948CE30E9451E621
:10C540006B017C010E94F21360E080E00E944DB21A
:10C5500061E379E088E795E10E9411D461E080E031
:10C560000E944DB269E279E088E795E10E9411D41A
:10C5700064E670E080E090E00E943D720E9470727C
:10C580006093FA0B7093FB0B8093FC0B9093FD0B65
:10C590000E9470728090FA0B9090FB0BA090FC0BA5
:10C5A000B090FD0B681979098A099B096C157D0506
:10C5B0008E059F0514F00C942F5483E090E00E94A8
:10C5C00092450E94707264E170E080E090E00E9409
:10C5D0003D72DECF30E3C32E35E7D32EE12CF12CB4
:10C5E000B1CF0E94EE328DEF9EE00E9422B10C94FA
:10C5F0002F5461E579E08AEE93E10E9462CA6AEE07
:10C6000073E1CE0101960E9470CB4AE050E070E0E9
:10C6100060E0CE0101960E94B01ACE0101960E9400
:10C62000E3CA3090060280910A0C811105C00E9475
:10C63000707281E080930A0C8091020C811105C018
:10C640000E94707281E08093020C1092390C10925B
:10C65000380CE090380CF090390C58E2E516F104F3
:10C660000CF07EC0832D0E94F571F701EE0FFF1FC5
:10C67000E25AF14F918380830E947AB220E030E049
:10C6800040EA50E40E948CE320E030E040E85AE3C6
:10C690000E948CE36B017C014090CF045090D00449
:10C6A0006090D1047090D204A30192016091CB04F8
:10C6B0007091CC048091CD049091CE040E94C6E488
:10C6C0009B01AC0160E070E080EC90E40E94C6E465
:10C6D0004B015C0120E030E0A9010E9426E320E04C
:10C6E00030E040E650E481111CC0C701B6010E9451
:10C6F0008CE36093FE0B7093FF0B8093000C909380
:10C70000010C64E170E080E090E00E943D72809155
:10C71000380C9091390C01969093390C8093380C19
:10C7200098CFC701B6010E948CE3A30192010E9439
:10C73000C7E420E030E040E850E40E94C6E4A501F0
:10C7400094010E94A5E520E030E040EC50E40E9416
:10C750008CE320E030E040E850E40E94C7E4C9CF19
:10C76000C090FE0BD090FF0BE090000CF090010CFD
:10C7700020E030E0A901C701B6010E94AEE687FDC6
:10C7800022C022E0B701A601CE0107960E94EBCAA3
:10C790006CE978E0CE0101960E9479CBBE01695F19
:10C7A0007F4FCE0101960E94F1C9BC0180EF93E159
:10C7B0000E9487CACE0101960E94E3CACE01079665
:10C7C0000E94E3CA06C062E479E080EF93E10E9430
:10C7D00062CA60EF73E1CE0101960E9470CB4AE01D
:10C7E00050E06FEF7FEFCE0101960E9416145BC000
:10C7F0008091A804882311F40C942F548091CF0DBC
:10C8000081112EC08091E51281112AC0C0908F0441
:10C81000D0909004E0909104F090920420E030E0F9
:10C820004AE754E4C701B6010E948CE30E9451E636
:10C830004B015C0120E030E040EA50E4C701B60162
:10C840000E948CE320E030E040EA50E40E94C7E41C
:10C850000E9451E6A50194010E94B33C0C942F5410
:10C8600021E030E040E050E06AE070E080E090E0FD
:10C87000F3CFC7010E94CC370C942F54C7010E94FC
:10C8800085650C942F548091D00D882311F40C945D
:10C890002F546FE979E0CE0101960E9467CBCE015B
:10C8A00001960E94BE13CE0101960E94E3CA0C9429
:10C8B0002F5480915C0E90915D0E892B81F481E064
:10C8C00090E090935D0E80935C0E8EE492E00E9467
:10C8D00081B468EC70E080E090E00E943D7262E913
:10C8E00079E0CE0101960E9467CB44E650E06FEFFD
:10C8F0007FEFCE0101960E941614CE0101960E9490
:10C90000E3CAF0E0E0E019950C942F540E94EDC7C3
:10C910000E94F2130E945D110C942F548091EA1230
:10C9200091E089278093EA12882309F48BC06BE891
:10C9300079E080EF93E10E9462CA0E947072609376
:10C94000E1127093E2128093E3129093E4128091CB
:10C95000ED129091EE12181619065CF42091EF1268
:10C960003091F0122817390724F01092F01210922B
:10C97000EF129091F1128091EC12981724F010921E
:10C98000F1121092F2128091EA128093E51260EF98
:10C9900073E1CE0101960E9470CB4AE050E068E05E
:10C9A00070E0CE0101960E94B01ACE0101960E945D
:10C9B000E3CA66E779E0CE0101960E9467CB4AE0C0
:10C9C00050E06FEF7FEFCE0101960E941614CE016A
:10C9D00001960E94E3CA68E679E080EF93E10E9445
:10C9E00004CA68E379E0CE0101960E9479CB60EF3A
:10C9F00073E1CE0101960E94F1C9BC0180EF93E181
:10CA00000E9487CACE0101960E94E3CA8091CF0D91
:10CA10008093F3128CE291E00E94ACB48091CF0D30
:10CA2000882311F40C942F5461E678E08CEF93E1A5
:10CA30000E9457C886EE9FEF9093430D8093420D5E
:10CA40000C942F5463E879E080EF93E10E9462CA6E
:10CA50009ACFF092430DE092420D8DEF9EE00E943E
:10CA600022B16AE579E080EF93E10E9462CA63E94E
:10CA70007BE0CE0101960E9479CB4AE050E070E065
:10CA800060E0CE0101960E94B01ACE01019698CEC8
:10CA90000E3F2FEF120711F40C940C5363E97BE067
:10CAA00080EF93E10E9457C8F8017C96E632F105C9
:10CAB00080F68827E15AFA498F4F0C9451E839647F
:10CAC00029658E6486645964436429653E642965DA
:10CAD0002965296529652965FA546555EB5534574B
:10CAE0003B57FC58AF59D75ADC5AD35B275C3C5CA8
:10CAF000405C2965825C865C335EF05F0C60386167
:10CB0000A3616F62F162F962F863CF92DF92EF92F4
:10CB1000FF920F931F93CF93DF93CDB7DEB762974A
:10CB20000FB6F894DEBF0FBECDBF8C0163E97BE08A
:10CB30008EE094E10E9457C80830110509F011C138
:10CB400062EF70E1CE0101960E9467CB44E650E0AF
:10CB50006FEF7FEFCE0101960E94B01ACE010196D1
:10CB60000E94E3CA66EE70E1CE0101960E9467CB97
:10CB700044E650E070E060E0CE0101960E94161499
:10CB8000CE0101960E94E3CA8DEF9EE00E9422B181
:10CB90004CE251E061E070E0CE0107960E94D0CBFC
:10CBA0008091D00D8823D1F060EA78E0CE01019623
:10CBB0000E9479CBBE01695F7F4FCE0101960E9432
:10CBC000F1C963EA78E00E94DBC9BC0184ED90E121
:10CBD0000E94FFD3CE0101960E94E3CA6BED77E07D
:10CBE000CE0101960E9479CBBE016F5F7F4FCE01CF
:10CBF00007960E94C0C9182FCE0101960E94E3CA71
:10CC0000112309F491C065EA78E08EE094E10E9476
:10CC100057C888E090E09093430D8093420D6EE0FA
:10CC200074E1CE0101960E9470CBCE0101960E9464
:10CC30003189182FCE0101960E94E3CA69ED70E197
:10CC4000CE0101960E9467CB44E650E070E060E0C0
:10CC5000CE0101960E941614CE0101960E94E3CAED
:10CC60008DEF9EE00E9422B148E552E061E070E065
:10CC7000CE0101960E94D0CBBE016F5F7F4FCE01E7
:10CC800007960E949ECACE0101960E94E3CA809137
:10CC9000D00D8823D1F060EA78E0CE0101960E94A1
:10CCA00079CBBE01695F7F4FCE0101960E94F1C929
:10CCB00063EA78E00E94DBC9BC0184ED90E10E9448
:10CCC000FFD3CE0101960E94E3CA68E678E0CE0168
:10CCD00001960E9479CBBE016F5F7F4FCE01079610
:10CCE0000E94C0C9082FCE0101960E94E3CA00230A
:10CCF000D9F06AEA78E08EE094E10E9457C86EE0CD
:10CD000074E1CE0101960E9470CBCE0101960E9483
:10CD10003189082FCE0101960E94E3CA002321F039
:10CD20006CEC70E1111102C065EC70E1CE0101966E
:10CD30000E9467CB44E650E070E060E0CE010196CF
:10CD40000E941614CE0101960E94E3CA63E97BE0BB
:10CD50008EE094E10E9457C8CE0107960E94E3CA74
:10CD600064C5093F2FEF120709F025C16BEB70E195
:10CD7000CE0101960E9467CB44E650E06FEF7FEF53
:10CD8000CE0101960E94B01ACE0101960E94E3CA1C
:10CD90006DEA70E1CE0101960E9467CB44E650E057
:10CDA00070E060E0CE0101960E941614CE0101965B
:10CDB0000E94E3CA8DEF9EE00E9422B14CE251E056
:10CDC00064E070E0CE0101960E94D0CB8091D00D3E
:10CDD0008823D1F060EA78E0CE0107960E9479CBF3
:10CDE000BE016F5F7F4FCE0107960E94F1C963EAD3
:10CDF00078E00E94DBC9BC0184ED90E10E94FFD382
:10CE0000CE0107960E94E3CA70E060E0CE01019671
:10CE10000E94AFC9082E000C990BC0970A9708F022
:10CE2000AFC060EB78E0CE0107960E9479CBBE01DF
:10CE30006F5F7F4FCE0107960E94F1C9BC018EE063
:10CE400094E10E9487CACE0107960E94E3CA89EF47
:10CE50009FEF9093430D8093420D6EE074E1CE01FD
:10CE600007960E9470CBCE0107960E943189182F39
:10CE7000CE0107960E94E3CA6FE970E1CE010796E2
:10CE80000E9467CB44E650E070E060E0CE01079678
:10CE90000E941614CE0107960E94E3CA8DEF9EE011
:10CEA0000E9422B148E552E065E070E0CE010796AD
:10CEB0000E94D0CBBE01695F7F4FCE0101960E94D8
:10CEC0009ECACE0107960E94E3CA8091D00D8823A6
:10CED000D1F060EA78E0CE0107960E9479CBBE01DE
:10CEE0006F5F7F4FCE0107960E94F1C963EA78E039
:10CEF0000E94DBC9BC0184ED90E10E94FFD3CE010A
:10CF000007960E94E3CA70E060E0CE0101960E949D
:10CF1000AFC9082E000C990BC0970A9788F565EBEE
:10CF200078E0CE0107960E9479CBBE016F5F7F4FFC
:10CF3000CE0107960E94F1C9BC018EE094E10E94E7
:10CF400087CACE0107960E94E3CA89EF9FEF9093AC
:10CF5000430D8093420D6EE074E1CE0107960E946E
:10CF600070CBCE0107960E943189082FCE0107961B
:10CF70000E94E3CA002321F062E970E1111102C0AE
:10CF80006BE870E1CE0107960E9467CB44E650E063
:10CF900070E060E0CE0107960E941614CE0107965D
:10CFA0000E94E3CA63E97BE08EE094E10E9457C8E7
:10CFB000CE010196D3CE61E870E1CE0101960E94C8
:10CFC00067CB44E650E06FEF7FEFCE0101960E9401
:10CFD000B01ACE0101960E94E3CA63E97BE08EE0BD
:10CFE00094E10E9457C8053F8FEF1807B9F46AEB28
:10CFF00078E08EE094E10E9457C867E770E1CE01C7
:10D0000001960E9467CB44E650E06FEF7FEFCE01C0
:10D0100001960E941614CE01019648C1063F9FEF6B
:10D02000190749F46EEB78E08EE094E10E9457C84E
:10D030006DE670E1E4CF013FEFEF1E0749F464ECC9
:10D0400078E08EE094E10E9457C86EE570E1D7CF9A
:10D05000023FFFEF1F0749F46AEC78E08EE094E1AD
:10D060000E9457C86EE470E1CACF033F2FEF12074A
:10D0700009F085C062E470E1CE0101960E9467CBA1
:10D0800044E650E06FEF7FEFCE0101960E94B01AA8
:10D09000CE0101960E94E3CA64E370E1CE010196DD
:10D0A0000E9467CB44E650E06FEF7FEFCE01019620
:10D0B0000E941614CE0101960E94E3CA44EF51E08B
:10D0C00062E070E0CE0101960E94D0CBBE016F5F9E
:10D0D0007F4F8EE094E10E949ECACE0101960E948D
:10D0E000E3CA66ED78E0CE0101960E9479CB6EE04E
:10D0F00074E1CE0101960E94F1C9BC018EE094E179
:10D100000E9487CACE0101960E94E3CA8091121440
:10D1100090911314892B09F488C36EE074E1CE0159
:10D1200001960E9470CBCE0101960E943189F82EA3
:10D13000CE0101960E94E3CA68EC70E080E090E0C6
:10D14000FF2009F481C30E943D726EEF7EE0CE01A4
:10D1500001960E9467CB44EF51E06FEF7FEFCE0165
:10D1600001960E941614CE0101960E94E3CA109304
:10D17000430D0093420DC8010E94C35156C30230B3
:10D18000110509F096C068E270E1CE0101960E9497
:10D1900067CB44E650E06FEF7FEFCE0101960E942F
:10D1A000B01ACE0101960E94E3CA68E170E1CE0197
:10D1B00001960E9467CB44E650E06FEF7FEFCE010F
:10D1C00001960E941614CE0101960E94E3CA44EF14
:10D1D00051E066E070E0CE0101960E94D0CBBE0126
:10D1E0006F5F7F4F8EE094E10E949ECACE01019650
:10D1F0000E94E3CA80911214909113140597B0F025
:10D2000070E060E08EE094E10E94AFC9082E000C4F
:10D21000990BC0970A9750F48EE094E10E94D4C80D
:10D220006135E3EC7E0781059105CCF46AE070E19D
:10D23000CE0101960E9467CB48EE53E06FEF7FEF7F
:10D24000CE0101960E941614CE0101960E94E3CAF7
:10D2500063E97BE08EE094E10E9457C857CF0E94BB
:10D260002DE320E030E048EC52E40E94A5E5AB015C
:10D27000BC0122E0CE0107960E94EBCA6FEB79E079
:10D28000CE0101960E9479CBBE01695F7F4FCE012E
:10D2900001960E94F1C9BC018EE094E10E9487CA08
:10D2A000CE0101960E94E3CACE0107960E94E3CA0E
:10D2B0002DCFC801C796059708F05BC08EEC9FEF95
:10D2C0007C01E01AF10AC70189569B4F6C01FC01F1
:10D2D00080818A30C8F56AEF7FE0CE0101960E9416
:10D2E00067CB44E650E06FEF7FEFCE0101960E94DE
:10D2F000B01ACE0101960E94E3CA8BE0F60180834A
:10D30000B701CE0107960E948EC86DE57AE0CE0186
:10D3100001960E9479CBBE01695F7F4FCE010196D5
:10D320000E94F1C9BC01CE010D960E9470CB44E66B
:10D3300050E06FEF7FEFCE010D960E941614CE01E4
:10D340000D960E94E3CAACCF69EE7FE0CE01019654
:10D350000E9467CB44E650E06FEF7FEFCE0101966D
:10D360000E94B01ACE0101960E94E3CAF601108213
:10D37000C7CF083CFFEF1F0709F0A0C06FED7FE0AB
:10D38000CE0101960E9467CB44E650E06FEF7FEF3D
:10D39000CE0101960E94B01ACE0101960E94E3CA06
:10D3A00062ED7FE0CE0101960E9467CB44E650E03B
:10D3B0006FEF7FEFCE0101960E941614CE01019609
:10D3C0000E94E3CA6DED78E0CE0101960E9479CB10
:10D3D000CE0101960E943189CE0101960E94E3CAD6
:10D3E00064EC7FE0CE0101960E9467CB44E650E0FA
:10D3F0006FEF7FEFCE0101960E94B01ACE01019629
:10D400000E94E3CA68EB7FE0CE0101960E9467CBE1
:10D4100044E650E06FEF7FEFCE0101960E941614B4
:10D42000CE0101960E94E3CA44EF51E061E070E052
:10D43000CE0101960E94D0CBBE016F5F7F4F8EE080
:10D4400094E10E949ECACE0101960E94E3CA809197
:10D45000121490911314892BA9F070E060E08EE013
:10D4600094E10E94AFC9082E000C990BC0970A974F
:10D4700048F48EE094E10E94D4C8623071058105C1
:10D4800091051CF06CEA7FE0D3CE62EE78E0CE012D
:10D4900001960E9479CBCE0101960E943189CE017E
:10D4A00001960E94E3CA67EE78E0CE0101960E94E1
:10D4B00079CBCE0101960E943189ADCD073C2FEF8B
:10D4C000120709F00BC162EA7FE0CE0101960E94CB
:10D4D00067CB44E650E06FEF7FEFCE0101960E94EC
:10D4E000B01ACE0101960E94E3CA65E97FE0CE0141
:10D4F00001960E9467CB44E650E06FEF7FEFCE01CC
:10D5000001960E941614CE0101960E94E3CA6CEEA9
:10D5100078E0CE0101960E9479CBCE0101960E945F
:10D520003189CE0101960E94E3CA67E87FE0CE010F
:10D5300001960E9467CB44E650E06FEF7FEFCE018B
:10D5400001960E94B01ACE0101960E94E3CA69E7D3
:10D550007FE0CE0101960E9467CB44E650E06FEF7A
:10D560007FEFCE0101960E941614CE0101960E9413
:10D57000E3CA63E97BE08EE094E10E9457C8F12C96
:10D58000E12C44EF51E061E070E0CE0101960E9491
:10D59000D0CBBE016F5F7F4F8EE094E10E949ECAA8
:10D5A000CE0101960E94E3CA809112149091131447
:10D5B000892BA9F070E060E08EE094E10E94AFC991
:10D5C000082E000C990BC0970A9748F48EE094E15E
:10D5D0000E94D4C86230710581059105CCF16DE6D9
:10D5E0007FE0CE0101960E9467CB48EE53E06FEFDB
:10D5F0007FEFCE0101960E941614CE0101960E9483
:10D60000E3CA6FE57FE0CE0101960E9467CB44E656
:10D6100050E06FEF7FEFCE0101960E941614CE010D
:10D6200001960E94E3CA63E97BE08EE094E10E94E8
:10D6300057C88FEFE81AF80A64E670E080E090E0DF
:10D640000E943D729EE1E916F1040CF49ACF5ECD82
:10D6500061EF78E0CE0101960E9479CBCE01019670
:10D660000E943189CE0101960E94E3CA8EE094E1C6
:10D670000E94D4C8672B682B692BA1F461E57FE079
:10D68000CE0101960E9467CB44E650E06FEF7FEF3A
:10D69000CE0101960E94B01ACE0101960E94E3CA03
:10D6A000F12CE12C8EE094E10E94D4C86130710528
:10D6B0008105910509F0BDCF66EF78E0CE010196B6
:10D6C0000E9479CBCE0101960E943189CE0101964C
:10D6D0000E94E3CA8FE1E82EF12CABCF063CEFEFBE
:10D6E0001E07D9F567E47FE0CE0101960E9467CB63
:10D6F00044E650E06FEF7FEFCE0101960E94B01A32
:10D70000CE0101960E94E3CA6AE37FE0CE01019652
:10D710000E9467CB44E650E06FEF7FEFCE010196A9
:10D720000E941614CE0101960E94E3CA6BEF78E0C6
:10D73000CE0101960E9479CBCE0101960E943189DB
:10D74000CE0101960E94E3CA60ED77E080E090E0B0
:10D750000E943D7262E079E0A8CE0630110509F022
:10D7600047C06AE27FE0CE0101960E9467CB44E6A3
:10D7700050E06FEF7FEFCE0101960E94B01ACE010C
:10D7800001960E94E3CA6DE17FE0CE0101960E94FE
:10D7900067CB44E650E06FEF7FEFCE0101960E9429
:10D7A0001614CE0101960E94E3CA69E079E0CE0129
:10D7B00001960E9479CBCE0101960E943189CE015B
:10D7C00001960E94E3CA64E670E080E090E00E9467
:10D7D0003D7261E17FE0CE0101960E9467CB44E695
:10D7E00050E06FEF7FEFCE0101960E94B01A13CC8C
:10D7F00068E07FE0CE0101960E9467CB44E650E0EE
:10D800006FEF7FEFCE0101960E941614CE010196B4
:10D810000E94E3CA63E97BE08EE094E10E9457C86E
:10D820000B3EFFEF1F0709F071CC62960FB6F8941C
:10D83000DEBF0FBECDBFDF91CF911F910F91FF9043
:10D84000EF90DF90CF9008950E943D7262EF7EE0EE
:10D85000CE0101960E9467CB44EF51E06FEF7FEF5E
:10D86000CE0101960E941614A3CB4F925F926F9245
:10D870007F928F929F92AF92BF92EF92FF920F93FF
:10D880001F93CF93DF93CDB7DEB762970FB6F894AF
:10D89000DEBF0FBECDBF7C015B0183E29CE00E9436
:10D8A000D9BA892BD9F463E97BE0C7010E9479CB0F
:10D8B000C70162960FB6F894DEBF0FBECDBFDF91F1
:10D8C000CF911F910F91FF90EF90BF90AF909F90DD
:10D8D0008F907F906F905F904F9008954091270CAC
:10D8E0005091280C6091290C70912A0CCE0107965A
:10D8F0000E94521B8091D00D882359F160E179E09C
:10D90000CE0101960E9479CBBE01695F7F4FCE01A7
:10D9100001960E94F1C96EE477E00E94DBC9BC0168
:10D9200084ED90E10E94F1D3CE0101960E94E3CAFA
:10D930004091270C5091280C6091290C70912A0C71
:10D9400020E184ED90E10E9472CD84ED90E10E948F
:10D95000BECD70E060E0CE0107960E94AFC9182FDF
:10D960008A3211F01092EF0C0E9470726093C70D12
:10D970007093C80D8093C90D9093CA0D63E97BE045
:10D98000CE010D960E9479CB812F110F990BC09774
:10D990000A9708F068C0CE0107960E94D4C8633089
:10D9A0007105810591050CF084C001E010E082E072
:10D9B000982E0A151B0509F47CC06CE271E080E02A
:10D9C00090E00E943D729092711110927411412C5E
:10D9D000512C320183E19CE00E94D9BA892B91F449
:10D9E0008EE1481651046104710449F16EE170E062
:10D9F00080E090E00E943D728FEF481A580A680A52
:10DA0000780AE8CF8EE14816510461047104B9F038
:10DA10004091170C5091180C6091190C70911A0CD0
:10DA2000CE0101960E94521BBE016F5F7F4FCE0157
:10DA30000D960E949ECACE0101960E94E3CA898972
:10DA40009A89892B39F0BE01635F7F4FCE0107961B
:10DA50000E945BCA0F5F1F4F63E97BE0CE010D960A
:10DA60000E9457C8A6CF6CE271E080E090E00E946F
:10DA70003D7282E08093711110927411812C912C6F
:10DA8000540183E19CE00E94D9BA892B61F58EE1B3
:10DA900088169104A104B10409F043C089899A89C8
:10DAA000892B39F0BE01635F7F4FCE0107960E943C
:10DAB0005BCA64E670E080E090E00E943D7282E024
:10DAC0008093711110927411BE01695F7F4FC7017D
:10DAD0000E945ECBCE010D960E94E3CACE0107964E
:10DAE0000E94E3CAE5CE8EE188169104A104B10438
:10DAF000A9F24091170C5091180C6091190C70917B
:10DB00001A0CCE0101960E94521BBE016F5F7F4F1F
:10DB1000CE010D960E949ECACE0101960E94E3CAD4
:10DB2000BDCF6EE170E080E090E00E943D728FEF2B
:10DB3000881A980AA80AB80AA4CFAF92BF92CF92C7
:10DB4000DF92EF92FF920F931F93CF93DF93CDB7A6
:10DB5000DEB72C970FB6F894DEBF0FBECDBF7C01A9
:10DB60005B010E9492B9182F811117C063E97BE015
:10DB7000C7010E9479CBC7012C960FB6F894DEBF7F
:10DB80000FBECDBFDF91CF911F910F91FF90EF900E
:10DB9000DF90CF90BF90AF9008958A3211F010922D
:10DBA000EF0C0E9470726093C70D7093C80D809344
:10DBB000C90D9093CA0D612FCE0107960E9445CBE7
:10DBC000812F012E000C990BC0970A9768F5CE01A2
:10DBD00007960E94D4C863307105810591050CF049
:10DBE00070C001E010E00A151B0509F46AC062E389
:10DBF00070E080E090E00E943D720E9492B9D12CCA
:10DC0000C12C81113BC08FEFC81AD80A85E1C81614
:10DC1000D10409F456C06EE170E080E090E00E940B
:10DC20003D720E9492B9EDCF612FCE0101960E9404
:10DC300045CBBE016F5F7F4FCE0107960E949ECA03
:10DC4000CE0101960E94E3CA62E370E080E090E0BA
:10DC50000E943D720E9492B910E000E0811121C043
:10DC60000F5F1F4F0F31110561F16EE170E080E031
:10DC700090E00E943D720E9492B9F0CF682FCE01D1
:10DC800001960E9445CBBE016F5F7F4FCE01079684
:10DC90000E945BCACE0101960E94E3CA0F5F1F4F2C
:10DCA000A2CF682FCE0101960E9445CBBE016F5FC7
:10DCB0007F4FCE0107960E945BCACE0101960E945B
:10DCC000E3CABE01695F7F4FC7010E945ECBCE01F0
:10DCD00007960E94E3CA4FCF0F931F93CF93DF9312
:10DCE00000D000D0CDB7DEB7182F8091D912909117
:10DCF000DA128130910509F044C0112331F068E94E
:10DD000074E084ED90E10E9411D40E947BC3082F3F
:10DD10008C30B9F062E874E084ED90E10E9411D497
:10DD20004AE0602FCE0101960E941BCBBE016F5FBF
:10DD30007F4F84ED90E10E94FFD3CE0101960E94B7
:10DD4000E3CA112389F04AE0602FCE0101960E94B8
:10DD50001BCBBE016F5F7F4F84ED90E10E94FFD32C
:10DD6000CE0101960E94E3CA0E9462C126960FB6B8
:10DD7000F894DEBF0FBECDBFDF91CF911F910F9101
:10DD80000895009709F09BC08AE097E5A4EFB2E4FC
:10DD90008093220E9093230EA093240EB093250E11
:10DDA0008BE794E1A6E6B3E480931E0E90931F0EDA
:10DDB000A093200EB093210E8DEC9CEEA2ECB3E468
:10DDC00080931A0E90931B0EA0931C0EB0931D0E01
:10DDD00089E29CE5AFE8BFE38093090590930A05CB
:10DDE000A0930B05B0930C0587ED93EAA0E9BFE380
:10DDF0008093050590930605A0930705B093080549
:10DE00008AE097EDA3E8BFE38093010590930205B4
:10DE1000A0930305B09304058EE10E9432B261E045
:10DE200070E08BE294E10E94A21486EF98E2ACE9E4
:10DE3000BFE380930D0590930E05A0930F05B0935B
:10DE4000100560E48BE294E10E94AA7063E070E048
:10DE50008BE294E10E94A2148BE294E10E94C678C6
:10DE60008091380E9091390E18161906C4F465E1A8
:10DE700079E084ED90E10E941BCF60910D057091D7
:10DE80000E0580910F059091100542E050E00E9430
:10DE9000BDCE69E279E084ED90E10E94C2CD11111E
:10DEA00005C01092390E1092380E60CF81E090E0DC
:10DEB0009093390E8093380E0E941DCF57CF019654
:10DEC00079F46DE674E0CE0101960E9467CBCE0135
:10DED00001960E94BE13CE0101960E94E3CA46CF6E
:10DEE00064EF71E080E090E00E943D723FCF84E6F5
:10DEF0009FEA892B49F080E090E0892B29F00E946D
:10DF000064AF81110E9400008AE59FEA892B49F0E5
:10DF100080E090E0892B29F00E945AAF81110E9485
:10DF2000000080E59FEA892B49F080E090E0892B92
:10DF300029F00E9450AF81110E94000086E49FEA00
:10DF4000892B49F080E090E0892B29F00E9446AFB0
:10DF500081110C94000008958150823108F05AC05C
:10DF6000E82FF0E08827E854F0498F4F0C9451E8EF
:10DF7000D86FDC6FCA6FD06FD46F0A70DF6FE56F38
:10DF8000E96FEF6FF36FF76FFD6F01700A70057047
:10DF90000B700F70809180008F77809380000895C0
:10DFA000809180008F7DF9CF80918000877FF5CFB1
:10DFB00084B58F7784BD089584B58F7DFBCF809124
:10DFC000B0008F778093B00008958091B0008F7D6E
:10DFD000F9CF809190008F77809390000895809181
:10DFE00090008F7DF9CF80919000877FF5CF809151
:10DFF000A0008F778093A00008958091A0008F7D6E
:10E00000F9CF8091A000877FF5CF809120018F7795
:10E01000809320010895809120018F7DF9CF809118
:10E020002001877FF5CFDC0180E0615090F09D9169
:10E030009827E92FEF70F0E0EB52F24E2491E92F90
:10E04000E295EF70F0E0EB51F24EE491822F8E27D3
:10E05000ECCF089580915A0E90915B0E891B990B1D
:10E0600008952091990D260F3327331F2132310552
:10E07000ECF42091D40EFC0190E080E0243069F0B3
:10E0800082E00895A091990D2191AC014758524F1B
:10E09000A40FB52FB11D2C930196861798F380918C
:10E0A000990D680F6093990D80E0089581E00895BF
:10E0B000089508950895E0915B0E80915A0EE81737
:10E0C00030F4F0E0E65CF14F808190E008958FEF4E
:10E0D0009FEF089590915B0E80915A0E2FEF3FEFC6
:10E0E000981748F4E92FF0E0E65CF14F208130E02A
:10E0F0009F5F90935B0EC9010895CF92DF92EF92DC
:10E10000FF920F931F93CF93DF937C01CB018A0182
:10E110002091DA0E222389F0EB016B01C40ED51E8B
:10E12000CC15DD0569F06991D701ED91FC91019065
:10E13000F081E02DC7011995F3CF642F0E94317053
:10E14000C801DF91CF911F910F91FF90EF90DF9069
:10E15000CF900895CF93DF931F92CDB7DEB7698339
:10E160002091DA0E2223F9F02091FC0E203258F093
:10E1700021E030E0FC013383228390E080E00F90C7
:10E18000DF91CF9108958091DB0EE82FF0E0E4520B
:10E19000F14F998190838F5F8093DB0E8093FC0E0B
:10E1A00081E090E0ECCF61E0CE0101960E943170F9
:10E1B000F7CF90E080E008950C943FE9E3E4F2E1CA
:10E1C00014A215A216A217A210A611A612A613A693
:10E1D00081E084A729E130E036A725A787A780E062
:10E1E00090E0A0EAB0E480AB91ABA2ABB3AB80E02F
:10E1F00090E0A8EAB1E484AB95ABA6ABB7AB809353
:10E20000F6049093F704A093F804B093F90480E027
:10E2100090E0A0E8BFE380938D1290938E12A093BC
:10E220008F12B09390128093F2049093F304A09312
:10E23000F404B093F5041092BA121092B9128BE064
:10E2400090E09093BC128093BB129093F104809362
:10E25000F0041092CA121092C9121092DA1210929F
:10E26000D91290E080E00C94D6B4FC01A48DA80FE4
:10E27000B92FB11DA35ABF4F2C91848D90E0019608
:10E280008F739927848FA689B7892C93A089B18928
:10E290008C91837080648C93938D848D981306C0C9
:10E2A0000288F389E02D80818F7D80830895CF934C
:10E2B000DF93282F30E0F901E153F14E8491F90109
:10E2C000E757F14ED491F901ED5BF14EC491CC23A7
:10E2D000A1F081110E94AC6FEC2FF0E0EE0FFF1F58
:10E2E000E75DF14EA591B491EC91ED2381E090E0D2
:10E2F00009F480E0DF91CF91089580E090E0FACFBB
:10E30000862F0C9457711F93CF93DF93282F30E003
:10E31000F901E153F14E8491F901E757F14ED4919F
:10E32000F901ED5BF14EC491CC23A9F0162F8111B8
:10E330000E94AC6FEC2FF0E0EE0FFF1FE15FF14E9B
:10E34000A591B4918FB7F894EC91111108C0D095B4
:10E35000DE23DC938FBFDF91CF911F910895DE2BD9
:10E36000F8CF862F642F0C948371CF93DF9390E0C6
:10E37000FC01E757F14E24918D5B914EFC01849195
:10E380008823C9F090E0880F991FFC01EB50F24EF2
:10E39000A591B491FC01E15FF14EC591D491611159
:10E3A0000DC09FB7F8948C91209582238C9388811F
:10E3B000282328839FBFDF91CF910895623051F4C5
:10E3C0009FB7F8943C91822F809583238C93E881AA
:10E3D0002E2BEFCF8FB7F894EC912E2B2C938FBF71
:10E3E000EACF862F642F0C94B571863308F08653DC
:10E3F00020917B00982F9870277F922B90937B0021
:10E400002091FA0490E4299F900111248770822BB7
:10E4100080937C0080917A00806480937A00809160
:10E420007A0086FDFCCF8091780090917900089564
:10E430003FB7F8948091C10D9091C20DA091C30D8A
:10E44000B091C40D26B5A89B05C02F3F19F00196C9
:10E45000A11DB11D3FBFBA2FA92F982F8827BC013E
:10E46000CD01620F711D811D911D42E0660F771F66
:10E47000881F991F4A95D1F708958F929F92AF9266
:10E48000BF92CF92DF92EF92FF926B017C010E94CC
:10E4900018724B015C01C114D104E104F104B9F01C
:10E4A0000E941872681979098A099B09683E7340AD
:10E4B0008105910580F321E0C21AD108E108F10835
:10E4C00088EE880E83E0981EA11CB11CE4CFFF905B
:10E4D000EF90DF90CF90BF90AF909F908F90089576
:10E4E0002FB7F8946091BD0D7091BE0D8091BF0D56
:10E4F0009091C00D2FBF08951F920F920FB60F92EB
:10E5000011242F933F938F939F93AF93BF93809149
:10E51000BD0D9091BE0DA091BF0DB091C00D309179
:10E52000BC0D23E0230F2D3758F50196A11DB11D19
:10E530002093BC0D8093BD0D9093BE0DA093BF0D95
:10E54000B093C00D8091C10D9091C20DA091C30DEB
:10E55000B091C40D0196A11DB11D8093C10D909382
:10E56000C20DA093C30DB093C40DBF91AF919F9105
:10E570008F913F912F910F900FBE0F901F90189584
:10E5800026E8230F0296A11DB11DD2CF0C944DE4B5
:10E590000895DF92EF92FF920F931F93CF93DF9333
:10E5A0007C018B01D42EDC011696ED91FC91138633
:10E5B0001586148612861186108617821682158299
:10E5C00014821382C0E0B801F701868197810E940E
:10E5D000B6C5D82F882329F0DC1629F0CF5FDC16CA
:10E5E00090F7D0E009C067E0C8010E941370D8011D
:10E5F00017969C918913F2CF8D2FDF91CF911F91A8
:10E600000F91FF90EF90DF900895DC012C9111960F
:10E61000ED91FC91F8948181822B81839281322F3C
:10E6200030959323928387E090E00197F1F7818101
:10E630008323818383E290E00197F1F790817894BE
:10E64000EFECF0E03197F1F7922381E009F480E0FC
:10E650000895FC0190810180F281E02D292F209501
:10E6600060FF14C0F8948281822382838181892B88
:10E670008183A3E2B0E01197F1F78281982B928316
:10E68000789487ED90E00197F1F70895F8948281EE
:10E69000822382838181892B8183AFEFB0E0119740
:10E6A000F1F78281982B928378948FE090E0EBCF02
:10E6B000DF92EF92FF920F931F93CF93DF93EC01C2
:10E6C000D62EE42E08E010E0FF24F39461E08D2DB7
:10E6D0008F2109F460E0CE010E942973FF0C0150E4
:10E6E0001109A1F7E11010C0F894E981FA81918134
:10E6F0008881809589238183E981FA81928188814B
:10E700008095892382837894DF91CF911F910F9117
:10E71000FF90EF90DF900895EF92FF920F931F9379
:10E72000CF93DF938C017B0140E065E50E94587335
:10E73000E70188E0E80EF11C699140E0C8010E9401
:10E740005873CE15DF05C1F7DF91CF911F910F915F
:10E75000FF90EF900895FC0190810180F281E02DFF
:10E76000F8948181292F20958223818378943DE735
:10E7700043E050E0315029F1DA011197F1F780813F
:10E780008923C1F3F8948281822382838181892B3A
:10E7900081837894ABE7B7E01197F1F7F894818122
:10E7A00082238183A3E1B1E01197F1F7808198235F
:10E7B00081E009F080E07894E3E6F6E03197F1F744
:10E7C000089580E008958F929F92AF92BF92CF926A
:10E7D000DF92EF92FF92CF93DF93EC018E819F81C6
:10E7E0000E94AB7340E06CEC8E819F810E94587355
:10E7F000488164E48E819F810E9458738A818823B6
:10E8000071F1E981E9508EEEC82E82E0D82EE33016
:10E8100038F4F0E0EE0FFF1FED57FA4FC080D180C3
:10E820008B81882339F18881811124C00E94707204
:10E830004B015C010D2C000CEE08FF088E819F81BE
:10E840000E940573813059F00E9470726C197D0925
:10E850008E099F09681579058A059B0578F3DF9174
:10E86000CF91FF90EF90DF90CF90BF90AF909F90AF
:10E870008F900895B601DD0C880B990BDF91CF9135
:10E88000FF90EF90DF90CF90BF90AF909F908F90D0
:10E890000C943D726F927F928F929F92AF92BF9233
:10E8A000CF92DF92EF92FF920F931F93CF93DF935C
:10E8B000EC017B018A018E819F810E94AB738111E3
:10E8C00002C090E037C0B7018E819F810E948C7397
:10E8D00040E06EEB8E819F810E9458737801680141
:10E8E00089E0C80ED11CAE80BF8088E0882E912CB4
:10E8F000712C66246394C5010E94057381117628EA
:10E90000660CE1E08E1A9108B1F7F70171927F0170
:10E91000EC15FD0541F78E819F810E94AB7381301C
:10E9200081F668E0C8010E94137091E0F80120852B
:10E930002813C7CF892FDF91CF911F910F91FF909F
:10E94000EF90DF90CF90BF90AF909F908F907F908F
:10E950006F900895CF93DF9300D000D000D0CDB753
:10E96000DEB7AE014F5F5F4F0E944A74882331F0DB
:10E970008D818F33A9F020F48F31A1F080E007C0A2
:10E980008F3521F08F37D1F78CE001C08BE02996CD
:10E990000FB6F894DEBF0FBECDBFDF91CF910895C3
:10E9A0008AE0F5CF89E0F3CF0F931F93CF93DF93E6
:10E9B000CDB7DEB761970FB6F894DEBF0FBECDBFFF
:10E9C0008C01462FBE01665F7F4F0E94C972811184
:10E9D0000FC060E070E08EEF92EC61960FB6F89495
:10E9E000DEBF0FBECDBFDF91CF911F910F91089574
:10E9F000AE014F5F5F4FBE01665F7F4FC8010E944F
:10EA00004A74882331F36A8170E0762F6627770F86
:10EA1000770F770F298148E0249F90011124262B3E
:10EA2000372B8A858031D1F4688570E08F81AB0106
:10EA3000481B5109CA019695982F88279795879565
:10EA40000E943DE8CB014097B90153E0660F771F64
:10EA50005A95E1F760789C01260F371F213854EE54
:10EA600035070CF4B6CFB901330F880B990B0E9410
:10EA70002DE320E030E040E05CE30E948CE3ADCF8A
:10EA8000EF92FF920F931F93CF93DF9300D000D0AC
:10EA90001F921F92CDB7DEB78C01DC011696ED9167
:10EAA000FC91179713861586148612861186108698
:10EAB0001782168215821482138214961C92149760
:10EAC00015961C92EE24E394BE016F5F7F4FF80110
:10EAD000868197810E94B6C5882309F46FC067E0DC
:10EAE000CE0101960E94137098858913EDCFD8014D
:10EAF0008C91811125C016968D919C910E94AB73CB
:10EB0000BE016F5F7F4FF801868197810E948C73F1
:10EB100040E064EBD80116968D919C910E94587349
:10EB2000F801868197810E940573F82ED801169608
:10EB30008D919C910E94AB73F11002C0F801E082AC
:10EB4000D8011196FC9089818031A1F1BE016F5FDF
:10EB50007F4FC8010E94AA748F15D0F4F8018181FB
:10EB6000D80111968C93119714968C9114978F5FFE
:10EB700014968C938981883231F0B0F4803119F089
:10EB8000823209F0A1CFF80185818F5F85839CCF08
:10EB90008981803111F48CE0E3CFBE016F5F7F4F3C
:10EBA000C8010E94AA74DCCF8B3369F3823409F068
:10EBB0008BCFE9CFFCE0FF1588F2EDCF28960FB69A
:10EBC000F894DEBF0FBECDBFDF91CF911F910F91A3
:10EBD000FF90EF9008951F93CF93DF93EC01162FD2
:10EBE00060E0812F0E94B571612F70E0FB01E75753
:10EBF000F14EE491E883FB01ED5BF14EE491F0E02E
:10EC0000EE0FFF1FE75DF14E859194919A83898302
:10EC10001B861D861C861A86198618861F821E82F0
:10EC20001D821C821B82DF91CF911F9108951F923C
:10EC30000F920FB60F9211240BB60F922F933F93A2
:10EC40004F935F936F937F938F939F93AF93BF93F4
:10EC5000EF93FF93809172110E945771209175116B
:10EC6000309176112F5F3F4F3093761120937511BD
:10EC700090917411953618F096E0909371119091DF
:10EC80007111943009F46EC0F8F4923031F1933080
:10EC900009F44CC090917311992319F0811171C03E
:10ECA0002F9AFF91EF91BF91AF919F918F917F919B
:10ECB0006F915F914F913F912F910F900BBE0F90ED
:10ECC0000FBE0F901F901895953009F457C09630DD
:10ECD00009F791E0909341124FC08111DBCF209151
:10ECE0007511309176112436310528F41092761181
:10ECF00010927511CFCF1092411210927411E091C1
:10ED0000741191E09E0F90937411F0E020917511B1
:10ED100030917611EE0FFF1FE958FE4E31832083AC
:10ED2000109276111092751193E019C0813009F09C
:10ED3000B1CFE091741191E09E0F90937411F0E0C7
:10ED40002091751130917611EE0FFF1FE958FE4E9C
:10ED500031832083109276111092751194E0909374
:10ED6000711198CF882359F2209175113091761145
:10ED70002536310508F48ECF95E0F1CF81118ACF89
:10ED8000B5CF2F988ECFCF92DF92EF92FF92CF9395
:10ED9000DF93EC01072E000C880B990B0E942DE3EA
:10EDA0006B017C0120E030E040E45FE30E948CE3F3
:10EDB00020E030E048E452E40E94A5E50E9451E6DC
:10EDC000C617D707D4F020E030E040EA5FE3C70180
:10EDD000B6010E948CE320E030E048E452E40E9457
:10EDE000A5E520E030E040E85FE30E94C7E40E9430
:10EDF00051E621E06C177D070CF420E0822F90E0B3
:10EE0000DF91CF91FF90EF90DF90CF9008950F9317
:10EE10001F93CF93DF93082F68E678E084ED90E1AD
:10EE20000E941BCFC7E0D0E010E0B8010C2E02C05A
:10EE3000759567950A94E2F76170772742E050E094
:10EE400084ED90E10E94CECE219778F7DF91CF91AB
:10EE50001F910F9108951092D40E81E08093D30EEC
:10EE60001092AE0E61E084E10E94837161E085E161
:10EE70000E948371E9EBF0E080818E7F8083808146
:10EE80008D7F808388E48093B80085E48093BC0004
:10EE90000895CF93DF9391E09093780D8823B9F094
:10EEA000C091B800D091BA008091BC008A7B809359
:10EEB000BC0060E084E10E94837160E085E10E9413
:10EEC00083710E942B77D093BA00C093B800DF9172
:10EED000CF91089585ED8093BC008091D60E9091DE
:10EEE000D70EA091D80EB091D90E0796A11DB11DD5
:10EEF00023E0B695A795979587952A95D1F7209108
:10EF0000BC0024FD03C01092D40E08954091D60E8B
:10EF10005091D70E6091D80E7091D90E452B462B8B
:10EF2000472B69F30097A105B10541F025E32A9528
:10EF3000F1F700000197A109B109E1CF8091D50E49
:10EF40000C9449771F920F920FB60F9211240BB6B3
:10EF50000F922F933F934F935F936F937F938F9372
:10EF60009F93AF93BF93EF93FF938091B900887FF6
:10EF7000803609F44DC008F040C0883209F4A9C0B9
:10EF800028F5803109F49DC0C8F4882309F4FBC03A
:10EF9000883009F496C0FF91EF91BF91AF919F9196
:10EFA0008F917F916F915F914F913F912F910F9032
:10EFB0000BBE0F900FBE0F901F901895883109F46B
:10EFC00088C0803241F78093D20E14C0803409F497
:10EFD0009DC040F48033B9F38833E9F68093D20EB4
:10EFE00085ECB0C0803509F485C0883509F496C039
:10EFF000883489F60E946A77CECF883909F48CC0AC
:10F0000038F5883729F050F4883611F0803719F632
:10F0100083E08093D40E1092BB0D57C0883809F45A
:10F020007BC0803919F0803809F0B5CF8091BB0DD5
:10F03000803208F071C0E091BB0D81E08E0F8093AB
:10F04000BB0D8091BB00F0E0E556F24F80833DC0E0
:10F05000803B39F0E0F4803A09F479C0883A09F04D
:10F060009ACF84E08093D40E10929A0D1092990D4D
:10F07000E091D30DF091D40D19958091990D8111E6
:10F080000FC081E08093990D1092790D09C0803CEA
:10F0900009F4A6CF883C09F4A3CF883B09F07BCFC5
:10F0A000E0919A0D81E08E0F80939A0DF0E0E75881
:10F0B000F24F80818093BB0090919A0D8091990DC1
:10F0C00029C08091AF0E8093BB0085EC8093BC007B
:10F0D00062CF9091D10E8091D00E981758F5E091A3
:10F0E000D10E81E08E0F8093D10EF0E0E055F14F0C
:10F0F0008081E9CFE091D10E81E08E0F8093D10E17
:10F100008091BB00F0E0E055F14F80839091D10EEB
:10F110008091D00E9817C8F285E8D8CFE091D10E33
:10F1200081E08E0F8093D10E8091BB00F0E0E0551E
:10F13000F14F80838091D30E81115CCF81E0809369
:10F14000AE0E84EA8093BC001092D40E24CF85ECDE
:10F150008093BC001092D40E8091BB0D803230F4AD
:10F16000E091BB0DF0E0E556F24F10826091BB0DCF
:10F1700070E0E091D10DF091D20D8BE99DE01995F1
:10F180001092BB0D08CF1092D20E34CF81E00C94B8
:10F1900042B10F931F93CF938C01C62FFC01848142
:10F1A0000E9432B2F8016385C62B6C2F70E08BE2AF
:10F1B00094E10E94A2148BE294E1CF911F910F91F0
:10F1C0000C94C6780F931F93CF938C01C62F0E9487
:10F1D000C9786C2F6460C8010E94C9786C2F6B7F5E
:10F1E000C8010E94C97883EC90E00197F1F7CF91B4
:10F1F0001F910F9108950F931F93CF938C01C62FEA
:10F20000607F61600E94E27880E1C89FB0011124B4
:10F210006160C8010E94E27881E090E0CF911F9187
:10F220000F910895862F642F0E943FB610925B0EB7
:10F2300080935A0E0895CF938EE10E9432B262E01D
:10F2400070E08BE294E10E94A21461E870E08BE22E
:10F2500094E10E94A2148BE294E10E94C67846E0F9
:10F2600050E06EE170E08BE294E10E9412798091AF
:10F270005A0E90915B0E891B990B069724F10E9400
:10F280002CB6C82F0E942CB620E0822B9C2B90938A
:10F29000370E8093360E0E942CB6C82F0E942CB6D3
:10F2A00020E0822B9C2B9093330E8093320E0E9491
:10F2B0002CB6C82F0E942CB620E0822B9C2B90935A
:10F2C000350E8093340ECF910895EF92FF920F93F5
:10F2D0001F93CF93DF93CDB7DEB768970FB6F8943F
:10F2E000DEBF0FBECDBF8C0162E277E0CE010D968E
:10F2F0000E9479CB67E379E0CE0143960E9479CBF7
:10F3000064E97BE1C8010E9467CBBE016D5E7F4F5F
:10F31000C8010E945BCA6BE87BE1C8010E9404CA75
:10F320008AEEE82E82E1F82EF701608170E0CE01CE
:10F3300001960E948EC8BE016F5F7F4FCE01079677
:10F340000E9470CBBE01635F7F4FCE0107960E9483
:10F35000F1C9BC01C8010E945BCACE0107960E9498
:10F36000E3CACE0101960E94E3CA6EE77BE1C801C1
:10F370000E9404CAF7016181062E000C770BCE01B2
:10F3800001960E948EC8BE016F5F7F4FCE01079627
:10F390000E9470CBBE01635F7F4FCE0107960E9433
:10F3A000F1C9BC01C8010E945BCACE0107960E9448
:10F3B000E3CACE0101960E94E3CA64E77BE1C8017B
:10F3C0000E9404CAF7016281062E000C770BCE0161
:10F3D00001960E948EC8BE016F5F7F4FCE010796D7
:10F3E0000E9470CBBE01635F7F4FCE0107960E94E3
:10F3F000F1C9BC01C8010E945BCACE0107960E94F8
:10F40000E3CACE0101960E94E3CA6CE67BE1C80123
:10F410000E9404CAF70163817481CE0101960E94A3
:10F420008EC8BE016F5F7F4FCE0107960E9470CBE2
:10F43000BE016D5E7F4FCE0107960E94F1C9BC01EF
:10F44000C8010E945BCACE0107960E94E3CACE01A2
:10F4500001960E94E3CA65E57BE1C8010E9404CAE7
:10F46000F70165817681CE0101960E948EC8BE01AA
:10F470006F5F7F4FCE0107960E9470CBBE01635F26
:10F480007F4FCE0107960E94F1C9BC01C8010E94BE
:10F490005BCACE0107960E94E3CACE0101960E9484
:10F4A000E3CA6CE47BE1C8010E9404CAF7016781EA
:10F4B000062E000C770B6F5F7F4FCE0101960E94E6
:10F4C0008EC8BE016F5F7F4FCE0107960E9470CB42
:10F4D000BE01635F7F4FCE0107960E94F1C9BC0158
:10F4E000C8010E945BCACE0107960E94E3CACE0102
:10F4F00001960E94E3CA61E47BE1C8010E9404CA4C
:10F50000F7016085062E000C770BCE0101960E9454
:10F510008EC8BE016F5F7F4FC8010E945BCACE01DB
:10F5200001960E94E3CACE0143960E94E3CACE012F
:10F530000D960E94E3CAC80168960FB6F894DEBF24
:10F540000FBECDBFDF91CF911F910F91FF90EF9034
:10F5500008954F925F926F927F928F929F92BF9287
:10F56000CF92DF92EF92FF920F931F93CF93DF938F
:10F57000CDB7DEB762970FB6F894DEBF0FBECDBF32
:10F580008EE492E00E944DE480935C0E8FE492E062
:10F590000E944DE480935D0E80915C0E90915D0E13
:10F5A0001816190664F41092EF04019741F41092B2
:10F5B0005D0E10925C0E8EE492E00E9481B440E0F9
:10F5C00052EC61E070E084ED90E10E94EA168091D7
:10F5D000EF04882331F068EE73E080E090E00E9451
:10F5E0003D7284ED90E10E9418AF182FB82E0AEEFC
:10F5F000C02E02E1D02E8CE2E82EFF24F394C70146
:10F600000E944DE4F60181936F01FFEFEF1AFF0AAC
:10F6100046E2E41642E0F40691F78091EB121816E8
:10F620001CF41D3609F011C163E97BE0CE010D9693
:10F630000E9479CB1092EA1288E18093EB1284E069
:10F640008093EC121092F1121092F21265EF7AE0B0
:10F65000CE010D960E9457C884EF92E1009739F0D1
:10F6600044E050E0BC01CE010D960E9400B581E05F
:10F670008093F81283E08093F91282E090E09093F7
:10F68000FB128093FA1285E090E09093FD12809334
:10F69000FC1262EF7AE0CE010D960E9457C88EEF01
:10F6A00092E1009739F044E050E0BC01CE010D96A4
:10F6B0000E9400B582E08093021383E080930313DD
:10F6C00082E090E0909305138093041385E090E02E
:10F6D00090930713809306136FEE7AE0CE010D9698
:10F6E0000E9457C888E093E1009739F044E050E069
:10F6F000BC01CE010D960E9400B583E080930C13EF
:10F7000080930D1382E090E090930F1380930E137B
:10F7100085E090E090931113809310136AE379E0F1
:10F72000CE010D960E9457C882E193E1009739F00F
:10F7300044E050E0BC01CE010D960E9400B585EF7B
:10F740008093161383E08093171382E090E09093E8
:10F7500019138093181385E090E090931B13809306
:10F760001A138CE291E00E9423B58091D00D88237A
:10F7700011F1CE0101960E946579BE016F5F7F4F46
:10F7800084ED90E10E94FFD3CE0101960E94E3CA6E
:10F7900062EF7BE184ED90E10E9411D42AE04AE01F
:10F7A00050E060E070E084ED90E10E9472CD84ED65
:10F7B00090E10E94BECD68EB7BE1CE0107960E94EE
:10F7C00067CBBE01695F7F4F84ED90E10E94FFD35C
:10F7D000F12CE12C8091EC12082E000C990BE8160C
:10F7E000F906A4F4B701CE0101960E94B71FBE012D
:10F7F0006F5F7F4F84ED90E10E94FFD3CE010196B1
:10F800000E94E3CA8FEFE81AF80AE4CFCE01079608
:10F810000E94E3CA8091D00D882399F062ED7BE1CC
:10F8200084ED90E10E9411D42AE04AEF50E060E0BC
:10F8300070E084ED90E10E9472CD84ED90E10E9431
:10F84000BECDCE010D960E94E3CA8091F3128111C4
:10F850008091EA128093E5120E9470726093E11227
:10F860007093E2128093E3129093E41200E0123757
:10F8700009F456C7B3E4EB2EB2E1FB2E4701D12CBD
:10F88000C12CC6010E944DE4F40181934F01FFEFAA
:10F89000CF1ADF0A48E9C416D10499F780914312C0
:10F8A00090914412A0914512B0914612853691056F
:10F8B000A105B1050CF4EDC18093EB049093EC0429
:10F8C000A093ED04B093EE048091471290914812FA
:10F8D000A0914912B0914A128093E7049093E804F2
:10F8E000A093E904B093EA0480914B1290914C12DA
:10F8F000A0914D12B0914E128093E3049093E404D2
:10F90000A093E504B093E6046091D9127091DA12E5
:10F91000072E000C880B990B0E942DE39B01AC0174
:10F920000E9413E8882321F01092DA121092D91263
:10F930006FE572E1CE0101960E9479CBBE016F5F47
:10F940007F4F86E695E10E949ECACE0101960E94F5
:10F95000E3CA6DEB72E1CE0101960E9479CBBE0144
:10F960006F5F7F4F80E695E10E949ECACE010196AF
:10F970000E94E3CA23E030E050E040E066E675E133
:10F98000CE0107960E948ACB23E030E050E040E0B1
:10F9900060E675E1CE0101960E948ACB2D813E8101
:10F9A0008B859C852817390709F589819A816F8194
:10F9B0007885009759F06115710509F002C1232B74
:10F9C00009F402C1FC01808190E00DC06115710550
:10F9D00009F4FAC0232B09F4F7C0FB01808190E001
:10F9E00091958195910901E0892B09F000E0CE0104
:10F9F00001960E94E3CACE0107960E94E3CA011154
:10FA000006C066E675E180E695E10E9487CA8091AE
:10FA10004F1290915012A0915112B09152128093B6
:10FA2000DF049093E004A093E104B093E20480919A
:10FA3000531290915412A0915512B0915612809386
:10FA4000DB049093DC04A093DD04B093DE0480918A
:10FA5000571290915812A0915912B0915A12809356
:10FA6000D7049093D804A093D904B093DA0480917A
:10FA70005B1290915C12A0915D12B0915E12809326
:10FA8000D3049093D404A093D504B093D60480916A
:10FA9000BB129091BC129093F1048093F00480917A
:10FAA000771290917812A0917912B0917A12809386
:10FAB000F6049093F704A093F804B093F9048091AE
:10FAC0008D1290918E12A0918F12B091901280930E
:10FAD000F2049093F304A093F404B093F50480919E
:10FAE000671290916812A0916912B0916A12809386
:10FAF000CF049093D004A093D104B093D20480910A
:10FB00006B1290916C12A0916D12B0916E12809355
:10FB1000CB049093CC04A093CD04B093CE04C090BA
:10FB2000C912D090CA12B6010D2C000C880B990B8B
:10FB30000E942DE39B01AC010E9413E8811104C0D7
:10FB4000D0926F0DC0926E0D4090D3125090D4128F
:10FB50006090D5127090D612A3019201C301B20138
:10FB60000E9413E8811132C04092C7045092C80429
:10FB70006092C9047092CA048091D7129091D812F1
:10FB80009093C6048093C5042091B3043091B404CB
:10FB900090E080E028173907A4F1F70140AD51AD9E
:10FBA00057FF0AC0FC01EE0FFF1FED54FB4F4081D1
:10FBB0005181F70151AF40AF0196F2E0EF0EF11C19
:10FBC000E9CF0E94EAEA0FCF01E011CF8091C7048C
:10FBD0009091C804A091C904B091CA048093D31233
:10FBE0009093D412A093D512B093D61283E090E0F4
:10FBF0009093D8128093D71290E080E00E94D6B400
:10FC0000C3CF6091671270916812809169129091D0
:10FC10006A129B01AC010E9413E881110FC0609130
:10FC20006B1270916C1280916D1290916E129B010B
:10FC3000AC010E9413E8882309F4CEC40E94DE7050
:10FC400051E9C52E52E1D52E66E4E62E6DE0F62E82
:10FC50007EE6872E7DE0972EF601419051906190CF
:10FC600071906F01A3019201C301B2010E9413E8D8
:10FC7000811105C0F7014082518262827382F4E0F3
:10FC8000EF0EF11C8E149F0439F781E090E00E9482
:10FC900099110EE8010F013009F442C51E3609F42E
:10FCA0003EC58091431290914412A0914512B091AB
:10FCB000461285369105A105B1050CF431C5809138
:10FCC000B9129091BA128D7F892B41F440E855E228
:10FCD00060E070E08DEF9EE00E94EA168091B9121C
:10FCE0009091BA12019741F440E052EC61E070E06B
:10FCF0008DEF9EE00E94EA1664E670E080E090E0FE
:10FD00000E943D728091B9129091BA12892B09F02C
:10FD1000B7C01E3671F08091431290914412A091A9
:10FD20004512B091461285369105A105B1050CF03A
:10FD3000A7C063E97BE0CE0107960E9479CB62E41D
:10FD400079E0CE0101960E9479CB60E675E1CE01A3
:10FD500001960E94F1C9BC01CE0107960E9487CA94
:10FD6000CE0101960E94E3CABE01695F7F4F8DEF0D
:10FD70009EE00E94F1D368EB7BE080E090E00E947F
:10FD80003D72BE01695F7F4FCE0101960E9470CB2C
:10FD9000CE0101960E94B71ECE0101960E94E3CAD1
:10FDA0006CE271E080E090E00E943D724091641549
:10FDB000509165154250510960E675E1CE010196FA
:10FDC0000E94EF18BE016F5F7F4FCE0107960E9421
:10FDD0009ECACE0101960E94E3CABE01695F7F4FB1
:10FDE000CE0101960E9470CBBE01695F7F4FCE01AC
:10FDF00001960E94F1C9BC01CE0107960E9487CAF4
:10FE0000CE0101960E94E3CA6AE479E0CE01019630
:10FE10000E9479CBBE01695F7F4FCE0101960E949F
:10FE2000F1C9BC01CE0107960E9487CACE01019696
:10FE30000E94E3CABE01695F7F4F8DEF9EE00E9482
:10FE4000F1D368EB7BE080E090E00E943D72BE0160
:10FE5000695F7F4FCE0101960E9470CBCE01019663
:10FE60000E94B71ECE0101960E94E3CA6CE271E0C7
:10FE700080E090E00E943D72CE0107960E94E3CAA6
:10FE8000113659F084ED90E10E9418AFB82E64E667
:10FE900070E080E090E00E943D720E947AC527E207
:10FEA000C22ED12CE12CF12C10E000E08C2D0E9410
:10FEB00032B28BE294E10E94C678811131C5C092C2
:10FEC0007C150F5F1F4F4FEFC41AD40AE40AF40ADF
:10FED00080E4C816D104E104F10441F7012B31F4A8
:10FEE0006CE679E084ED90E10E94C2CD10917C1522
:10FEF000E1E6BE1213C060EB7DE184ED90E10E946B
:10FF000011D4412F50E070E060E020E184ED90E1F9
:10FF10000E9472CD84ED90E10E94BECD8091D912F5
:10FF20009091DA12019729F4103319F487E2809343
:10FF30007C150E94EDC780E40E943CB20BEA14E0FD
:10FF400093EBE92E94E0F92EF80161918F0188E797
:10FF500095E10E94FB78E016F106B1F70E94F213DA
:10FF60000E945D1160EA7DE1CE0101960E9467CB9F
:10FF70004AE050E06FEF7FEFCE0101960E94B01A89
:10FF8000CE0101960E94E3CA60E97DE1CE010196AF
:10FF90000E9467CB44EF51E06FEF7FEFCE010196F7
:10FFA0000E941614CE0101960E94E3CA0E947AC5EF
:10FFB00064E670E080E090E00E943D72F1E6BF12DE
:10FFC000C4C481E00E946C6E81E00E94D22064E68D
:10FFD00070E080E090E00E943D726091CB127091E1
:10FFE000CC128091CD129091CE126093290D709316
:10FFF0002A0D80932B0D90932C0D0091CF12109110
:020000021000EC
:10000000D0122091D1123091D2120093250D10936D
:10001000260D2093270D3093280D9B01AC010E94E3
:1000200013E8882381F083E393EFACE8B4E4809392
:10003000290D90932A0DA0932B0DB0932C0D90E0D9
:1000400080E00E94D6B46091250D7091260D8091BC
:10005000270D9091280D9B01AC010E9413E8882385
:10006000C1F080E090E0A8ECB1E48093250D90937E
:10007000260DA093270DB093280D8093CF12909357
:10008000D012A093D112B093D21290E080E00E94DF
:10009000D6B4F89482E08093B0008093B10094E6E7
:1000A0009093B3001092B200809370007894809384
:1000B0007111109274118091721160E00E94B571FB
:1000C00063E97BE080EF93E10E9457C88091B91209
:1000D0009091BA12892B31F46CEF75E080EF93E1C7
:1000E0000E9457C88091B9129091BA12019731F4C9
:1000F00066EF75E080EF93E10E9457C88091B912D6
:100100009091BA12029731F460E076E080EF93E1CB
:100110000E9457C88091F4139091F513892BC1F078
:1001200060E675E180EF93E10E945BCA60EF73E1E6
:10013000CE0101960E9470CB4AE050E06FEF7FEF56
:10014000CE0101960E941614CE0101960E94E3CAC8
:100150008091B9129091BA12019709F05CC0CE015A
:1001600007960E94E14C8B859C85009709F449C055
:10017000EF81F8852081222309F443C0079708F412
:1001800040C06DE77DE180EF93E10E9462CABE014D
:10019000695F7F4F80EF93E10E945BCA60EF73E17C
:1001A000CE0101960E9470CBCE0101960E94BE1333
:1001B000CE0101960E94E3CA64E77DE1CE0101967B
:1001C0000E9467CB48EC50E06FEF7FEFCE010196C5
:1001D0000E94F719CE0101960E94E3CABE01695F31
:1001E0007F4FCE0101960E9470CB48EC50E06FEF3C
:1001F0007FEFCE0101960E941614CE0101960E9457
:10020000E3CA68EE73E080E090E00E943D72CE01A8
:1002100007960E94E3CA67E57DE180EF93E10E94C3
:1002200062CA68E379E0CE0101960E9479CB60E66C
:1002300075E1CE0101960E94F1C960EF73E10E9461
:10024000F1C9BC0180EF93E10E9487CACE010196FB
:100250000E94E3CA60EF73E1CE0101960E9470CB69
:10026000CE0101960E94BE13CE0101960E94E3CA00
:1002700063E97BE080EF93E10E9457C864E670E099
:1002800080E090E00E943D7283E090E09093450D05
:100290008093440D8CE40E946BB56B017C0162E39A
:1002A00070E080E090E00E943D72A7019601C701D6
:1002B000B6010E9413E88823B9F086E60E946BB568
:1002C0006B017C0162E370E080E090E00E943D728F
:1002D000A7019601C701B6010E9413E8882321F007
:1002E0001092450D1092440D8091440D9091450D52
:1002F000039709F02FC362E47DE1CE0101960E94CD
:1003000067CBCE0101960E94B71ECE0101960E94D6
:10031000E3CA83E0809314140E947AC580ED0E94A2
:100320000EB7853509F039C38AEA0E9431B7909338
:100330001614809315148CEA0E9431B79093181408
:10034000809317148EEA0E9431B790931A14809309
:10035000191480EB0E9431B79093261480932514D2
:1003600082EB0E9431B7909328148093271484EB7A
:100370000E9431B790932A148093291486EB0E942F
:1003800031B790931C1480931B1488EB0E9431B7F3
:1003900090931E1480931D148AEB0E9431B79093A2
:1003A000201480931F148CEB0E9431B79093221479
:1003B000809321148EEB0E9431B790932414809384
:1003C000231469E07DE180EF93E10E9462CA0E94FC
:1003D00076B70E942DE30E9451E60E942DE320E0B3
:1003E00030E048EC52E40E94A5E5AB01BC0122E0FC
:1003F000CE0101960E94EBCABE016F5F7F4FCE0116
:1004000007960E9470CB63EC79E0CE0107960E94BC
:10041000DBC9BC0180EF93E10E945BCACE01079665
:100420000E94E3CACE0101960E94E3CA60EF73E125
:10043000CE0101960E9470CBCE0101960E94B71E9C
:10044000CE0101960E94E3CA63EF7CE180EF93E165
:100450000E9462CA6091EB047091EC048091ED04FB
:100460009091EE040E942DE320E030E048EC52E44D
:100470000E94A5E5AB01BC0122E0CE0101960E94DD
:10048000EBCABE016F5F7F4FCE0107960E9470CB13
:1004900063EC79E0CE0107960E94DBC9BC0180EFD6
:1004A00093E10E945BCACE0107960E94E3CACE0187
:1004B00001960E94E3CA60EF73E1CE0101960E94AB
:1004C00070CBCE0101960E94B71ECE0101960E940C
:1004D000E3CA64E670E080E090E00E943D728091A3
:1004E000440D9091450D892BA1F461E08091A60403
:1004F0000E94B57160E08091A4040E94B571609182
:10050000A0047091A1048091A2049091A3040E9480
:10051000401160E08091A6040E94B5718091EF04C3
:10052000882331F068EE73E080E090E00E943D7235
:1005300062EF7AE08CEF93E10E9457C882E090E08E
:100540009093430D8093420D8091EF04882309F42A
:1005500075C369EB7CE1CE0101960E9467CB4CE24A
:1005600051E06FEF7FEFCE0101960E941614CE018D
:1005700001960E94E3CA60919E0470919F0480914D
:10058000F0049091F1040E94A91484E1C82ED12CAA
:10059000E12CF12C10E000E00F5F1F4FC701B60106
:1005A0000E943D7260919E0470919F048091F004BE
:1005B0009091F1040E94A914033011053CF00A3017
:1005C00011050CF0FBC1892B09F4FBC144E1C40EF9
:1005D000D11CE11CF11CE0CF70906F12672D072C2D
:1005E000000C770B880B990B0E942DE39B01AC014B
:1005F0000E9413E8811122CB8090701290907112AA
:10060000B401092C000C880B990B0E942DE39B016F
:10061000AC010E9413E8811111CB00917212602F7E
:10062000002E000C770B880B990B0E942DE39B0189
:10063000AC010E9413E8811101CBC0907312D090DD
:100640007412E0907512F0907612A7019601C7011E
:10065000B6010E9413E88111F1CA6091771270917E
:1006600078128091791290917A129B01AC010E94CC
:1006700013E88111E3CA60918D1270918E128091FE
:100680008F12909190129B01AC010E9413E881118E
:10069000D5CA6091B9127091BA12072E000C880B5E
:1006A000990B0E942DE39B01AC010E9413E881117C
:1006B000C5CA6091BB127091BC12072E000C880B4A
:1006C000990B0E942DE39B01AC010E9413E881115C
:1006D000B5CA6091C9127091CA12072E000C880B1E
:1006E000990B0E942DE39B01AC010E9413E881113C
:1006F000A5CA43E047150CF4A1CA05300CF09ECA08
:100700008BEF881691040CF099CA20E030E0A90123
:10071000C701B6010E9426E387FD90CA91CA0CEF7B
:100720008091EB049091EC04A091ED04B091EE0463
:100730008093431290934412A0934512B0934612B3
:100740008091E7049091E804A091E904B091EA0453
:100750008093471290934812A0934912B0934A1283
:100760008091E3049091E404A091E504B091E60443
:1007700080934B1290934C12A0934D12B0934E1253
:10078000133751F160E086E695E10E942ECA60E0E1
:1007900080E695E10E942ECA40916A1550916B1532
:1007A0004115510549F08FE592E1009729F0BC0110
:1007B00086E695E10E9400B540916415509165155B
:1007C0004115510549F08DEB92E1009729F0BC01EC
:1007D00080E695E10E9400B58091DF049091E004ED
:1007E000A091E104B091E20480934F1290935012D3
:1007F000A0935112B09352128091DB049091DC04CB
:10080000A091DD04B091DE048093531290935412B2
:10081000A0935512B09356128091D7049091D804AA
:10082000A091D904B091DA04809357129093581292
:10083000A0935912B0935A128091D3049091D4048A
:10084000A091D504B091D60480935B1290935C1272
:10085000A0935D12B0935E1290E080E00E94D6B447
:10086000E6E4FDE0A1E9B2E141915191619171911C
:100870004D935D936D937D934DE0EE36F407A1F7B4
:100880006FEB7DE1CE0101960E9467CBCE01019610
:100890000E94B71ECE0101960E94E3CA33EBC32E1D
:1008A00034E0D32E4BE7842E42E1942EF12CE12C40
:1008B0008091B3049091B4048E159F054CF1F6011C
:1008C000819191916F01F401819391934F018091F6
:1008D000D00D8823C9F068E379E084ED90E10E94AF
:1008E0001BCF4AE050E0B70184ED90E10E94CECEEC
:1008F0006DE379E084ED90E10E941BCFF601329721
:10090000808191810E9408CFFFEFEF1AFF0AD0CFBC
:10091000023008F0D4C990E080E00E94D6B4CFC97C
:10092000843009F0D0CA61E579E084ED90E10E945D
:100930001BCF20E1B701A60184ED90E10E9472CDAA
:1009400084ED90E10E94BECDBECA80E00E946C6E34
:1009500080E03BCB86E00E9491C5BC0190E080E046
:100960000E942BE32AE037ED43EA5CE30E948CE32C
:1009700023E333E948E853E40E94C6E420E030E092
:1009800048E453E40E9426E387FFC3CC82E090E072
:100990009093AA048093A904BCCC6CE17DE1CE01C4
:1009A00001960E9467CBCE0101960E94BE13CE0134
:1009B00001960E94E3CA1092A8048BCD892B09F0FE
:1009C000EAC18091F0049091F1048B30910509F017
:1009D00092C18091871490918814A0918914B0914C
:1009E0008A1480933E0D90933F0DA093400DB093D9
:1009F000410D8091831490918414A0918514B0913D
:100A0000861480933A0D90933B0DA0933C0DB093C8
:100A10003D0D40913E0D50913F0D6091400D709104
:100A2000410D21E0CE0101960E94EBCA60E976E01B
:100A3000CE0107960E9479CBBE016F5F7F4FCE013A
:100A400007960E94F1C9BC0180EF93E10E9487CA1A
:100A5000CE0107960E94E3CACE0101960E94E3CA26
:100A600040913A0D50913B0D60913C0D70913D0DC0
:100A700021E0CE0101960E94EBCA6AE678E0CE0141
:100A800007960E9479CBBE016F5F7F4FCE0107961C
:100A90000E94F1C9BC0180EF93E10E945BCACE01C4
:100AA00007960E94E3CACE0101960E94E3CA6CE356
:100AB00078E080EF93E10E9451CA63E97BE0CE01C8
:100AC00001960E9479CB44E150E070E060E0CE01F5
:100AD00001960E94B01ACE0101960E94E3CAC0900E
:100AE0003E0DD0903F0DE090400DF090410D20E084
:100AF00030E0A901C701B6010E94AEE620E030E077
:100B000040E05FE387FD17C1C701B6010E94C7E45B
:100B10000E9451E6AB01BC01CE0101960E9461C862
:100B2000BE016F5F7F4F8AEE93E10E949ECACE01A5
:100B300001960E94E3CA60E087E00E944DB26AEE2F
:100B400073E188E795E10E94F1D36FED88E795E1C5
:100B50000E94D4CD60E778E088E795E10E941BCF42
:100B600060913A0D70913B0D80913C0D90913D0D3F
:100B70000E9451E64AE050E088E795E10E94CECE1F
:100B80006CE378E088E795E10E941BCF64E670E0B3
:100B900080E090E00E943D72C0903E0DD0903F0DED
:100BA000E090400DF090410D20E030E040EF51E446
:100BB000C701B6010E94AEE66AEA7CE187FF28C061
:100BC00020E030E040ED51E4C701B6010E94AEE6FE
:100BD00087FDB6C06AE97CE1CE0101960E9467CB31
:100BE0004AE050E06FEF7FEFCE0101960E941614AD
:100BF000CE0101960E94E3CA8091EF04882331F070
:100C00006CED75E080E090E00E943D726AE87CE166
:100C1000CE0101960E9467CB4AE050E06FEF7FEF74
:100C2000CE0101960E941614CE0101960E94E3CADD
:100C300062E370E080E090E00E943D726BED7CE149
:100C400080EF93E10E9462CA68E379E0CE010196E9
:100C50000E9479CB60E675E1CE0101960E94F1C950
:100C600060EF73E10E94F1C9BC0180EF93E10E9443
:100C700087CACE0101960E94E3CA60EF73E1CE01FC
:100C800001960E9470CBCE0101960E94BE13CE0148
:100C900001960E94E3CA67EC7CE180EF93E10E9439
:100CA00062CA60EF73E1CE0101960E9470CBCE0163
:100CB00001960E94BE13CE0101960E94E3CA63E929
:100CC0007BE080EF93E10E9457C862960FB6F894DC
:100CD000DEBF0FBECDBFDF91CF911F910F91FF906F
:100CE000EF90DF90CF90BF909F908F907F906F900C
:100CF0005F904F9008958631910509F46ACE0C9764
:100D000009F087CE8091310D9091320DA091330D75
:100D1000B091340D80933E0D90933F0DA093400D04
:100D2000B093410D80912D0D90912E0DA0912F0D1E
:100D3000B091300D66CEC701B6010E94C6E4E8CE80
:100D400020E030E040EB51E4C701B6010E94AEE67E
:100D50006CE77CE187FF5CCF6DE67CE1CE0101961C
:100D60000E9467CB4AE050E06FEF7FEFCE01019623
:100D70000E941614CE0101960E94E3CA8091EF04EE
:100D8000882331F06CED75E080E090E00E943D72C8
:100D90006FE57CE13DCF0E94F2136EE170E080E0F0
:100DA00090E00E943D720E943DB96B017C0164E6B7
:100DB00070E080E090E00E943D7260E976E080EFB4
:100DC00093E10E9457C821E0B701A601CE01019628
:100DD0000E94EBCABE016F5F7F4F80EF93E10E94DC
:100DE0005BCACE0101960E94E3CA60EF73E1CE01B7
:100DF00001960E9470CB4AE050E070E060E0CE01C6
:100E000001960E94B01ACE0101960E94E3CA809119
:100E10009D04882379F08091FB04882359F06FEDBD
:100E200088E795E10E94D4CD6FEE78E088E795E100
:100E30000E941BCF68EB76E080EF93E10E9451CADD
:100E4000C0923E0DD0923F0DE092400DF092410DC8
:100E500020E030E040EF51E4C701B6010E94AEE669
:100E60006FE47CE187FF28C020E030E040ED51E4F2
:100E7000C701B6010E94AEE687FD3EC06FE37CE18C
:100E8000CE0101960E9467CB4AE050E06FEF7FEF02
:100E9000CE0101960E941614CE0101960E94E3CA6B
:100EA0008091EF04882331F06CED75E080E090E0F4
:100EB0000E943D726FE27CE1CE0101960E9467CBF9
:100EC0004AE050E06FEF7FEFCE0101960E941614CA
:100ED000CE0101960E94E3CA6CE271E080E090E0EE
:100EE0000E943D728091EF04882309F4A7CE68EE3A
:100EF00073E080E090E0A0CE20E030E040EB51E4F1
:100F0000C701B6010E94AEE661E27CE187FFD4CF63
:100F100062E17CE1CE0101960E9467CB4AE050E09D
:100F20006FEF7FEFCE0101960E941614CE0101965D
:100F30000E94E3CA8091EF04882331F06CED75E0E4
:100F400080E090E00E943D7264E07CE1B5CFBF920A
:100F5000CF92DF92EF92FF920F931F93CF93DF9385
:100F6000CDB7DEB762970FB6F894DEBF0FBECDBF28
:100F70008C016B0163E97BE00E9479CB1092EE0C4F
:100F800063E97BE0CE010D960E9479CBFF24F394B8
:100F900084ED90E10E943AAF2091EE0C18161906EC
:100FA0007CF521112DC084ED90E10E9418AF8A30AC
:100FB00009F07FC089899A89892B09F482C0F0924F
:100FC000EE0C62E879E0CE0107960E9479CBBE0173
:100FD000635F7F4FCE0107960E94F1C9BC01CE012D
:100FE00001960E9470CBCE0101960E94B71ECE01E1
:100FF00001960E94E3CACE0107960E94E3CA61C02F
:10100000F12CE12CBB24B394222309F461C089891B
:101010009A89019709F045C063E477E0CE01019613
:101020000E9479CBBE016F5F7F4FCE010D960E946B
:10103000C0C9F12C811115C064EF78E0CE0107968C
:101040000E9479CBBE01695F7F4FCE010D960E9451
:10105000C0C9FF24F3948111F12CCE0107960E94A0
:10106000E3CACE0101960E94E3CAFF20A1F050E03E
:1010700040E0BE01635F7F4FCE0101960E94EF18F2
:10108000BE016F5F7F4F8CEF93E10E949ECACE013D
:1010900001960E94E3CA64E170E080E090E00E9463
:1010A0003D72BE01635F7F4FCE0101960E945ECB11
:1010B00091C08D3009F47ECF682FCE010D960E942D
:1010C0002ECA6AE070E080E090E00E943D7260CF3E
:1010D0008DEF9EE00E943AAF1816190614F58DEFB9
:1010E0009EE00E9418AF8A30A9F08D3099F090915F
:1010F000EE0C91110FC0682FCE010D960E942ECAE2
:101100008FEFE81AF80A65E070E080E090E00E9456
:101110003D72DECF89899A89892BA9F3B092EE0CB2
:10112000F2CF64E170E080E090E00E943D72EF2831
:10113000D1F189899A89892BB1F18091D00D8823C9
:1011400061F168E379E0CE0101960E9479CBBE019E
:101150006F5F7F4FCE010D960E94C0C9F82ECE0161
:1011600001960E94E3CAF11018C06BE879E084EDA3
:1011700090E10E941BCFBE01635F7F4FCE010196BD
:101180000E9470CBBE016F5F7F4F84ED90E10E94A3
:10119000FFD3CE0101960E94E3CA64E170E080E0D3
:1011A00090E00E943D7289899A892091EE0C21116C
:1011B00030CF009709F02DCF64E670E080E090E03A
:1011C0000E943D720E94707263E97BE0CE0101963D
:1011D0000E9479CBCE010D960E94E3CABE016F5FDB
:1011E0007F4FC8010E94D7CACE0101960E94E3CA70
:1011F000F80184819581892B79F4B601CE0101969D
:101200000E949D6DBE016F5F7F4FC8010E94D7CACB
:10121000CE0101960E94E3CAF80184819581892B51
:1012200079F4B601CE0101960E94356CBE016F5F64
:101230007F4FC8010E94D7CACE0101960E94E3CA1F
:10124000C80162960FB6F894DEBF0FBECDBFDF9126
:10125000CF911F910F91FF90EF90DF90CF90BF90B3
:1012600008954F925F926F927F929F92AF92BF923A
:10127000CF92DF92EF92FF920F931F93CF93DF9362
:10128000CDB7DEB7A8970FB6F894DEBF0FBECDBFBF
:10129000BC0188E094E10E9487CA0E9413C76FEBEB
:1012A00079E0CE0101960E9479CBBE016F5F7F4F3E
:1012B00088E094E10E94C0C9182FCE0101960E94D7
:1012C000E3CA112309F4F8C0809112149091131409
:1012D0004097C0F0F12C8F2DA8960FB6F894DEBF82
:1012E0000FBECDBFDF91CF911F910F91FF90EF9077
:1012F000DF90CF90BF90AF909F907F906F905F9066
:101300004F90089542E050E06EE074E1CE01019606
:101310000E94EF18BE016F5F7F4F8AEE93E10E943B
:101320009ECACE0101960E94E3CA6AEE73E1CE0125
:1013300001960E9470CBCE0101960E94B71ECE018D
:1013400001960E94E3CA8AEE93E10E94C9C820E098
:1013500030E048EC52E40E948CE30E9451E6AB017D
:10136000BC014093EB045093EC046093ED04709344
:10137000EE04CE0101960E9461C8CE0101960E9442
:10138000B71ECE0101960E94E3CA6091EB047091F2
:10139000EC048091ED049091EE048B019C010059C6
:1013A0001F452140310901341C4921053105C8F18F
:1013B00062E979E0CE0101960E9479CB6AEE73E191
:1013C000CE0101960E94F1C965EA79E00E94DBC96D
:1013D000BC0180EF93E10E9487CACE0101960E9472
:1013E000E3CA68E379E0CE0101960E9479CB60EF11
:1013F00073E1CE0101960E94F1C9BC01CE01459670
:101400000E9470CBCE0145960E94BE13CE01459638
:101410000E94E3CACE0101960E94E3CA1092000521
:1014200048C21A821982FE01339626E0DF011D921E
:101430002A95E9F70E942DE320E030E048EC52E4E1
:101440000E94A5E58E010F5F1F4F22E047E00E943A
:1014500077DEBC0180EF93E10E94BAC865EB79E0CA
:10146000CE0145960E9479CB60EF73E1CE0145969F
:101470000E94F1C962EC79E00E94DBC9BC0180EFF7
:1014800093E10E9487CACE0145960E94E3CA8091EB
:10149000EB049091EC04A091ED04B091EE048093E4
:1014A000431290934412A0934512B093461290E0D9
:1014B00080E00E94D6B495CF8E010B5E1F4F66E28E
:1014C0007AE1C8010E9467CBB80188E094E10E94EC
:1014D000C0C9FF24F394811116C061E27AE1CE0104
:1014E00001960E9467CBBE016F5F7F4F88E094E159
:1014F0000E94C0C9FF24F394811101C0F12CCE01D8
:1015000001960E94E3CAC8010E94E3CAFF2009F4C1
:1015100071C042E050E06EE074E1CE0101960E949D
:10152000EF18BE016F5F7F4F8AEE93E10E949ECA63
:10153000CE0101960E94E3CA6CE17AE1CE010196E8
:101540000E9467CBBE016F5F7F4F88E094E10E94ED
:10155000C0C9E82ECE0101960E94E3CAEE2099F0A0
:1015600044E050E06EE074E1CE0101960E94EF1875
:10157000BE016F5F7F4F8AEE93E10E949ECACE014B
:1015800001960E94E3CA8AEE93E10E94D4C86730B4
:10159000710558F570936F0D60936E0D80916E0D0F
:1015A00090916F0D9093CA128093C91290E080E0E1
:1015B0000E94D6B468E379E0CE0101960E9479CB0F
:1015C00060EF73E1CE0101960E94F1C9BC01C80130
:1015D0000E9470CBC8010E94BE13C8010E94E3CADA
:1015E000CE0101960E94E3CA76CE10926F0D109242
:1015F0006E0DD4CF67E17AE1CE0101960E9467CBF0
:10160000BE016F5F7F4F88E094E10E94C0C9F82E51
:10161000CE0101960E94E3CAFF20A1F126E030E04E
:1016200044E050E06EE074E1CE0101960E948ACB66
:10163000BE016F5F7F4F8AEE93E10E949ECACE018A
:1016400001960E94E3CA8AEE93E10E94D4C8709387
:10165000BC126093BB127093F1046093F0046EE0CF
:1016600074E1CE0101960E9470CBCE0101960E94DA
:10167000B71ECE0101960E94E3CA90E080E00E946E
:10168000D6B4CCCE60E17AE1CE0101960E9467CB60
:10169000BE016F5F7F4F88E094E10E94C0C9F82EC1
:1016A000CE0101960E94E3CAFF20A1F146E050E07E
:1016B0006EE074E1CE0101960E94EF18BE016F5FEB
:1016C0007F4F8AEE93E10E949ECACE0101960E944E
:1016D000E3CA8091EE139091EF13892B61F08AEEAB
:1016E00093E10E94C9C86093A0047093A104809301
:1016F000A2049093A3046EE074E1CE0101960E94CF
:1017000070CBCE0101960E94B71ECE0101960E94B9
:10171000E3CA84CE67EC79E0CE0101960E9479CBD2
:10172000BE016F5F7F4F88E094E10E94C0C9F82E30
:10173000CE0101960E94E3CAFF2009F4BDC06CE00F
:101740007AE1CE0101960E9467CBBE016F5F7F4FA9
:1017500088E094E10E94C0C9F82ECE0101960E9453
:10176000E3CAFF20D1F184E090E00E94E41060938E
:10177000CF047093D0048093D1049093D2046CEF83
:1017800079E180EF93E10E9462CA4091CF045091C9
:10179000D0046091D1047091D20422E0CE01019670
:1017A0000E94EBCABE016F5F7F4F80EF93E10E9402
:1017B0005BCACE0101960E94E3CA8091CF0490914A
:1017C000D004A091D104B091D20480936712909379
:1017D0006812A0936912B0936A126AEC79E0CE01A4
:1017E00001960E9479CBBE016F5F7F4F88E094E144
:1017F0000E94C0C9F82ECE0101960E94E3CAFF20C4
:10180000F1F18AE090E00E94E4106093CB047093C1
:10181000CC048093CD049093CE046BEE79E180EFFD
:1018200093E10E9462CA4091CB045091CC04609134
:10183000CD047091CE0422E0CE0101960E94EBCA45
:10184000BE016F5F7F4F80EF93E10E945BCACE01C4
:1018500001960E94E3CA8091CB049091CC04A091A0
:10186000CD04B091CE0480936B1290936C12A09330
:101870006D12B0936E1290E080E00E94D6B468E3DF
:1018800079E0CE0101960E9479CB60EF73E1CE0141
:1018900001960E94F1C9BC01C8010E9470CBC80129
:1018A0000E94BE13C8010E94E3CACE0101960E94A5
:1018B000E3CAFF24F3940FCD6EEB78E0CE010196DE
:1018C0000E9479CBBE016F5F7F4F88E094E10E9458
:1018D000C0C9F82ECE0101960E94E3CAFF2009F488
:1018E000BDC080911214909113140797F8F046E050
:1018F00050E06EE074E1CE0101960E94EF18BE0147
:101900006F5F7F4F8AEE93E10E949ECACE010196DF
:101910000E94E3CA8AEE93E10E94C9C86093F6046C
:101920007093F7048093F8049093F90480918D04E8
:1019300090918E0499270E94A5122DE038E643E588
:101940005BE30E948CE36B017C01209129053091BF
:101950002A0540912B0550912C050E9426E318166C
:101960000CF460C06091110570911205809113050F
:101970009091140520E030E048EC52E40E948CE3A2
:101980006B017C0120E030E0A9010E9426E31816DB
:1019900034F0C12CD12CF8EAEF2EF1E4FF2EC092E6
:1019A000F604D092F704E092F804F092F904C092A1
:1019B0007712D0927812E0927912F0927A12809196
:1019C000D00D882381F069ED79E184ED90E10E94EA
:1019D00011D46091F6047091F7048091F80490910D
:1019E000F9040E94BFCE90E080E00E94D6B46FEC74
:1019F00079E180EF93E10E9462CA4091F604509130
:101A0000F7046091F8047091F90422E0CE01019688
:101A10000E94EBCABE016F5F7F4F80EF93E10E948F
:101A20005BCAA6C020913D0530913E0540913F051F
:101A300050914005C701B6010E94AEE687FF05C080
:101A4000C701B6010E94A4B395CF6091250570919E
:101A5000260580912705909128058CCF6BEC79E1C4
:101A6000CE0101960E9467CBBE016F5F7F4F88E079
:101A700094E10E94C0C9F82ECE0101960E94E3CAEB
:101A8000FF2009F47DC070908B0460E0872D0E94D8
:101A9000B571E9E1AE2EB12CC12CD12C7601872D88
:101AA0000E94F571BC01990F880B990B0E942DE3E0
:101AB0009B01AC01C701B6010E94C7E46B017C0128
:101AC0006AE070E080E090E00E943D72B1E0AB1A05
:101AD000B10829F720E030E040EA50E4C701B60140
:101AE0000E948CE320E030EC4FE754E40E94A5E52F
:101AF00020E030E048EC51E40E94A5E56093F20458
:101B00007093F3048093F4049093F50460938D1222
:101B100070938E1280938F129093901290E080E0D9
:101B20000E94D6B468EB79E180EF93E10E9462CA2B
:101B30004091F2045091F3046091F4047091F50423
:101B400022E0CE0101960E94EBCABE016F5F7F4F7B
:101B5000C8010E9470CB69E078E0C8010E94DBC92F
:101B6000BC0180EF93E10E945BCAC8010E94E3CAF6
:101B7000CE0101960E94E3CA60EF73E10C948C974A
:101B800064EC78E0CE0101960E9479CBBE016F5FD4
:101B90007F4F88E094E10E94C0C9F82ECE010196E3
:101BA0000E94E3CAFF2009F441C080917212082EFE
:101BB000000C990B0197039790F589E390E00E9440
:101BC000A5122AE137E64CE950E40E948CE36093C9
:101BD000731270937412809375129093761290E042
:101BE00080E00E94D6B467E979E180EF93E10E943A
:101BF00062CA409173125091741260917512709183
:101C0000761222E0CE0101960E94EBCABE016F5F00
